:020000040800F2
:1000000000090020B1010008952300084D230008D5
:10001000752300084D2300086D230008B301000874
:10002000B3010008B3010008B3010008313400082F
:10003000B3010008B3010008B3010008B3010008D0
:10004000B3010008B3010008B3010008B3010008C0
:10005000B3010008B301000889410008B14100085C
:10006000D94100080142000829420008B3010008F4
:10007000B3010008B3010008B3010008B301000890
:10008000B3010008B3010008B30100080123000810
:100090002D2300083D230008B30100085142000849
:1000A000B3010008B3010008B3010008B301000860
:1000B00025430008B3010008B3010008B30100089C
:1000C000B3010008B3010008B3010008B301000840
:1000D000B3010008B3010008B3010008B301000830
:1000E000B5420008B3010008B3010008B3010008DD
:1000F000B3010008B3010008B3010008B301000810
:10010000B3010008B3010008B3010008B3010008FF
:10011000B3010008B3010008B3010008B3010008EF
:10012000B3010008B3010008B3010008B3010008DF
:10013000B3010008B3010008B3010008B3010008CF
:10014000B3010008B3010008B3010008B3010008BF
:10015000B3010008B3010008B3010008B3010008AF
:10016000B3010008B3010008B3010008B30100089F
:10017000B3010008B3010008B3010008B30100088F
:10018000B3010008B3010008B3010008B30100087F
:10019000B3010008B3010008B3010008B30100086F
:1001A000010F000800000000000000000000000037
:1001B00002E000F000F8FEE772B6374880F30888E6
:1001C000364880F3098836483649086040F2000016
:1001D000CCF200004EF63471CEF200010860BFF39D
:1001E0004F8FBFF36F8F40F20000C0F2F0004EF669
:1001F0008851CEF200010860BFF34F8FBFF36F8FBD
:100200004FF00000E1EE100A4EF63C71CEF2000114
:100210000860062080F31488BFF36F8F03F0D0FDD1
:1002200003F052FE4FF055301F491B4A91423CBF2C
:1002300041F8040BFAE71D49184A91423CBF41F8C6
:10024000040BFAE71A491B4A1B4B9A423EBF51F86E
:10025000040B42F8040BF8E700201849184A9142B1
:100260003CBF41F8040BFAE703F0AEFD03F07EFE5D
:10027000144C154DAC4203DA54F8041B8847F9E7D7
:1002800000F042F8114C124DAC4203DA54F8041B52
:100290008847F9E703F096BD00090020001100200F
:1002A0000000000808ED00E0000100200009002027
:1002B00028450008001100207C110020801100203A
:1002C000043B0020A0010008A4010008A4010008CC
:1002D000A40100082DE9F04F2DED108AC1F80CD0D3
:1002E000C3689D46BDEC108ABDE8F08F002383F300
:1002F00011882846A047002003F00AFAFEE703F021
:1003000093F900DFFEE70000F8B500F00BFE03F004
:10031000F9FC074603F04AFD0646C0BB274B9F4247
:1003200035D001339F4235D0254B27F0FF029A424A
:1003300033D1F8B200F03AFC354642F2107400F0C6
:100340003BFC08B10024254601F0E2F848B3032045
:1003500000F03AF80024254636B11A4B9F4203D0EC
:1003600003F01CFD00242546002003F0D5FC0DB150
:1003700000F040F800F054FC02F014F80546ACB967
:1003800000F096FC4FF47A7003F0C8F9F7E73546B1
:100390000024D4E704460125D1E705464FF47A74DA
:1003A000CDE7B4F57A7F08BF0125D5E701F0FAFF64
:1003B000431BA342E4D900F01DF8DDE7010007B0BC
:1003C000000008B0263A09B0084B187003280CD872
:1003D000DFE800F008050208022000F001BE02205C
:1003E00000F0F4BD024B00225A60704780110020DB
:1003F0008411002010B501F08BF830B1234B03229B
:100400001A70234B00225A6010BD224B224A1C4610
:1004100019680131F8D004339342F9D16268A242DD
:10042000F2D31E4B9B6803F1006303F520439A420D
:10043000EAD203F085FC03F097FC002000F08CFD6D
:100440000220FFF7C1FF164B9A6D00229A65996F43
:100450009A67996FD96DDA65D96FDA67D96F196EB6
:100460001A66D3F88010C3F88020D3F8803072B6B3
:100470004FF0E0233021C3F8084DD4E9003281F376
:1004800011889D4683F308881047BDE7801100203E
:100490008411002000A0000820A000080011002006
:1004A00000100240094A136849F2690099B21B0C16
:1004B00000FB01331360064B186844F2506182B2AE
:1004C000000C01FB0200186080B27047141100207C
:1004D0001011002010B500211022044600F09AFDF2
:1004E000034B03CB206061601868A06010BD00BFA3
:1004F0009075FF1FF0B5ADF5517D6EAC4FF4C47231
:1005000007460D462046002100F084FD01F04AFF19
:10051000264B4FF47A72B0FBF2F0186093E80700B4
:10052000022384E807000DF5ED702382FFF7D2FF68
:1005300042F204631E49238407A803F08FFF1D23A2
:1005400084F832310DF2EB2207AB0DF1340C1E466C
:1005500003CE664510605160334602F10802F6D1C1
:1005600030681060337913710FAE31460122204696
:1005700000F09CFD00230393AB7E029305F1190369
:10058000019380B20123CDE904600093E97E05A3C5
:10059000D3E90023384602F01BFB0DF5517DF0BD79
:1005A000AFF300809E6AC421818A46EE8C11002040
:1005B0006C4400082DE9F0412C4C237ADAB08046D7
:1005C0000D465BBB27A9284600F096FE074600288B
:1005D00042D19DF89D60C82E3ED801464FF4A662D8
:1005E000204600F017FD4FF48073C4F8F8314FF443
:1005F0000073C4F80C334FF44073C4F8203432460F
:100600000DF19E0104F1090000F0F2FC26449DF872
:100610009C30777223720BB9EB7E2372812200210A
:1006200006AC27A800F0F6FC0122214627A800F01E
:10063000A9FE00230393AB7E029305F1190380B258
:1006400001932823CDE904400093E97E05A3D3E973
:100650000023404602F0BCFA5AB0BDE8F08100BF6A
:10066000AFF3008026417272DF25D7B7D421002076
:10067000F0B5254E4FF48A7505FB0065F1B096F88C
:10068000D83085F8DC300024D822214685F8E840AF
:100690003AA800F0BFFC06F1090000F0B3FCD5F861
:1006A000E4308DF8F000C2B206AF06F109010DF199
:1006B000F100CDE93A3400F09BFC394601223AA81A
:1006C00000F096FE80B2CDE9047008230127CDE941
:1006D000023706F1D803019330230093317A0B4897
:1006E00007A3D3E9002302F073FAA04206DD01F06C
:1006F00059FEC5F8E000384671B0F0BD2046FBE772
:1007000078F6339F93CACD8DD4210020A4210020F8
:100710002DE9F0411D4D1E4E1E4F86B0284602F0B9
:1007200083FA034658B30024CDE90344ADF81440DE
:10073000027B8DF8142099684068029403AA03C2D2
:100740001B68DFF8548043F00043029301F02CFE55
:10075000821941F10003009402A9384601F0C0F863
:10076000A04205DD284602F063FA88F80040D5E78C
:1007700098F80030072B05D8013388F8003006B010
:10078000BDE8F081014802F053FAF8E7A421002007
:1007900040420F00102700200927002070B50D46A9
:1007A00014461E4602F070F950B9022E10D1012CE9
:1007B0000ED112A3D3E90023C5E90023012007E0ED
:1007C000282C10D005D8012C09D0052C0FD00020E2
:1007D00070BD302CFBD10BA3D3E90023ECE70BA3B6
:1007E000D3E90023E8E70BA3D3E90023E4E70BA355
:1007F000D3E90023E0E700BFAFF30080401DA12054
:1008000026812A0B78F6339F93CACD8D9E6AC42128
:10081000818A46EE26417272DF25D7B7F017304A3B
:1008200039059E5638B505460E4C0021013500F0BD
:10083000B5FBA4F82C55B4F82C0500F097FB78B163
:10084000B4F82C0500F0A2FB014648B9B4F82C0519
:1008500000F0A4FBB4F82C350133A4F82C35EAE7FA
:1008600038BD00BFD421002010B50A4B0A4A1A60D7
:1008700003F5805393F870203AB9DC6E2CB1204612
:1008800000F0C4FE204601F001F8BDE81040034826
:1008900000F0BCBE10270020C844000868370020C4
:1008A0002DE9F04F8FB000AF05460C4602F0ECF892
:1008B00000284BD1237E022B1BD1E38A012B18D1B8
:1008C00001F070FD0646FFF7EDFD03464FF4C870DA
:1008D000DFF8D482B3FBF0F206F5167602FB103394
:1008E00016FA83F3C8F80030E37E33B9A74B002231
:1008F0001A703C37BD46BDE8F08F07F12401204651
:1009000000F0AEFC0028F4D107F11400FFF7E2FD7F
:1009100097F8264007F11401224607F1270003F05B
:100920006BFD0028E2D10F2C08D8984B1C70D8F82A
:100930000030A3F51673C8F80030DAE797F82410F2
:100940000029D6D0284602F097F8D2E7E38A282B70
:1009500033D010D8012B2BD0052BCAD1BFF34F8F2A
:100960008B498C4BCA6802F4E0621343CB60BFF33F
:100970004F8F00BFFDE7302BBBD1874EE17E327A2F
:100980009142B6D1607E3146002291F8DC5085421A
:1009900000F0AD800132042A01F58A71F5D1326888
:1009A00040F6B831FA328A4294BF32603160A0E733
:1009B00021462846FFF79EFD9BE721462846FFF784
:1009C000F9FD96E7B2F8EC507B6005F103094FEAB8
:1009D00099094FEA8902D11DC908A8EBC1039D46B8
:1009E000EB460021584600F015FB04F1EE012A46C3
:1009F0003144584600F0FCFA7B6813B9012000F03E
:100A0000ABFA96F8D20000F0B1FA044630B9307271
:100A100000F0CCFA204600F09FFAB0E0D6F8D420DF
:100A20003AB996F8D200B6F82C25824201D8FFF7E1
:100A3000F9FED6F8D4202A44944208D296F8D2007F
:100A4000B6F82C250130824201D8FFF7EBFE706822
:100A50005FFA89F2594600F0E5FA08B9C54679E02F
:100A6000726896F8D2002A447260D6F8D42005EB5A
:100A70000209C6F8D49000F079FA814509D396F8B6
:100A8000D220D6F8D4000132001B86F8D220C6F856
:100A9000D400FF2D0FD80024347200F087FA2046CE
:100AA00000F05AFA00F034FD3C4B188108B9FFF70A
:100AB000A1FCC5461DE7BB6896F8D9000AFB036296
:100AC000FB68D2F8E41082F8E83001F58061C2F8E2
:100AD000E030C2F8E410FFF7CBFDFFF719FE96F8FF
:100AE000D920013202F0030286F8D920B6E74FF48C
:100AF0008A7A0AFB02F505F1EA013144204600F04A
:100B0000ABFCF86000287FF4F4AE3544012285F890
:100B1000E82001F047FCD5F8E020D6ED007ADFEDC3
:100B2000206A801A192838BF192040F6B83290423E
:100B300028BF1046B8EE677A07EE900AF8EEE77A1B
:100B400067EEA67ADFED176AE7EE267AFCEEE77A23
:100B5000C6ED007A96F8D9307168BB600AFB03F4E1
:100B6000321992F8E8505DB1D2F8E4308B42E84691
:100B70003FF428AF002182F8E810C2F8E010C54623
:100B80007368064A9B0A01331381B2E69D21002057
:100B900000ED00E00400FA05D42100208C110020B3
:100BA000CDCCCC3D6666663FA0210020014B18707D
:100BB000704700BF9811002038B54FF00054144B17
:100BC00022689A4221D1607DF0B1124B124918700F
:100BD0001248237D03724FF48073C0F8F8314FF44C
:100BE0000073C0F80C3300254FF44073C0F8203474
:100BF000C0F8E450C922093000F0FAF9E022294691
:100C0000204600F007FA012038BD0020FCE700BFB5
:100C10009AAD44C59811002016000020D421002070
:100C200037B500F075FC194D1949288102230122BE
:100C300018486B7101F050FA00230193164B1749C5
:100C400000931748174B4FF4805201F0EDFE164BFE
:100C5000197811B1124801F00FFF01F0A3FB04460F
:100C6000FFF720FC4FF4C873B0FBF3F202FB130351
:100C700004F5167010FA83F00C4B186003F096F828
:100C800008B10F232B8103B030BD00BF8C110020B1
:100C900040420F00102700209D0700089C110020F3
:100CA000A4210020A108000898110020A021002004
:100CB0002DE9F04F2DED028B0FF23829D9E900898B
:100CC000834C93B00BAE9FED7E8BFFF721FD814FE0
:100CD000DFF828A200230A93ADF834300B93736039
:100CE0004FF0000B5B468DED008B01250DF11D02D1
:100CF00007A938468DF81C508DF81DB001F09AF9FF
:100D00009DF81C30002B40F0A580204601F0BCFE71
:100D10000646002845D1704F01F044FB3B689842DD
:100D20003FD301F03FFB8246FFF7BCFB4FF4C87393
:100D3000B0FBF3F202FB13030AF5167010FA83F00E
:100D40003860664F97F800B0CBF1100ABBF1000F86
:100D500014BF33462B465FFA8AFA0EA88DF8283066
:100D6000FFF7B8FBBAF1060F28BF4FF0060A0EAB2B
:100D700003EB0B0152460DF1290000F039F90AABE3
:100D80000393182302930AF10102554BD2B2CDE925
:100D90000053049220464CA3D3E9002301F0BAFE8D
:100DA0003E7001F0FFFA4F4A4F4D1368C31AB3F576
:100DB0007A7F2ED3106001F0F7FA02460B462046E8
:100DC00001F040FF204601F05FFE10B32B7A474E42
:100DD000002B14BF03230223737101F0E3FA0EAF5B
:100DE0004FF47A730122B0FBF3F03946306030469D
:100DF00000F00EFA182302933D4B019380B240F2AB
:100E00005513CDE90370009342464B46204601F04E
:100E100081FE2B7A93B101F0C5FA002607464FF404
:100E20008A7A95F8D900304400F003000AFB005399
:100E300093F8E82092B30136042EF2D1C82002F0D4
:100E40006DFC2B7A002B7FF43DAF13B0BDEC028B11
:100E5000BDE8F08FDAF8143083F00803CAF81430D4
:100E6000594610220EA800F0D5F80DF11E0308AA6D
:100E70000AA9384600F03AFE96E803000FAB83E873
:100E800003009DF834308DF844300A9B0E930EA970
:100E9000DDE90823204602F0A9F821E7D3F8E02095
:100EA00042B12B68FA2B38BFFA23BA1A0533B2EBDA
:100EB000430FC0D3FFF7DCFB0028BCD1BEE700BF67
:100EC0000000000000000000401DA12026812A0B28
:100ED000A421002010270020A02100209D21002017
:100EE0009C21002004270020D42100208C11002008
:100EF00008270020F1C6A7C1D068080F00040048E9
:100F000008B5054800F090FEBDE80840034A0449D2
:100F1000002003F04DBA00BF102700203038002019
:100F20006908000870B502F095FD094E094D308042
:100F3000002428683388834208D902F087FD2B6893
:100F400004440133B4F5204F2B60F2D370BD00BFD1
:100F500024380020F837002002F02EBE00F1006097
:100F6000920000F5204002F0B1BD0000054B1A6868
:100F7000054B1B889B1A834202D9104402F066BDC0
:100F800000207047F837002024380020024B1B68EF
:100F9000184402F061BD00BFF8370020024B1B6807
:100FA000184402F06BBD00BFF8370020064991F8E5
:100FB000243033B10023086A81F824300822FFF777
:100FC000CDBF0120704700BFFC370020022802BFC0
:100FD000024B4FF400229A61704700BF00040048A2
:100FE000022802BF014B08229A61704700040048A2
:100FF00010B50023934203D0CC5CC4540133F9E70D
:1010000010BD000003460246D01A12F9011B002948
:10101000FAD1704702440346934202D003F8011B01
:10102000FAE770472DE9F8431F4D144695F8242040
:101030000746884652BBDFF870909CB395F8243081
:101040002BB92022FF2148462F62FFF7E3FF95F8D6
:101050002400C0F10802A24228BF2246D6B241466F
:10106000920005EB8000FFF7C3FF95F82430A41B26
:101070001E44F6B2082E17449044E4B285F824606A
:10108000DBD1FFF793FF0028D7D108E02B6A03EBF1
:1010900082038342CFD0FFF789FF0028CBD1002005
:1010A000BDE8F8830120FBE7FC3700202DE9F3477A
:1010B0000D46044600219046284640F27912FFF77B
:1010C000A9FF234620220021284601F031FF231DDD
:1010D00002222021284601F02BFF631D032222213A
:1010E000284601F025FFA31D03222521284601F0F3
:1010F0001FFF04F1080310222821284601F018FFE1
:1011000004F1100308223821284601F011FF04F1F0
:10111000110308224021284601F00AFF04F11203BE
:1011200008224821284601F003FF04F1140320227D
:101130005021284601F0FCFE04F1180340227021E2
:10114000284601F0F5FE04F120030822B0212846CC
:1011500001F0EEFE04F121030822B821284601F037
:10116000E7FE04F12207C0263B4631460822284606
:10117000083601F0DDFEB6F5A07F07F10107F3D1D7
:1011800094F832308DF8073031460DF1070308220C
:10119000284601F0CDFE002604F1330A9DF8073001
:1011A0004FEAC6099E4209F5A47720D394F832315C
:1011B000502B28BF50238DF80730B8F1000F08D10D
:1011C00039460DF107030722284601F0B1FE09F266
:1011D0004F17002604F233149DF807309E4207EBA8
:1011E000C6010DD30731C80802B0BDE8F0870AEB8D
:1011F000060308223946284601F09AFE0136CDE75B
:10120000A3190822284601F093FE0136E4E7000006
:1012100013B504460846002101602346C0F80310B8
:101220002022019001F084FE0198231D022220213A
:1012300001F07EFE0198631D0322222101F078FE59
:101240000198A31D0322252101F072FE019804F1EB
:1012500008031022282101F06BFE072002B010BD08
:10126000F7B5047F05460E462CB1838A122B02D9AE
:10127000012003B0F0BD002319460722009628463E
:1012800001F01AFD731C0093012200230721284658
:1012900001F012FDD4B9B31C0093052223460821A6
:1012A000284601F009FD0D24B378102BE0D837460D
:1012B000B278BB1B934210D32B7FA88A0734E40873
:1012C000B3B9844294BF00200120D2E7AB8ADB008F
:1012D000083BDB08B3700824E6E7FB1C00932146BB
:1012E00000230822284601F0E7FC08340137DFE735
:1012F000201A18BF0120BCE7F7B5047F05460E464B
:101300002CB1838ACA2B02D9012003B0F0BD00237F
:10131000194600960822284601F0CEFC731CD4B969
:101320000822009311462346284601F0C5FC1024EC
:101330007378C82BE8D8012372785F1C013B934275
:1013400010D32B7FA88A0734E408B3B9844294BF32
:1013500000200120D9E7AB8ADB00083BDB08737073
:101360000824E5E7F31900932146002308222846C4
:1013700001F0A2FC08343B46DEE7201A18BF01202A
:10138000C3E70000F7B50D4604460021164628467F
:101390008122FFF73FFE234608220021284601F064
:1013A000C7FD94F901206378002AB8BF7F238DF828
:1013B00007309EB90DF1070307220821284601F0E6
:1013C000B7FD0F27002602349DF807309E4207EB39
:1013D000C60105D30731C80803B0F0BD0827F1E7FF
:1013E000A3190822284601F0A3FD0136ECE700000E
:1013F000F7B50E460546002114463046CE22FFF7CB
:1014000009FE2B4628220021304601F091FD2B7A5F
:10141000C82B28BFC8238DF807308CB90DF10703FE
:1014200008222821304601F083FD30242F469DF804
:1014300007207B1B934205D3E01DC00803B0F0BD1D
:101440002824F3E707F1090321460822304601F07A
:101450006FFD08340137EAE7F7B5047F05460E460D
:1014600034B1838AB3F5827F02D9012003B0F0BD85
:101470000096012310220021284601F01DFCDCB952
:10148000B31C0093092223461021284601F014FCC6
:1014900019247388B3F5807FE7D837467288BB1B61
:1014A000934210D32B7FA88A0734E408B3B984424F
:1014B00094BF00200120D9E7AB8ADB00103BDB089A
:1014C00073801024E5E73B1D00932146002308228A
:1014D000284601F0F1FB08340137DFE7201A18BF76
:1014E0000120C3E730B5094D0A4491420DD011F8EF
:1014F000013B5840082340F30004013B2C4013F00B
:10150000FF0384EA5000F6D1EFE730BD2083B8ED49
:10151000F7B5384A106851686B4603C36A463649C6
:101520003648082302F078FF0446002833D10A2504
:10153000334A106851686B4603C36A4631492F48E5
:10154000082302F069FF0446002849D00369B3F577
:10155000583F45D8B0F8661040F2264291423FD13C
:10156000294A024402F15C018B4239D35C3B234996
:1015700000209E1AFFF7B6FF3246074604F16401C9
:101580000020FFF7AFFFA3689F4229D1E36898428C
:1015900008BF002524E00369B3F5583F27D8418BE5
:1015A00040F22642914220D1174A024402F1100132
:1015B0008B4218D3103B114900209D1AFFF792FF70
:1015C0002A46064604F118010020FFF78BFFA368A6
:1015D0009E4202D1E368984201D00D25A8E700257C
:1015E000284603B0F0BD1025A2E70C25A0E70B2587
:1015F0009EE700BF8C440008DC5F030000A00008E9
:1016000095440008905F03000860FFF710B5037C65
:10161000044613B9006802F0E7FE204610BD000042
:101620000023BFF35B8FC360BFF35B8FBFF35B8FA0
:101630008360BFF35B8F7047BFF35B8F0068BFF3BE
:101640005B8F704770B505460C30FFF7F5FF05F16D
:10165000080604463046FFF7EFFFA04206D93046A1
:101660006D68FFF7E9FF2544281A70BD3046FFF783
:10167000E3FF201AF9E7000070B50546406898B10D
:1016800005F10800FFF7D8FF05F10C0604463046C7
:10169000FFF7D2FF8442304694BF6D680025FFF704
:1016A000CBFF013C2C44201A70BD000038B50C461D
:1016B0000546FFF7C7FFA04210D305F10800FFF76A
:1016C000BBFF04446868B4FBF0F100FB1144BFF3B6
:1016D0005B8F0120AC60BFF35B8F38BD0020FCE75F
:1016E0002DE9F041144607460D46FFF7C5FF844239
:1016F00028BF0446D4B1B84658F80C6B4046FFF7F3
:101700009BFF3044286040467E68FFF795FF331A00
:101710009C4203D86C600120BDE8F0816B60A41B83
:101720003B68AB602044E8600220F5E72046F3E721
:1017300038B50C460546FFF79FFFA04210D305F1D0
:101740000C00FFF779FF04446868B4FBF0F100FB7C
:101750001144BFF35B8F0120EC60BFF35B8F38BD9A
:101760000020FCE72DE9FF41884669460746FFF760
:10177000B7FF6C4606B204EBC6060025B44209D09A
:101780006268206808EB0501FFF732FC63680834E3
:101790001D44F3E729463846FFF7CAFF284604B040
:1017A000BDE8F081F8B505460C300F46FFF744FF61
:1017B00005F1080604463046FFF73EFFA0423046DA
:1017C00088BF6C68FFF738FF201A386020B13046B8
:1017D0002C68FFF731FF2044F8BD000073B51446B4
:1017E00006460D46FFF72EFF844228BF04460190AF
:1017F000DCB101A93046FFF7D5FF019B33B9326850
:10180000C5E90233C5E9002401200CE09C4238BF41
:1018100001942860019868608442F5D93368AB6010
:10182000241AEC60022002B070BD2046FBE70000E5
:101830002DE9FF410F466946FFF7D0FF6C4600B225
:1018400004EBC0050026AC4209D0D4F8048054F85B
:10185000081BB8194246FFF7CBFB4644F3E7304676
:1018600004B0BDE8F081000038B50546FFF7E0FFA1
:10187000044601462846FFF719FF204638BD000000
:101880000121884238BF084602F098BD08B102F035
:10189000ABBD704710B4026854681A4623465DF821
:1018A000044B184700207047002070477047000025
:1018B000002070470E20704700F5805090F8D80047
:1018C000C0F340007047000000F5805090F9E00040
:1018D0007047000000F58050C0F8DC100120704710
:1018E000F7B50C68BDF8207014F0005473D10D7B6F
:1018F000082D70D8302585F31188456AAE687601C9
:101900000CD4AC68240108D4AC6814F0805460D1C5
:1019100084F31188204603B0F0BD01240E6804F161
:10192000180C002EB8BFF6004FEA0C1CB4BF46F0EE
:101930000406760545F80C600E680FFA84FC16F074
:10194000804F18BF05EB0C1E05EB0C1C1EBFDEF80C
:10195000806146F00206CEF880610E7BCCF884618F
:1019600005EB04158E68C5F88C614E68C5F8886172
:10197000DCF8805145F00105CCF8805141F2780542
:1019800000EB441C660105EB4414AC440444CCE970
:1019900000230D46083401F10C0C55F804EB44F813
:1019A00004EB6545F9D12D882580841904F5805410
:1019B00007F0030594F8946026F00B06354384F88D
:1019C0009450002484F31188009700F035FD012025
:1019D000A1E70224A2E74FF0FF309CE713B500F522
:1019E00080540191E06EFFF747FE1F280AD9019944
:1019F000E06E2022FFF7B6FEA0F1200358425841C6
:101A000002B010BD0020FBE708B5302383F3118836
:101A100000F58050C06EFFF703FE002383F31188AA
:101A200008BD00000022026082814260826070472F
:101A300010B500220023C0E90023002304460381DF
:101A40000C30FFF7EFFF204610BD0000F0B5054653
:101A500000F580500C4690F8D83013F0040FC3F313
:101A6000800108BF114661F3820380F8D83005EB8E
:101A7000441303F58453103389B01B79D8074FEA18
:101A800044162FD582B319072ED46846FFF7D0FF2E
:101A900005EB441303F5845303AA03F10807186800
:101AA0005968144603C40833BB422246F7D118686C
:101AB00020609B88A380DDE90E23CDE9002301236C
:101AC000ADF808302B6869461B6C284698473544AA
:101AD00005F5845510352B791A075CBF43F00803D0
:101AE0002B7101E0002AF2D109B0F0BD2DE9F047D9
:101AF0009A4688B0074688469146302383F311887A
:101B000007F580546846FFF793FFE06EFFF79AFDF4
:101B10001F282AD9E06E20226946FFF7A5FE20285B
:101B200023D103AD444605AB2E4603CE9E42206032
:101B30006160354604F10804F6D130682060B3884E
:101B4000A380DDE90023C9E90023BDF80830AAF825
:101B50000030002383F3118853464A4641463846F5
:101B600008B0BDE8F04700F02BBC002080F31188DE
:101B700008B0BDE8F08700002DE9F84F18220446B0
:101B80000F4604300021FFF745FA2046234B40F86A
:101B9000283BFFF747FF04F13800FFF749FF04F146
:101BA000580804F582554646183530462036FFF76A
:101BB0003FFFAE42F9D104F580554FF480534FF00A
:101BC0000009C5E91739C5F858800123EE6604F508
:101BD000875804F58456C5F8649085F8683085F810
:101BE0007030183608F118084FF0000A4FF0000B5B
:101BF00046E908ABA6F11800FFF714FF203646F8B7
:101C0000289C4645F4D185F8E07017B1044800F0EF
:101C1000C3FB044B63622046BDE8F88FC84400084C
:101C2000A04400080064004010B5044B1978044635
:101C30004A1C1A70FFF7A0FF204610BD2C38002068
:101C40002DE9F047002950D0294B2A4FB7FBF1F579
:101C500099428CBF0A231123581EB5FBF3FC03FBEA
:101C60001C53C4B22BB102280346F5D80020BDE8AE
:101C7000F0870CF1FF36B6F5806FF7D2C4EBC40ED7
:101C80000EF103034FEAE309C3F3C703A4EB030810
:101C900009F1010A4FF47A755FFA88F009FB0555DE
:101CA0005AFA88F8B5FBF8F5B5F5617FC1BF0EF1BA
:101CB000FF33C3F3C703E01AC0B25C1C50FA84F4CC
:101CC0000CFB04F4B7FBF4F4A142CFD1013BDBB22F
:101CD0000F2BCBD80138C0B20728C7D8002110710C
:101CE00016809170D3700120C1E70846BFE700BF9E
:101CF0003F420F0000B4C40470B505460E464FF4D1
:101D00007A746B6A5B6803F00103B34207D04FF447
:101D10007A7001F003FD013CF3D1204670BD012033
:101D2000FCE7000070B5426A936913F0700F17D09A
:101D300000230C4D936141F2900400EB43122244C6
:101D400011794E0709D5890707D5416A55F82360EF
:101D50008E60117941F0040111710133032BECD134
:101D600070BD00BFB444000873B51D46436A1646F3
:101D70009A68D207044609D59A6801219960C2F38E
:101D80004002CDE900650021FFF760FE636A9A68B2
:101D9000D1050BD59A684FF480719960C2F3402247
:101DA000CDE9006501212046FFF750FE636A9A687D
:101DB000D2030BD59A684FF480319960C2F3404248
:101DC000CDE9006502212046FFF740FE04F580536F
:101DD000D3F8DC0010B103681B699847204602B0B5
:101DE000BDE87040FFF79EBFF8B50446466A00297B
:101DF00077D106F10C073868800775D006EB01151E
:101E00003868D5F8B00110F0040FD5F8B0011ABF4A
:101E1000C00840F00040400DA062D5F8B0C11CF0F1
:101E2000020F1CBF40F08040A062D5F8B40106EB61
:101E3000011100F00F0084F83400D1F8B80184F8E3
:101E40002C00D1F8B801000A84F82D00D1F8B801AF
:101E5000000C84F82E00D1F8B801000E84F82F0091
:101E6000D1F8BC0184F83000D1F8BC01000A84F834
:101E70003100D1F8BC01000C84F83200D1F8BC115B
:101E8000090E84F833103821396004F1440004F15C
:101E9000280104F1340551F8046B40F8046BA942A1
:101EA000F9D109880180C4E90E2321460023A4F852
:101EB000403051F8383B20461B6C984704F580535E
:101EC00093F8D820D3F8DC0042F0040283F8D8203D
:101ED00010B103681B6998472046BDE8F840FFF73A
:101EE00021BF06F1100786E7F8BD000010B50446D3
:101EF00000F05AFA02460B4652EA030102D0013AB8
:101F000063F100030449086820B12146BDE8104090
:101F1000FFF76ABF10BD00BF28380020F0B53021A0
:101F200081F31188DFF848E000F58351183100246F
:101F300041F2900C00EB441565442E7977070ED4DE
:101F4000F6060CD5D1E9007697429E4107D2466A43
:101F50005EF82470B7602E7946F004062E710134C5
:101F6000032C01F12001E5D1002383F31188F0BD9A
:101F7000B444000808B5302383F31188FFF7D2FE7C
:101F8000002383F3118808BD2DE9F041436A04461C
:101F9000986800F0E050B0F1E05F0E4622D0F8B152
:101FA000302383F31188002504F5845741F290080B
:101FB00004EB451343441B791A0706D50135032D5D
:101FC00007F12007F4D1012007E05B07F6D439467A
:101FD000304600F083FA0028F0D1002383F3118803
:101FE000BDE8F0810120FBE708B5302383F31188B9
:101FF00000F58050C06EFFF725FB002383F31188A6
:1020000043090CBF0120002008BD0000F8B51D46A3
:10201000002313700F4606461446FFF7E5FF80F0D5
:102020000100387025B129463046FFF7ADFF20701A
:10203000F8BD00002DE9B8410C4615461F46804604
:1020400000F0B2F90B462178024609B9287850B160
:102050004046FFF763FFFFF78DFF3B462A462146C8
:10206000FFF7D4FF0120BDE8B881000070B530262D
:1020700086F31188174B9A6D42F000729A659A6B3D
:1020800042F000729A639A6B22F000729A63002306
:1020900083F3118800F5805494F8D83013F00105CB
:1020A00016D1A9B186F311880321132001F032FA69
:1020B0000321142001F02EFA0321152001F02AFA41
:1020C00094F8D83043F0010384F8D83085F31188B0
:1020D00070BD00BF001002402DE9F04700F58055AB
:1020E00088B095F8E030012B04468846164600F289
:1020F0008280824F57F823200AB947F82300D7F887
:1021000000A0C4F81C8084F82060BAF1000F64D0ED
:1021100095F8E030012B70D001212046FFF7A6FF93
:10212000302383F31188626A136823F0020313607B
:10213000626A136843F001031360636A00275F61FA
:1021400087F3118801212046FFF7D6FD002800F013
:102150009580E86EFFF764FA04F58359BA4609F1F1
:102160001809202200216846FEF754FF02A8FFF755
:1021700059FCCDF818A06A4609EB07030DF1180EBB
:102180009446BCE80300F44518605960624603F1C8
:102190000803F5D1DCF80000186020379CF8042013
:1021A0001A71602FDDD195F8D8306FF382030027C4
:1021B00085F8D8306A4641462046ADF80070ADF843
:1021C00002708DF80470FFF73BFD636A48BB4FF463
:1021D00000421A6008B0BDE8F08741F2E800FFF75E
:1021E0004FFB814610B15146FFF7C6FCC7F800907F
:1021F000B9F1000F8CD10020ECE7386803681B6B45
:1022000098470146002887D13868FFF72FFF3868C4
:10221000036832465B684146984700287FF47CAFEC
:10222000E9E761221A609DF802309DF803201B0641
:10223000120402F4702203F040731343BDF800202F
:10224000C2F3090213439DF804201205022E02F482
:10225000E0020CBF4FF0004100211343626A0B43C0
:10226000D361636A13225A61626A136823F001031F
:10227000136039462046FFF73FFD08B9636AA6E7B9
:1022800095F8E03093BB616AD1F8002242F0010278
:10229000C1F80022616AD1F8002222F47C5222F0B7
:1022A0000E02C1F80022616AD1F8002242F4606295
:1022B000C1F80022626AC2F81432626AC2F80432BB
:1022C000626A41F6FF71C2F80C12626AC2F84032CB
:1022D000626AC2F84432636A0122C3F81C22626A4D
:1022E000D2F8003223F00103C2F8003295F8D8305A
:1022F00043F0020385F8D8306CE700BF283800208F
:1023000008B500F051F850EA0103024602D0421E1F
:1023100061F10001044B186810B10B46FFF724FD72
:10232000BDE8084001F0B8B82838002008B5002002
:10233000FFF7DCFDBDE8084001F0AEB808B50120AC
:10234000FFF7D4FDBDE8084001F0A6B800B59BB08A
:10235000EFF3098168226846FEF74AFEEFF3058332
:10236000014B9B6BFEE700BF00ED00E008B5FFF7F7
:10237000EDFF000000B59BB0EFF3098168226846CD
:10238000FEF736FEEFF30583014B5B6BFEE700BF04
:1023900000ED00E0FEE700000FB408B5029801F080
:1023A0006DF9FEE701F048BC01F02ABC0139C9B261
:1023B00002299EBF00EBC1000023C0E90133704732
:1023C000F8B51B885B0705460E4615D4044600F198
:1023D0001807BC4210D0636853B12B682846DB6BEA
:1023E0009847A368C1B23246606898470834F0E75E
:1023F000A368002BF1D1F9E70120F8BD73B56C4655
:1024000084E80600014600224E68D5B26EB98E6897
:102410005EB900EBC200021D94E80300013582E8BA
:1024200003001D70012002B070BD0132032A01F1CA
:102430000801E9D10020F6E72DE9F04F89B0044604
:10244000BDF848700E46054600F118084FF0000927
:1024500007F004074FF0000A4FF0000BA84538D0F2
:102460006B680BB9AB684BB157B923682046DB6B7F
:102470009847AB68C1B23246686898470835EDE7BF
:10248000B9F1000FFAD1CDE900ABADF808903346B1
:1024900003AA06F1080E186859689446ACE80300D0
:1024A000083373456246F6D11868CCF800009B8863
:1024B000ACF80430FFF778FF0423ADF80830236848
:1024C000CDE900011B6C6946204698474FF0010991
:1024D000D4E7012009B0BDE8F08F000030B50368F3
:1024E0000968DD0FB5EBD17F23F0604421F0604235
:1024F0004FEAD1700BD0002BB8BFA40C0029B8BF95
:10250000920C944202D034BF0120002030BD94428E
:1025100005D1C1F38070C3F380738342F6D1944236
:102520002CBF00200120F1E72DE9F041456A15B9E3
:102530004162BDE8F0814B6823F06047C3F38A46EF
:102540004FEAD37EC3F3807816EA230638BF3E46AF
:10255000AC462B465A68BEEBD27F22F060440AD0CC
:10256000002A18DAA40CB44217D19D420FD10D6095
:10257000DEE71346EEE7A74207D102F08044C2F33C
:10258000807242450BD054B1EFE708D2EDE7CCF8AA
:1025900000100B60CDE7B44201D0B442E5D81A6810
:1025A0009C46002AE5D11960C3E700002DE9F047F9
:1025B000089D01F007044FEAD508224405F00705FD
:1025C00000EBD1004FF47F49944201D1BDE8F08780
:1025D00004F0070705F0070A57453E4638BF564640
:1025E000C6F10806111B8E4228BF0E46E10808EB13
:1025F000D50E415C13F80EC0B94029FA06F721FA4E
:102600000AF1FFB28CEA010147FA0AF739408CEA75
:10261000010C03F80EC034443544D5E780EA0120AC
:10262000082341F2210201B24000002980B203F1E7
:10263000FF33B8BF504013F0FF03F4D170470000E0
:1026400038B50C468D18A54200D138BD14F8011BD1
:10265000FFF7E4FFF7E7000042684AB11368436000
:102660004389818901339BB29942438138BF838179
:102670001046704770B588B0202204460D46684663
:102680000021FEF7C7FC20460495FFF7E5FF024650
:1026900058B16B46054608AE1C4603CCB4422860D0
:1026A0006960234605F10805F6D1104608B070BDF3
:1026B000082817D909280CD00A280CD00B280CD0D0
:1026C0000C280CD00D280CD00E2814BF4020302030
:1026D00070470C2070471020704714207047182056
:1026E0007047202070470000082817D90C280CD903
:1026F00010280CD914280CD918280CD920280CD94A
:1027000030288CBF0F200E207047092070470A2008
:1027100070470B2070470C2070470D207047000059
:102720002DE9F843078C072F04461ED9D0E90298FB
:1027300000254FF6FF73C5F12006A5F1200029FA08
:1027400005F108FA06F628FA00F031430143C9B250
:102750001846FFF763FF0835402D0346EBD1E169CA
:102760003A46BDE8F843FFF76BBF4FF6FF70BDE890
:10277000F883000010B54B6823B9CA8A63F30902D5
:10278000CA8210BD04691A681C600361C38A013BD8
:10279000C3824A60EFE700002DE9F84F1D46CB8A5F
:1027A0000F46C3F309010529814692460B4630D0F6
:1027B0000020AAB207F11A049EB2042E1FFA80F874
:1027C0000FD8904503F1010306D3FB8A0A4462F354
:1027D0000903FB8201201AE01AF80060E654013078
:1027E000EAE79045F1D2A1F1050B1C237C68BBFB05
:1027F000F3F203FB12BB1FFA8BF6002C45D14846BF
:10280000FFF72AFF044638B978606FF00200BDE890
:10281000F88F4FF00008E6E7002606607860ADB25A
:102820004FF0000B454510D90AEB0803221D13F8A1
:10283000011B9155B1B208F101081B291FFA88F854
:102840002BD0454506F10106F1D8FB8AC3F30902F6
:10285000154465F30903BCE7013292B21C462368B4
:10286000002BF9D16B1F0B441C21B3FBF1F3013397
:102870009BB29A42D3D2BBF1000FD0D14846FFF7AA
:10288000EBFE20B9C4F800B0BFE70122E7E7C0F8CB
:1028900000B05E4620600446C1E74545D5D94846AC
:1028A000FFF7DAFE08B92060AFE7C0F800B00026F5
:1028B00020600446B6E700002DE9F04F2DED028BB5
:1028C0001C4683B05B69019207468846002B00F0E6
:1028D000A780238C2BB1E269002A00F0A180072B8E
:1028E00035D807F10C00FFF7B7FE054638B96FF091
:1028F0000205284603B0BDEC028BBDE8F08F142220
:102900000021FEF787FB228CE16905F10800FEF744
:102910006FFB208C013080B2FFF7E6FEFFF7C8FEA8
:10292000013880B22084013028746369228C1B78BE
:102930002A4403F01F0363F03F0348F00041137281
:10294000384669602946FFF7EFFD0125D1E70233DC
:102950009BB20722C18A0633B3FBF2F3828A521A72
:102960009BB292B29342C2D800F10C034FF000091F
:1029700008EE103A4FF0800A4E464D4618EE100A07
:10298000FFF76AFE83460028B1D014220021FEF72B
:1029900041FB002E3AD1019BABF8083002220BF12B
:1029A000080E1FFA82FC0CF10100BCF1060F218C0D
:1029B00080B201D88E422BD3FFF796FEFFF778FE48
:1029C00062691278013802F01F028E4208BF4FF090
:1029D000400A42EA49121BFA80F14AEA020A01302F
:1029E00048F0004281F808A08BF81000CBF80420D2
:1029F00059463846FFF798FD238C0135B3422DB276
:102A000089F001094FF0000AB8D172E70022C6E749
:102A1000E169895D0EF802100136B6B20132C0E7F5
:102A20006FF0010565E70000F8B515460E46302247
:102A3000002104461F46FEF7EDFA069B6360B5F5DC
:102A4000001F079BA76034BF6A094FF6FF72A3629D
:102A500097B2E66104F1100000239A4206D80023E1
:102A60000360A782E3822383E360F8BD066001333D
:102A700030462036F1E7000003781BB94BB2002B3B
:102A8000C8BF01707047000000787047F8B50C4669
:102A9000C969074611B9238C002B37D1257E1F2D1C
:102AA00034D8387828BB228C072A2CD8268A36F0CE
:102AB00003032BD14FF6FF70FFF7C2FD20F001009A
:102AC0003102400441EA0561400C41EA40254FF6DD
:102AD000FF72234629463846FFF7EEFE002807DD41
:102AE000626913780133DBB21F2B88BF0023137098
:102AF000F8BD218A2D0645EA012505432046FFF74A
:102B00000FFE0246E5E76FF00300F1E76FF001000A
:102B1000EEE7000070B58AB0044616460021282270
:102B200068461D46FEF776FABDF83830ADF810302D
:102B30000F9B05939DF840308DF81830119B07933B
:102B40006946BDF84830ADF820302046CDE9026531
:102B5000FFF79CFF0AB070BD2DE9F041D36905462F
:102B60000C4616460BB9138C5BBB377E1F2F28D83B
:102B700095F80080B8F1000F26D03046FFF7D0FD61
:102B80003378210241EAC33141EA0801338A41EA3C
:102B9000076141EA03410246334641F0800128467D
:102BA000FFF78AFE00280ADD3378012B07D172690E
:102BB00013780133DBB21F2B88BF00231370BDE8ED
:102BC000F0816FF00100FAE76FF00300F7E7000013
:102BD000F0B58BB004460D46174600212822684602
:102BE0001E46FEF717FA9DF84C305A1E53425341C9
:102BF0008DF800309DF84030ADF81030119B0593F2
:102C00009DF848308DF81830149B07936A46BDF83C
:102C10005430ADF8203029462046CDE90276FFF742
:102C20009BFF0BB0F0BD0000406A00B1043070475C
:102C3000436A1A68426202691A600361C38A013BEF
:102C4000C38270472DE9F041D0F82080194E144618
:102C50001D464146002709B9BDE8F081D1E90223AC
:102C6000A21A65EB0303964277EB03031ED2036AB5
:102C70008B420DD1FFF77EFD036A1B680362036977
:102C80000B60C38A0161016A013BC3828846E2E7A7
:102C9000FFF770FD0B68C8F8003003690B60C38A4A
:102CA0000161013BC382D8F80010D4E78846096867
:102CB000D1E700BF80841E002DE9F04F8BB00D4698
:102CC000DDF8509014469B468046002800F019819C
:102CD000B9F1000F00F01581531E3F2B00F2118156
:102CE000012A03D1BBF1000F40F00B810023CDE995
:102CF0000833B8F81430B5EBC30F4FEAC30703D35A
:102D000000200BB0BDE8F08F2B199F42D8F80C3093
:102D10003ABF7F1BFFB227461BB9D8F81030002BF3
:102D20007AD0272D4ED8C5F12806B7424FF00003C0
:102D30002CBFF6B23E4600932946D8F8080008ABEF
:102D40003246FFF733FCA7EB060A35445FFA8AFAEE
:102D5000B8F8143003F10053053BDB000493D8F8B6
:102D60000C3003932821039B13B1BAF1000F2CD12F
:102D7000D8F8100040B1BAF1000F05D0009608ABAA
:102D80005246691AFFF712FC38B2002FB8D0660716
:102D90000AD00AAB03EBD401624211F8083C02F0FE
:102DA0000702134101F8083C082C3CD9102C40F2D2
:102DB000B580202C40F2B780BBF1000F00F09C8062
:102DC000082334E0BA460026C2E7049BE02B28BF64
:102DD000E02306930B44AB42059314D95A1B039886
:102DE0000096924534BF5246D2B2691A08AB0430FD
:102DF0000792FFF7DBFB079A1644AAEB020A154479
:102E0000F6B25FFA8AFA049B069A05999B1A049314
:102E1000039B1B680393A6E70093D8F8080008AB50
:102E20003A462946AEE7BBF1000F13D00123B4EBBD
:102E3000C30F6CD0082C12D89DF82030621E23FAE4
:102E400002F2D50706D54FF0FF3202FA04F423430D
:102E50008DF820309DF8203089F8003051E7102C93
:102E600012D8BDF82030621E23FA02F2D10706D52F
:102E70004FF0FF3202FA04F42343ADF82030BDF8DE
:102E80002030A9F800303CE7202C0FD80899631EA9
:102E900021FA03F3DA0705D54FF0FF3202FA04F402
:102EA0000C430894089BC9F800302AE7402C2BD02B
:102EB000DDE90865611EC4F12102A4F1210326FAAF
:102EC00001F105FA02F225FA03F311431943CB0786
:102ED00012D50122A4F12003C4F1200102FA03F368
:102EE00022FA01F1A240524243EA010363EB430399
:102EF00032432B43CDE90823DDE90823C9E9002348
:102F0000FFE66FF00100FCE66FF00800F9E6082C20
:102F1000A0D9102CB3D9202CEED8C3E7BBF1000FF9
:102F2000ADD0022383E7BBF1000FBBD004237EE7C3
:102F300030B5012A144638BF0124402C85B028BF83
:102F400040240025012ACDE9025518D81B788DF8B8
:102F5000083063070AD004AB03EBD405624215F8CE
:102F6000083C02F00702934005F8083C0091034634
:102F70002246002102A8FFF719FB05B030BD082A40
:102F8000E4D9102A03D81B88ADF80830E1E7202ADD
:102F90008DBFD3E900231B680293CDE90223D8E754
:102FA00010B5CB681BB98B600B618B8210BD0469B7
:102FB0001A681C600361C38A013BC382CA60F0E7E0
:102FC00003064CBFC0F3C0300220704708B502466C
:102FD000FFF7F6FF022806D15306C2F30F2001D1F6
:102FE00000F0030008BDC2F30740FBE72DE9F04FF6
:102FF00093B0CDE903230A6804461046FFF7E0FFCB
:10300000022814BFC2F306260026002A0D46824677
:1030100080F2F78112F0C04940F0F381097B00296A
:1030200000F0EF81022803D02378B34240F0EC8116
:10303000C2F304630693104602F07F030593FFF783
:10304000C5FF059B29444FEA834848EA0A4848EAF5
:103050004668CE7800230022CDE90823F309834691
:1030600048EA0008029367D0059B00930246676810
:10307000534608A92046B847002800F0C881276AAF
:103080004FB9414604F10C00FFF7F4FA074690B936
:103090006FF0020054E03B6998450DD03F68002F67
:1030A000F9D1414604F10C00FFF7E4FA0746002885
:1030B000EED0236A3B60276297F817C006F01F081E
:1030C000CCF3840CACEB08001FFA80FE0028B8BFDC
:1030D0000EF12000A8EB0C031FFA83FED7E90221B2
:1030E000B8BF00B2002B0793BEBF0EF120031BB286
:1030F000079352EA010338D0039BDFF824E39A1ABE
:10310000049B4FF0000C63EB010196457CEB01033F
:103110002BD36B7B97F81AE0734519D1029B002BD8
:1031200078D0012821DC7868F8B9DFF8F0C294453E
:1031300070EB010316D337E0276A27B96FF00C0054
:1031400013B0BDE8F08F3B699845B5D03F68F4E710
:10315000B24890427CEB010301D30020F0E7029BD0
:10316000002BFAD0079B0F2B17DCFA7DB30002F07F
:10317000030203F07C031343FB7539462046FFF737
:10318000F9FA6B7BBB76029B3BB9FB7DC3F38402F0
:10319000013262F38603FB75D0E76A7BBB7E9A42FD
:1031A000DBD1029B002B35D0B309022B32D0039B1D
:1031B000BB60049BFB60142200210DA8FDF72AFFD1
:1031C000039B0A93049B0B932B1D0C932B7BADF855
:1031D0003EB0013BDBB2ADF83C30069B8DF842308F
:1031E000059B8DF8433094F82C308DF840A083F087
:1031F00001038DF844308DF84180A3680AA9204668
:103200009847FB7DC3F38403013303F01F039B0244
:10321000FB82A2E7FB7DC6F34012B2EBD31F40F066
:10322000F980C3F38403434540F0FC80029A2B7B72
:10323000B609002A52D016F0010661D1032B40F2E4
:10324000F480039BBB60049BFB60FB8A66F309036D
:10325000FB822B7BAE1D033BDBB23246394604F1C9
:103260000C00FFF799FA00280CDA39462046FFF7E0
:1032700081FAFB7DC3F38403013303F01F039B0238
:10328000FB8205E7DDE90884AB883B834FF6FF73DB
:10329000C9F12000A9F1200228FA09F104FA00F08E
:1032A000014324FA02F211431846C9B2FFF7B6F9F6
:1032B00009F10809B9F1400F0346E9D1B8822A7B28
:1032C000033AD2B23146FFF7BBF9FB7DB882DA434D
:1032D000C2F3C01262F3C713FB753EE786B92E1D19
:1032E000013BDBB23246394604F10C00FFF754FAD9
:1032F0000028BADB2A7BB88A013AD2B23146E2E72B
:10330000F98AC1F30901013B0429DAB25BD8281D0F
:10331000002307F11B069A4208D910F801CB06F8E2
:1033200001C0013101330529DBB2F4D103990A91BF
:1033300004990B91934207F11B010C9138BF0433A0
:1033400079680D9134BF55FA83F300230E93FB8AFD
:10335000ADF83EB0C3F309031A44069B8DF8423022
:10336000059B8DF8433094F82C30ADF83C2083F069
:1033700001038DF8443000238DF840A08DF8418082
:103380007B602A7BB88A013A291DFFF759F93B8BEC
:10339000B882834203D1A3680AA9204698472046F1
:1033A0000AA9FFF7FDFDFB7DBA8AC3F3840301334D
:1033B00003F01F039B02FB823B8B9A420CBF002051
:1033C0006FF01000BCE67B68002BAFD0052001E059
:1033D0001C3033461E68002EFAD1091A081D2E1D16
:1033E000184401EB090CBCF11B0F5FFA89F39DD85F
:1033F0009A429BD916F8013B00F8013B09F10109FB
:10340000EFE76FF009009BE66FF00A0098E66FF0B7
:103410000B0095E66FF00D0092E600BF40420F00F2
:1034200080841E006FF00E008AE66FF00F0087E6C2
:10343000EFF3098305494A6B22F001024A636833BE
:1034400083F30988002383F31188704700EF00E0BD
:10345000302080F3118862B60C4B0D4AD96821F4F4
:10346000E0610904090C0A43DA60D3F8FC20094939
:1034700042F08072C3F8FC200A6842F001020A6040
:103480002022DA7783F82200704700BF00ED00E0C9
:103490000003FA05001000E010B5302383F3118813
:1034A0000E4B5B6813F4006314D0F1EE103AEFF3A7
:1034B0000984683C4FF08073E361094BDB6B236642
:1034C00084F3098800F0A4F810B1064BA36110BD85
:1034D000054BFBE783F31188F9E700BF00ED00E03F
:1034E00000EF00E0FF020008020300084FF0E023B5
:1034F000002258684FF0FF31930003F1604303F559
:10350000614301329042C3F88010C3F88011F3D2B6
:103510007047000000F1604303F561430901C9B23F
:1035200083F80013012200F01F039A4043099B0017
:1035300003F1604303F56143C3F880211A607047CB
:1035400000230375826803691B6899689142FBD266
:103550005A6803604260106058607047002303752A
:10356000826803691B6899689142FBD85A680360B6
:10357000426010605860704708B50846302383F3F6
:1035800011880B7D032B05D0042B0DD02BB983F3B1
:10359000118808BD8B6900221A604FF0FF338361E8
:1035A000FFF7CEFF0023F2E7D1E9003213605A6043
:1035B000F3E70000FFF7C4BF054BD968087518682A
:1035C00002681A60536001220275D860FCF782BE5F
:1035D0003838002030B50C4BDD684B1C87B00446F2
:1035E0000FD02B46094A684600F02AF92046FFF71B
:1035F000E3FF009B13B1684600F02CF9A86907B0FF
:1036000030BDFFF7D9FFF9E73838002079350008D9
:10361000044B1A68DB6890689B68984294BF00204E
:103620000120704738380020084B10B51C68D86856
:1036300022681A60536001222275DC60FFF78EFF5A
:1036400001462046BDE81040FCF744BE3838002053
:1036500038B5074C074908480123002523706560E9
:1036600000F0EAFB0223237085F3118838BD00BF08
:10367000603A0020104500083838002008B572B6BE
:10368000044B186500F0ACFA00F058FB024B032223
:103690001A70FEE738380020603A002000F010B9B8
:1036A0008B60022308618B82084670478368A3F110
:1036B000840243F8142C026943F8442C426943F80D
:1036C000402C094A43F8242CC26843F8182C0222E3
:1036D00003F80C2C002203F80B2C044A43F8102C9E
:1036E000A3F12000704700BFED0200083838002029
:1036F00008B5FFF7DBFFBDE80840FFF75BBF000040
:10370000024BDB6898610F20FFF756BF3838002066
:10371000302383F31188FFF7F3BF000008B501469B
:10372000302383F311880820FFF754FF002383F32D
:10373000118808BD10B503689C68A2420CD85C686B
:103740008A600B604C602160596099688A1A9A609F
:103750004FF0FF33836010BD1B68121BECE70000C5
:103760000A2938BF0A2170B504460D460A26601999
:1037700000F05CFB00F048FB041BA54203D8751C5D
:103780002E460446F3E70A2E04D9BDE87040012016
:1037900000F092BB70BD0000F8B5144B0D46D96126
:1037A00003F1100141600A2A1969826038BF0A22B8
:1037B000016048601861A818144600F029FB0A2728
:1037C00000F022FB431BA342064606D37C1C2819AB
:1037D00000F02CFB27463546F2E70A2F04D9BDE856
:1037E000F840012000F068BBF8BD00BF3838002069
:1037F000F8B506460D4600F007FB0F4A134653F88E
:10380000107F9F4206D12A4601463046BDE8F84067
:10381000FFF7C2BFD169BB68441A2C1928BF2C46D8
:10382000A34202D92946FFF79BFF224631460348AF
:10383000BDE8F840FFF77EBF383800204838002048
:1038400010B4C0E9032300235DF8044B4361FFF784
:10385000CFBF000010B5194C236998420DD0D0E9B4
:103860000032816813605A609A680A449A600023A3
:1038700003604FF0FF33A36110BD2346026843F895
:10388000102F53600022026022699A4203D1BDE8E2
:10389000104000F0C5BA936881680B44936000F053
:1038A000B3FA2269E1699268441AA242E4D9114448
:1038B000BDE81040091AFFF753BF00BF3838002099
:1038C0002DE9F047DFF8BC8008F110072C4ED8F83E
:1038D000105000F099FAD8F81C40AA68031B9A42CD
:1038E0003ED81444D5E900324FF00009C8F81C4016
:1038F00013605A60C5F80090D8F81030B34201D177
:1039000000F08EFA89F31188D5E9033128469847EB
:10391000302383F311886B69002BD8D000F074FA40
:103920006A69A0EB04094A4582460DD2022000F0E4
:10393000C3FA0022D8F81030B34208D151462846C5
:10394000BDE8F047FFF728BF121A2244F2E712EB56
:10395000090938BF4A4629463846FFF7EBFEB5E766
:10396000D8F81030B34208D01444211AC8F81C000B
:10397000A960BDE8F047FFF7F3BEBDE8F08700BFE0
:10398000483800203838002038B500F03DFA054AA4
:10399000D2E90845031B181945F10001C2E90801E5
:1039A00038BD00BF3838002000207047FEE7000017
:1039B000704700004FF0FF3070470000BFF34F8F9B
:1039C000024A1369DB03FCD4704700BF00200240A9
:1039D00008B5094B1B7873B9FFF7F0FF074B5A691D
:1039E000002ABFBF064A9A6002F188329A601A68BC
:1039F00022F480621A6008BD783A0020002002405C
:103A00002301674508B50B4B1B7893B9FFF7D6FF29
:103A1000094B5A6942F000425A611A6842F48052D6
:103A20001A601A6822F480521A601A6842F480629E
:103A30001A6008BD783A0020002002407F289ABF13
:103A400000F58030C0020020704700004FF4006095
:103A500070470000802070477F2808B50BD8FFF71B
:103A6000EDFF00F500630268013204D104308342A7
:103A7000F9D1012008BD0020FCE700007F2810B527
:103A800004461FD8FFF79AFFFFF7A2FF0E4BF32261
:103A90001A6102225A615A6942EAC0025A615A699D
:103AA00042F480325A61FFF789FF4FF40061FFF75B
:103AB000C5FF00F03FF9FFF7A5FF2046BDE8104025
:103AC000FFF7CABF002010BD002002402DE9F843D7
:103AD00040EA020313F00703144606D0304B40F2CD
:103AE00082321A600020BDE8F88385182D4A95427D
:103AF0000CD92B4A40F287311160F3E7031D1B6894
:103B00004A68934208D1083C08300831072C14D980
:103B100002680B689A42F1D0FFF75AFFFFF74EFF99
:103B2000214E08314FF001084FF00009012CA1F19E
:103B3000080706D8FFF766FF01E0002CECD1012052
:103B4000D1E7C6F81480054651F8083C45F8043B17
:103B500051F8043C4360FFF731FF336943F0010340
:103B60003361C6F81490026851F8083C9A420CD0B0
:103B70000B4B40F2AF321A600C4B18600C4B1C60C0
:103B80000C4B1F60FFF73EFFACE72D6851F8043C7B
:103B90009D4201F10801EBD1083C0830C6E700BFA7
:103BA000743A00200000040800200240683A002017
:103BB000703A00206C3A0020084908B50B7828B10B
:103BC0001BB9FFF705FF01230B7008BD002BFCD0CC
:103BD000BDE808400870FFF715BF00BF783A002025
:103BE00002484FF47F4100F0A7B800BF0001002059
:103BF0000846114600F0E2BB084600F0F5BB0000A5
:103C000038B5EFF311859DB9EFF30584C4F30804CB
:103C1000302334B183F31188FFF7B6FE85F31188A2
:103C200038BD83F31188FFF7AFFE84F3118838BDE8
:103C3000BDE83840FFF7A8BE38B5FFF7E1FF114CEB
:103C4000114AC00840EA4170A0FB025EC908A0FB0F
:103C5000040C1CEB050CA1FB04404FF000035B417E
:103C6000A1FB02121CEB040C43EB000011EB0E0154
:103C700042F10002411842F10000090941EA0070D6
:103C800038BD00BFCFF753E3A59BC42010B5024455
:103C9000064BD2B2904200D110BD441C00B253F882
:103CA000200041F8040BE0B2F4E700BF50280040C8
:103CB000114B30B5D3F89040240409D4D3F8904088
:103CC000C3F89040D3F8904044F40044C3F89040C7
:103CD0000A4C236843F4807323600244084BD2B239
:103CE000904200D130BD441C00B251F8045B43F84F
:103CF0002050E0B2F4E700BF001002400070004026
:103D00005028004007B5012201A90020FFF7BEFF9F
:103D1000019803B05DF804FB13B50446FFF7F2FF0A
:103D2000A04205D0012201A900200194FFF7C0FFA5
:103D300002B010BD704700007047000070470000DF
:103D4000074B45F255521A6003225A6040F2FF7247
:103D50009A604CF6CC421A60024B01221A707047EE
:103D600000300040803A0020034B1B781BB1034B0E
:103D70004AF6AA221A607047803A002000300040BC
:103D8000054B1A6832B902F1804202F50432D2F8CA
:103D900094201A60704700BF7C3A0020024B4FF419
:103DA0000002C3F8942070470010024008B5FFF7E6
:103DB000E7FF024B1868C0F3407008BD7C3A002052
:103DC00070470000FEE700000A4B0B480B4A904288
:103DD0000BD30B4BDA1C121AC11E22F003028B42CA
:103DE00038BF00220021FDF715B953F8041B40F835
:103DF000041BECE7A4450008043B0020043B002022
:103E0000043B002000F0BEB84FF08043586A704772
:103E10004FF08043002258631A610222DA60704733
:103E20004FF080430022DA60704700004FF080437B
:103E300058637047FEE7000070B51B4B0163002517
:103E4000044686B0586085620E46FFF701FB04F118
:103E50001003C4E904334FF0FF33C4E90635C4E965
:103E60000044A560E562FFF7CFFF2B460246C4E998
:103E7000082304F134010D4A256580232046FFF70D
:103E80000FFC0123E0600A4A0375009272680192F8
:103E9000B268CDE90223074B6846CDE90435FFF748
:103EA00027FC06B070BD00BF603A00201C4500082A
:103EB00021450008353E0008024AD36A1843D06203
:103EC000704700BF38380020244B2548DA6A42F09A
:103ED000070210B4DA62DA6A224C22F00702DA62D0
:103EE000DA6ADA6C42F00702DA64DA6E42F007024C
:103EF000DA664FF09042DB6E4FF0AA310023536038
:103F00009160D0604FF6FF7050611362536214608D
:103F10001024C2F80434C2F80814C2F80C444FF656
:103F2000F774C2F814449924C2F82034C2F8244427
:103F30000D4CC2F80044C2F80438C2F80818C2F8A0
:103F40000C38C2F81408C2F82038C2F82438C2F875
:103F500000385DF8044B00F055B800BF0010024077
:103F6000000100240001002850000A0008B500F0FC
:103F700005FAFFF76DFBBDE80840FFF701BF000041
:103F8000704700000F4B9A6D42F001029A659A6FDC
:103F900042F001029A670C4A9B6F936843F0010359
:103FA00093604FF080434F229A624FF0FF32DA6203
:103FB00000229A615A63DA605A6001225A611A60DB
:103FC000704700BF00100240002004E04FF0804224
:103FD00008B51169D3680B40D9B2C9439B07116179
:103FE00007D5302383F31188FFF758FB002383F3B1
:103FF000118808BD08B5FFF779FABDE8084000F060
:1040000099B900005A4B4FF0FF319A6A99629A6A47
:1040100000229A62986AD86A60F00700D862D86A6B
:1040200000F00700D862D86A186B1963186B1A631E
:10403000186B986B9963986B9A63986BD86BD9637C
:10404000D86BDA63D86B186C1964196C1A641A6C23
:10405000484A4FF4E06111601A6E474942F001028C
:104060001A66D3F8802022F00102C3F88020D3F82A
:1040700080209A6D42F080529A659A6F22F08052A9
:104080009A679A6F4FF440720A604A6912F480622C
:10409000FBD14A601A6822F0F00242F060021A6016
:1040A0001A6842F001021A601A689107FCD50022D2
:1040B0009A609A6812F00C02FBD1D3F8901011F4B8
:1040C000407F1EBF4FF48031C3F89010C3F890209A
:1040D00061221A601A689207FCD500229A609A68D9
:1040E00012F00C0FFBD169221A60D3F8942022F44D
:1040F000706242F4C062C3F894201A6842F48032BD
:104100001A601A689003FCD5D3F8902022F003229D
:10411000C3F89020194ADA601A6842F080721A6077
:104120001A689101FCD5164A1A611A6842F0806239
:104130001A601A681201FCD500229A600D49114AD2
:10414000C3F888200A6822F0070242F004020A60DD
:104150000A6802F00702042AFAD19A6842F00302C0
:104160009A609A6802F00C020C2AFAD1704700BFDC
:1041700000100240002002400070004003140001C3
:10418000000C100055550134074A08B5536903F077
:104190000103536123B1054A13680BB15068984776
:1041A000BDE80840FFF778B900040140843A0020D8
:1041B000074A08B5536903F00203536123B1054A66
:1041C00093680BB1D0689847BDE80840FFF764B921
:1041D00000040140843A0020074A08B5536903F0FF
:1041E0000403536123B1054A13690BB15069984721
:1041F000BDE80840FFF750B900040140843A0020B0
:10420000074A08B5536903F00803536123B1054A0F
:1042100093690BB1D0699847BDE80840FFF73CB9F6
:1042200000040140843A0020074A08B5536903F0AE
:104230001003536123B1054A136A0BB1506A9847C2
:10424000BDE80840FFF728B900040140843A002087
:10425000164B10B55C6904F478725A61A30604D554
:10426000134A936A0BB1D06A9847600604D5104A86
:10427000136B0BB1506B9847210604D50C4A936B16
:104280000BB1D06B9847E20504D5094A136C0BB10A
:10429000506C9847A30504D5054A936C0BB1D06CBC
:1042A0009847BDE81040FFF7F7B800BF0004014091
:1042B000843A0020194B10B55C6904F47C425A61C1
:1042C000620504D5164A136D0BB1506D984723054E
:1042D00004D5134A936D0BB1D06D9847E00404D513
:1042E0000F4A136E0BB1506E9847A10404D50C4AC7
:1042F000936E0BB1D06E9847620404D5084A136FD1
:104300000BB1506F9847230404D5054A936F0BB146
:10431000D06F9847BDE81040FFF7BEB800040140D9
:10432000843A002008B5FFF751FEBDE80840FFF7CA
:10433000B3B80000062108B50846FFF7EBF80621E0
:104340000720FFF7E7F806210820FFF7E3F806212A
:104350000920FFF7DFF806210A20FFF7DBF8062126
:104360001720FFF7D7F806212820FFF7D3F8BDE87C
:10437000084007211C20FFF7CDB8000008B5FFF763
:1043800039FE00F007F8FFF7FBFDBDE80840FFF736
:1043900039BD00000023054A19460133102BC2E93C
:1043A000001102F10802F8D1704700BF843A0020E2
:1043B0000B460146184600F009B80000024B0A46B9
:1043C00001461868FFF714BC1811002010B5054C01
:1043D00013462CB10A4601460220AFF3008010BDFF
:1043E0002046FCE700000000024B01461868FFF77A
:1043F00003BC00BF1811002010B5013902449042DF
:1044000001D1002005E0037811F8014FA34201D04B
:10441000181B10BD0130F2E72DE9F041A3B1C91A14
:1044200017780144044603F1FF3C8C42204601D931
:10443000002009E00578BD4204F10104F5D10CEB40
:104440000405D618A54201D1BDE8F08115F8018D0B
:1044500016F801EDF045F5D0E7E70000034611F846
:10446000012B03F8012B002AF9D170476F72672ED8
:104470006172647570696C6F742E4D6174656B4CFC
:104480003433312D4453686F7400000040A2E4F1CE
:10449000646891060041A3E5F26569920700000097
:1044A0004261642043414E496661636520696E64E0
:1044B00065782E0080000000008000000000800071
:1044C000000000000000000095180008D920000836
:1044D00035200008D5180008E1180008ED1A00087A
:1044E000A5180008B5180008A9180008B118000898
:1044F000AD180008091A0008B9180008FD230008C3
:10450000AD230008C9180008DD1900086330000059
:104510000C45000890380020603A00206D61696EFB
:104520000069646C650000002604000000000000C3
:104530000060030000000000FE2A0100D204000019
:104540001C1100200000000000000000000000001E
:10455000000000000000000000000000000000005B
:10456000000000000000000000000000000000004B
:10457000000000000000000000000000000000003B
:10458000000000000000000000000000000000002B
:10459000000000000000000000000000000000001B
:1045A00000000000FFFFFFFFFFFFFFFFFFFFFFFF17
:1045B000FFFFFFFFFFFFFFFFFFFFFFFFFFFFFFFF0B
:1045C000FFFFFFFFFFFFFFFFFFFFFFFFFFFFFFFFFB
:1045D000FFFFFFFFFFFFFFFFFFFFFFFFFFFFFFFFEB
:1045E000FFFFFFFFFFFFFFFFFFFFFFFFFFFFFFFFDB
:10A0000000040020A1AF0008D974010835740108CC
:10A01000A1740108357401086D740108A3AF00082C
:10A02000A3AF0008A3AF0008A3AF000819EF010811
:10A03000A3AF0008A3AF0008A3AF0008A3AF0008B8
:10A04000A3AF0008A3AF0008A3AF0008A3AF0008A8
:10A05000A3AF0008A3AF0008612602088926020802
:10A06000B1260208D9260208012702084DF6010888
:10A0700061F6010875F6010889F601089DF60108E8
:10A08000B1F60108C5F60108A3AF0008F56601089E
:10A090002167010831670108A3AF000829270208DA
:10A0A00025280208352802085528020859280208E0
:10A0B0006D280208A3AF0008A3AF0008A3AF0008F3
:10A0C000A3AF000839FA01086DFB0108A3AF00082F
:10A0D000A3AF0008FD270208A3AF0008112802085B
:10A0E0008D270208A3AF0008A3AF0008A3AF0008A4
:10A0F000A3AF0008A3AF0008A3AF0008A3AF0008F8
:10A10000A3AF0008A3AF0008A3AF0008A3AF0008E7
:10A11000A3AF0008A3AF0008A3AF0008A3AF0008D7
:10A12000D9F60108EDF6010801F7010815F7010855
:10A1300029F70108A3AF0008A3AF0008A3AF0008E8
:10A14000A3AF0008A3AF0008A3AF0008A3AF0008A7
:10A150003DF7010851F70108A3AF0008A3AF0008BD
:10A16000A3AF0008A3AF0008A3AF0008A3AF000887
:10A17000A3AF0008A3AF0008A3AF0008A3AF000877
:10A18000A3AF0008A3AF0008A3AF0008A3AF000867
:10A19000A3AF0008A3AF0008A3AF0008A3AF000857
:10A1A0005DB60008110B0108B51B01084D37010809
:10A1B000416E01088D88010825AE010851D60108BD
:10A1C00011DC010800000000000000000000000099
:10A1D00040A2E4F1646891069C6C7EB803E3986C3D
:10A1E0008444020003BEC59300002604FFFFFFFF66
:10A1F000FFFFFFFF81F0004102E000BF83F000435A
:10A2000030B54FEA41044FEA430594EA050F08BF11
:10A2100090EA020F1FBF54EA000C55EA020C7FEAD5
:10A22000645C7FEA655C00F0E2804FEA5454D4EB52
:10A230005555B8BF6D420CDD2C4480EA020281EA1C
:10A24000030382EA000083EA010180EA020281EA54
:10A250000303362D88BF30BD11F0004F4FEA0131A6
:10A260004FF4801C4CEA113102D0404261EB4101B5
:10A2700013F0004F4FEA03334CEA133302D052423B
:10A2800063EB430394EA050F00F0A780A4F10104F7
:10A29000D5F1200E0DDB02FA0EFC22FA05F2801831
:10A2A00041F1000103FA0EF2801843FA05F3594117
:10A2B0000EE0A5F120050EF1200E012A03FA0EFC96
:10A2C00028BF4CF0020C43FA05F3C01851EBE371C0
:10A2D00001F0004507D54FF0000EDCF1000C7EEBDD
:10A2E00000006EEB0101B1F5801F1BD3B1F5001F1B
:10A2F0000CD349085FEA30004FEA3C0C04F101043A
:10A300004FEA445212F5800F80F09A80BCF1004F62
:10A3100008BF5FEA500C50F1000041EB045141EAE4
:10A32000050130BD5FEA4C0C404141EB0101013CAD
:10A3300028BFB1F5801FE9D291F0000F04BF01469C
:10A340000020B1FA81F308BF2033A3F10B03B3F16E
:10A3500020020CDA0C3208DD02F1140CC2F10C02FE
:10A3600001FA0CF021FA02F10CE002F11402D8BF5C
:10A37000C2F1200C01FA02F120FA0CFCDCBF41EA28
:10A380000C019040E41AA2BF01EB0451294330BDF7
:10A390006FEA04041F3C1CDA0C340EDC04F11404D4
:10A3A000C4F1200220FA04F001FA02F340EA0300AB
:10A3B00021FA04F345EA030130BDC4F10C04C4F1F1
:10A3C000200220FA02F001FA04F340EA03002946D1
:10A3D00030BD21FA04F0294630BD94F0000F83F41B
:10A3E000801306BF81F480110134013D4EE77FEAFE
:10A3F000645C18BF7FEA655C29D094EA050F08BF4A
:10A4000090EA020F05D054EA000C04BF194610462A
:10A4100030BD91EA030F1EBF0021002030BD5FEA6E
:10A42000545C05D14000494128BF41F0004130BD96
:10A4300014F580043CBF01F5801130BD01F00045EA
:10A4400045F0FE4141F470014FF0000030BD7FEA5D
:10A45000645C1ABF194610467FEA655C1CBF0B4658
:10A46000024650EA013406BF52EA033591EA030F6F
:10A4700041F4002130BD00BF90F0000F04BF002167
:10A48000704730B54FF4806404F132044FF000059A
:10A490004FF0000150E700BF90F0000F04BF002113
:10A4A000704730B54FF4806404F1320410F0004579
:10A4B00048BF40424FF000013EE700BF42004FEA74
:10A4C000E2014FEA31014FEA02701FBF12F07F43F1
:10A4D00093F07F4F81F06051704732F07F4208BFA8
:10A4E000704793F07F4F04BF41F40021704730B5AF
:10A4F0004FF4607401F0004521F000411CE700BFFB
:10A5000050EA010208BF704730B54FF000050AE07D
:10A5100050EA010208BF704730B511F0004502D57E
:10A52000404261EB41014FF4806404F132045FEA80
:10A53000915C3FF4D8AE4FF003025FEADC0C18BF29
:10A5400003325FEADC0C18BF033202EBDC02C2F11B
:10A55000200300FA03FC20FA02F001FA03FE40EAAD
:10A560000E0021FA02F11444BDE600BF70B54FF0B1
:10A57000FF0C4CF4E06C1CEA11541DBF1CEA13558F
:10A5800094EA0C0F95EA0C0F00F0DEF82C4481EAF7
:10A59000030621EA4C5123EA4C5350EA013518BF17
:10A5A00052EA033541F4801143F4801338D0A0FB04
:10A5B00002CE4FF00005E1FB02E506F00042E0FBB1
:10A5C00003E54FF00006E1FB03569CF0000F18BFB7
:10A5D0004EF0010EA4F1FF04B6F5007F64F540745F
:10A5E00004D25FEA4E0E6D4146EB060642EAC621F2
:10A5F00041EA55514FEAC52040EA5E504FEACE2E5F
:10A60000B4F1FD0C88BFBCF5E06F1ED8BEF1004F61
:10A6100008BF5FEA500E50F1000041EB045170BDDD
:10A6200006F0004646EA010140EA020081EA030121
:10A63000B4EB5C04C2BFD4EB0C0541EA045170BD1D
:10A6400041F480114FF0000E013C00F3AB8014F197
:10A65000360FDEBF002001F0004170BDC4F10004E0
:10A66000203C35DA0C341BDC04F11404C4F1200561
:10A6700000FA05F320FA04F001FA05F240EA0200BC
:10A6800001F0004221F0004110EBD37021FA04F6F2
:10A6900042EB06015EEA430E08BF20EAD37070BDAC
:10A6A000C4F10C04C4F1200500FA04F320FA05F00B
:10A6B00001FA04F240EA020001F0004110EBD3700D
:10A6C00041F100015EEA430E08BF20EAD37070BD7D
:10A6D000C4F1200500FA05F24EEA020E20FA04F356
:10A6E00001FA05F243EA020321FA04F001F0004105
:10A6F00021FA04F220EA020000EBD3705EEA430E76
:10A7000008BF20EAD37070BD94F0000F0FD101F0A4
:10A710000046400041EB010111F4801F08BF013CDD
:10A72000F7D041EA060195F0000F18BF704703F01B
:10A730000046520043EB030313F4801F08BF013DA2
:10A74000F7D043EA0603704794EA0C0F0CEA13555E
:10A7500018BF95EA0C0F0CD050EA410618BF52EA18
:10A760004306D1D181EA030101F000414FF000001E
:10A7700070BD50EA410606BF1046194652EA43062C
:10A7800019D094EA0C0F02D150EA013613D195EAA0
:10A790000C0F05D152EA03361CBF104619460AD1E8
:10A7A00081EA030101F0004141F0FE4141F47001F2
:10A7B0004FF0000070BD41F0FE4141F4780170BDE2
:10A7C00070B54FF0FF0C4CF4E06C1CEA11541DBF47
:10A7D0001CEA135594EA0C0F95EA0C0F00F0A7F849
:10A7E000A4EB050481EA030E52EA03354FEA013176
:10A7F00000F088804FEA03334FF0805545EA131389
:10A8000043EA12634FEA022245EA111545EA106550
:10A810004FEA00260EF000419D4208BF964244F1E7
:10A82000FD0404F5407402D25B084FEA3202B61A06
:10A8300065EB03055B084FEA32024FF480104FF4DA
:10A84000002CB6EB020E75EB030E22BFB61A75464E
:10A8500040EA0C005B084FEA3202B6EB020E75EBE1
:10A86000030E22BFB61A754640EA5C005B084FEA49
:10A870003202B6EB020E75EB030E22BFB61A754616
:10A8800040EA9C005B084FEA3202B6EB020E75EB21
:10A89000030E22BFB61A754640EADC0055EA060EE2
:10A8A00018D04FEA051545EA16754FEA06164FEA25
:10A8B000C30343EA52734FEAC2025FEA1C1CC0D1D1
:10A8C00011F4801F0BD141EA00014FF000004FF05E
:10A8D000004CB6E711F4801F04BF01430020B4F11F
:10A8E000FD0C88BFBCF5E06F3FF6AFAEB5EB030CD7
:10A8F00004BFB6EB020C5FEA500C50F1000041EBD4
:10A90000045170BD0EF0004E4EEA113114EB5C04A0
:10A91000C2BFD4EB0C0541EA045170BD41F4801173
:10A920004FF0000E013C90E645EA060E8DE60CEA7B
:10A93000135594EA0C0F08BF95EA0C0F3FF43BAF98
:10A9400094EA0C0F0AD150EA01347FF434AF95EA4F
:10A950000C0F7FF425AF104619462CE795EA0C0F33
:10A9600006D152EA03353FF4FDAE1046194622E700
:10A9700050EA410618BF52EA43067FF4C5AE50EADA
:10A9800041047FF40DAF52EA43057FF4EBAE12E7CA
:10A990004FF0FF3C06E000BF4FF0010C02E000BFAB
:10A9A0004FF0010C4DF804CD4FEA410C7FEA6C5C8E
:10A9B0004FEA430C18BF7FEA6C5C1BD001B050EA31
:10A9C000410C0CBF52EA430C91EA030F02BF90EA1C
:10A9D000020F0020704710F1000F91EA030F58BFDB
:10A9E000994208BF90422CBFD8176FEAE37040F03D
:10A9F000010070474FEA410C7FEA6C5C02D150EADB
:10AA0000013C07D14FEA430C7FEA6C5CD6D152EA95
:10AA1000033CD3D05DF8040B704700BF844610465A
:10AA200062468C461946634600E000BF01B5FFF759
:10AA3000B7FF002848BF10F1000F01BD4DF808ED29
:10AA4000FFF7F4FF0CBF012000205DF808FB00BFFA
:10AA50004DF808EDFFF7EAFF34BF012000205DF854
:10AA600008FB00BF4DF808EDFFF7E0FF94BF0120A1
:10AA700000205DF808FB00BF4DF808EDFFF7CEFFA2
:10AA800094BF012000205DF808FB00BF4DF808EDE1
:10AA9000FFF7C4FF34BF012000205DF808FB00BFB2
:10AAA0004FEA410C7FEA6C5C02D150EA013C0AD1CA
:10AAB0004FEA430C7FEA6C5C02D152EA033C02D1BC
:10AAC0004FF0000070474FF0010070474FEA41021D
:10AAD00012F5001215D211D56FF47873B3EB6252F0
:10AAE00012D94FEAC12343F0004343EA505311F017
:10AAF000004F23FA02F018BF404270474FF00000A9
:10AB0000704750EA013005D111F0004008BF6FF0E6
:10AB1000004070474FF00000704700BF4A0011D25C
:10AB200012F5001211D20DD56FF47873B3EB6252A7
:10AB30000ED44FEAC12343F0004343EA505323FAB3
:10AB400002F070474FF00000704750EA013002D128
:10AB50004FF0FF3070474FF0000070474FEA41025E
:10AB6000B2F1E04324BFB3F5001CDCF1FE5C0DD96B
:10AB700001F0004C4FEAC0024CEA5070B2F1004FB5
:10AB800040EB830008BF20F00100704711F0804FB8
:10AB900021D113F13872BCBF01F00040704741F47D
:10ABA00080114FEA5252C2F11802C2F1200C10FA81
:10ABB0000CF320FA02F018BF40F001004FEAC12365
:10ABC0004FEAD32303FA0CFC40EA0C0023FA02F309
:10ABD0004FEA4303CCE77FEA625307D150EA0133DF
:10ABE0001EBF4FF0FE4040F44000704701F00040AF
:10ABF00040F0FE4040F40000704700BF7BB972B9DE
:10AC00000029BEBF00204FF0004106E008BF002829
:10AC10001CBF6FF000414FF0FF3000F0BFB9ADF145
:10AC2000080C6DE904CE002909DB002B1ADB00F0CB
:10AC30004DF8DDF804E0DDE9022304B0704740423E
:10AC400061EB4101002B1BDB00F040F8DDF804E074
:10AC5000DDE9022304B0404261EB4101524263EB63
:10AC600043037047524263EB430300F02FF8DDF8D3
:10AC700004E0DDE9022304B0404261EB410170478A
:10AC8000524263EB430300F021F8DDF804E0DDE914
:10AC9000022304B0524263EB4303704753B94AB9ED
:10ACA000002908BF00281CBF4FF0FF314FF0FF30D4
:10ACB00000F074B9ADF1080C6DE904CE00F006F8AF
:10ACC000DDF804E0DDE9022304B070472DE9F04728
:10ACD000089D04468E46002B4DD18A42944669D980
:10ACE000B2FA82F252B101FA02F3C2F1200120FA63
:10ACF00001F10CFA02FC41EA030E94404FEA1C48B1
:10AD0000210CBEFBF8F61FFA8CF708FB16E341EAAC
:10AD1000034306FB07F199420AD91CEB030306F132
:10AD2000FF3080F01F81994240F21C81023E634453
:10AD30005B1AA4B2B3FBF8F008FB103344EA0344F7
:10AD400000FB07F7A7420AD91CEB040400F1FF330C
:10AD500080F00A81A74240F207816444023840EA49
:10AD60000640E41B00261DB1D4400023C5E9004382
:10AD70003146BDE8F0878B4209D9002D00F0EF8005
:10AD80000026C5E9000130463146BDE8F087B3FA38
:10AD900083F6002E4AD18B4202D3824200F2F98020
:10ADA000841A61EB030301209E46002DE0D0C5E923
:10ADB000004EDDE702B9FFDEB2FA82F2002A40F06F
:10ADC0009280A1EB0C014FEA1C471FFA8CFE012672
:10ADD000200CB1FBF7F307FB131140EA01410EFB16
:10ADE00003F0884208D91CEB010103F1FF3802D2BD
:10ADF000884200F2CB804346091AA4B2B1FBF7F0B7
:10AE000007FB101144EA01440EFB00FEA64508D9D9
:10AE10001CEB040400F1FF3102D2A64500F2BB8016
:10AE20000846A4EB0E0440EA03409CE7C6F1200765
:10AE3000B34022FA07FC4CEA030C20FA07F401FAAB
:10AE400006F31C43F9404FEA1C4900FA06F3B1FB34
:10AE5000F9F8200C1FFA8CFE09FB181140EA014199
:10AE600008FB0EF0884202FA06F20BD91CEB010136
:10AE700008F1FF3A80F08880884240F28580A8F18E
:10AE800002086144091AA4B2B1FBF9F009FB1011E0
:10AE900044EA014100FB0EFE8E4508D91CEB01017E
:10AEA00000F1FF346CD28E456AD90238614440EA21
:10AEB0000840A0FB0294A1EB0E01A142C846A646A1
:10AEC00056D353D05DB1B3EB080261EB0E0101FA2A
:10AED00007F722FA06F3F1401F43C5E90071002687
:10AEE0003146BDE8F087C2F12003D8400CFA02FCDD
:10AEF00021FA03F3914001434FEA1C471FFA8CFEED
:10AF0000B3FBF7F007FB10360B0C43EA064300FBDC
:10AF10000EF69E4204FA02F408D91CEB030300F17A
:10AF2000FF382FD29E422DD9023863449B1B89B231
:10AF3000B3FBF7F607FB163341EA034106FB0EF3BA
:10AF40008B4208D91CEB010106F1FF3816D28B4267
:10AF500014D9023E6144C91A46EA004638E72E4633
:10AF6000284605E70646E3E61846F8E64B45A9D22B
:10AF7000B9EB020864EB0C0E0138A3E74646EAE79A
:10AF8000204694E74046D1E7D0467BE7023B614448
:10AF900032E7304609E76444023842E7704700BFB1
:10AFA00002E000F000F8FEE772B6374880F3088848
:10AFB000364880F3098836483649086040F2000078
:10AFC000CCF200004EF63471CEF200010860BFF3FF
:10AFD0004F8FBFF36F8F40F20000C0F2F0004EF6CB
:10AFE0008851CEF200010860BFF34F8FBFF36F8F1F
:10AFF0004FF00000E1EE100A4EF63C71CEF2000177
:10B000000860062080F31488BFF36F8F17F0DEF816
:10B0100017F0E6F94FF055301F491B4A91423CBFEB
:10B0200041F8040BFAE71D49184A91423CBF41F828
:10B03000040BFAE71A491B4A1B4B9A423EBF51F8D0
:10B04000040B42F8040BF8E700201849184A914213
:10B050003CBF41F8040BFAE717F0BCF817F024FAEC
:10B06000144C154DAC4203DA54F8041B8847F9E739
:10B0700000F0E4FA114C124DAC4203DA54F8041B10
:10B080008847F9E717F0A4B800040020000E00205C
:10B0900000A0000808ED00E00001002000040020EE
:10B0A00088E20208000E0020FC0F002000100020A3
:10B0B000507C0020A0A10008C4A10008C4A1000881
:10B0C000C4A100082DE9F04F2DED108AC1F80CD075
:10B0D000C3689D46BDEC108ABDE8F08F002383F362
:10B0E00011882846A047002016F068FAFEE716F0FF
:10B0F000DFF800DFFEE7000010F8012B11F8013B3C
:10B10000012A28BF9A42F7D0D01A7047034613F895
:10B11000012B002AFBD1181A0138704701F0FF01FA
:10B12000102A2BDB10F0070F08D010F8013B013A72
:10B130008B422DD010F0070F42B3F6D1F0B441EAA4
:10B14000012141EA014122F007047FF000070023BA
:10B15000F0E80256083C85EA010586EA010685FA10
:10B1600047F5A3FA87F586FA47F6A5FA87F68EB96A
:10B17000EED1F0BC01F0FF0102F0070232B110F88D
:10B18000013B013A83EA010313B1F8D10020704773
:10B1900001387047002D06BF35460338073815F0D3
:10B1A000010F07D1013015F4807F02BF013015F483
:10B1B000C03F0130F0BC0138704700BF38B50022F5
:10B1C000002304460D46FFF743FC28B920462946D4
:10B1D000BDE8384000F00AB8204605F1004100F013
:10B1E00005F8404261EB410138BD00BFD0B50C4BC2
:10B1F000002206460F46FFF7B9F9FFF78FFC044619
:10B20000FFF73AF9074B0022FFF7B0F902460B4669
:10B2100030463946FEF7F2FFFFF780FC2146D0BDED
:10B220000000F03D0000F0417047000070B504469A
:10B23000283005F0A1FD04F14C000AF0C5F904F531
:10B240002F7006F0E7FB04F2446006F0BBFC04F547
:10B25000D4630021012043E9020104F5D5600AF01E
:10B260002FFB154B1549196004F2CC6000231426FE
:10B270009DB206FB05120133127C002AF8D1104B57
:10B280001D80104B1A6812B10F480CF029F9186094
:10B2900004F58053012104F5F450C3F8802E83F89F
:10B2A0007E1E04300BF0DCFA084B1A680AB108481D
:10B2B000EBE71C60204670BD802F00201C6E02084A
:10B2C0007E2F0020402F0020FC6C0208041000207C
:10B2D000176D020838B5224D044616F02BFF16F004
:10B2E0003DFF286820231A46006C4FF4E13102F03C
:10B2F00075FF28684FF4807380224FF4E131C06CF1
:10B3000002F06CFF204600F0CDF916F027FF204632
:10B3100001F0A6FA04F1280005F03CFE16F01EFF2D
:10B320000AF0BAFA2B68D86A03685B68984710B1CC
:10B330000C480BF017FB2B68586A03681B6898478A
:10B34000204601F005FD04F2446006F0F9FD04F525
:10B35000D5600AF059FB0CF0F1F8034B186038BDCA
:10B3600030100020386D0208001000200148FFF75F
:10B37000B1BF00BF38100020F0B52DED028B90F961
:10B380005236082B8BB06BD1374D2C78002C67D1FF
:10B390000CF0D4F8354B196840F2DC53411A99424D
:10B3A00002460CD901232B70224623462146204613
:10B3B0000BB0BDEC028BBDE8F04006F0DDBD2C4EBD
:10B3C0003368C31A1D2B4BD92A4B04AD03F1180760
:10B3D000186859682C4603C40833BB422546F7D188
:10B3E000254D9FED268A326000242B78234403F0FC
:10B3F00007030AAA03EB43031344013413F8162C82
:10B4000007EE902AF8EEE77A13F8172C13F8183C99
:10B4100067EE887AFCEEE77ACDED017A07EE902AA6
:10B42000F8EEE77A9DF8042067EE887AFCEEE77A7A
:10B43000CDED027A07EE903AF8EEE77A9DF8081023
:10B4400067EE887A0023FCEEE77ACDED037A9DF86B
:10B450000C0006F091FD082CC7D12B7801332B701E
:10B460000BB0BDEC028BF0BD0810002000100020D6
:10B470000C100020F86B0208101000209A99993ED9
:10B480002DE9F341144C154EDFF86080144F20462F
:10B4900016F0B8FD134A0146121B134801F02AFBAF
:10B4A00015F028FE0446A4B1206AE1690191B0427A
:10B4B00014BF251AA8EB060516F0A4FD0199024653
:10B4C0002B46384601F016FB204615F023FE0446B5
:10B4D000E9E702B0BDE8F08100010020000400208F
:10B4E000626D020800040020586D0208000E002062
:10B4F00010B5114C2368586A0368DB6C984704F058
:10B5000073FA2368986A03680522DB69002198476B
:10B510002368986A036864211B6998472368986ABE
:10B52000036828215B6898472368986A0368BDE828
:10B5300010401B69002118473010002038B505461F
:10B540000BF0FCFF2F4A1368C31AB3F57A7F044649
:10B550000BD92D4B10601B7823B92C4A536983F00B
:10B5600008035361284601F0DFFB05F0F7FD284A88
:10B57000136841F28831E31A8B4206D9016821B180
:10B5800014600289234801F0B5FA2B7EDA070AD548
:10B59000214A136841F28831E31A8B4203D92846C5
:10B5A0001460FFF76DFF2B7E9B0711D41B4A1368B5
:10B5B000E31A132B04D905F24460146006F0C2FCB0
:10B5C000284601F01BFB2846BDE83840FFF7D4BEF3
:10B5D0000BF0B4FF43F698239842E7D91048FFF7E1
:10B5E00087FF104816F0BAFCBFF34F8F0E490F4B80
:10B5F000CA6802F4E0621343CB60BFF34F8F00BF11
:10B60000FDE700BF14100020000E002000040048D9
:10B610001C100020746D020818100020201000205B
:10B6200038100020010007B000ED00E00400FA052A
:10B630000148FFF783BF00BF3810002038B5054B25
:10B640001C6823680A461D68034B01462046A8472C
:10B65000002038BD301000202410002010B50A4C06
:10B660002046FFF7E3FD094A0949204617F056F93D
:10B670000BF0DEFB074B084A1860BDE81040074995
:10B68000074802F0C5BC00BF38100020E04600208B
:10B6900029B200083010002031B600086DB3000850
:10B6A0002410002013B5044605F088F803F0BAFE14
:10B6B000204605F003F818B1B4F90030022B0BD086
:10B6C00005F000FB03F080FB02230DF1060120468C
:10B6D000ADF8063005F0AAFA02230DF10601204666
:10B6E000ADF8063005F094FA02B0BDE8104004F061
:10B6F00023BF000030B52DED028B83B069461046A4
:10B7000001F0A4FE002840D1224B1C68224B1A787D
:10B7100052B9606A01251D7003681B689847E06A8A
:10B72000036829469B6B98470BF008FF9FED1B8A27
:10B73000DDED017A1A4B9FED1B0A186067EE887ADF
:10B74000194BDFED1A0AFCEEE77A2520C3ED007AEB
:10B75000174B93F8513607EE103AB8EEC77AB7EEAA
:10B76000001A27EE000A03F0A9FADDED017AE06A7B
:10B7700067EE887A0368FCEEE77AF0EE400ADB6B4E
:10B780009DED000A17EE901A984703B0BDEC028BAE
:10B7900030BD00BF30100020E02E002000007A44B1
:10B7A000DC2E00200AD7233CD82E00200000000009
:10B7B0003810002010B50C4C2368A3B10BF0BEFE6E
:10B7C0002368C01A094B1B6898420CD9084BDFED5F
:10B7D000090A1B68D86A03680021DB6BB0EE600AB7
:10B7E00098470023236010BDDC2E0020D82E0020B7
:10B7F0003010002000000000BFF34F8F0549064BBA
:10B80000CA6802F4E0621343CB60BFF34F8F00BFFE
:10B81000FDE700BF00ED00E00400FA0513B51022BB
:10B82000002104468DF8072017F088F9054B1B68A6
:10B83000D86A03680DF107021B6B2146984702B0D6
:10B8400010BD00BF30100020F0B58BB01746044685
:10B850000E460BF073FE054603F076FA03464FF4EE
:10B86000C87005F5167504F58054B3FBF0F202FBC1
:10B87000103315FA83F3C4F8783EFD7E35B91F48BE
:10B880000BF070F884F87C5E0BB0F0BD384605A96B
:10B8900001F0E6FF07460028F6D101A8FFF7BEFF3A
:10B8A0009DF8165001A92A460DF1170017F00EF960
:10B8B00028B113480BF056F884F87C7EE4E70F2D8E
:10B8C0000CD8D4F8783E84F87C5EA3F51673C4F8DF
:10B8D000783E29460B480BF045F8D5E79DF8141043
:10B8E0000029D1D0304612F007FE9DF8142094F8BC
:10B8F0007E1E05480BF036F8C6E700BF5C6F0208F5
:10B90000876F0208A86F0208CA6F020813B50446C1
:10B9100001A9104601F09AFB20B99DF804102046B9
:10B9200001F0CEFA02B010BD07B5104601A901F032
:10B9300045FE58B9074B9DF804101B68D86AA1F161
:10B94000FF02036851421B685141984703B05DF8FC
:10B9500004FB00BF3010002010B504460846114615
:10B960001A46002306F008FB012384F8383610BD80
:10B970002DE9F0432DED028B97B0804601A91046CA
:10B9800001F0C4FD00285ED1DFED318A074608F2E0
:10B9900044699DF80420FBB29A4254D916AA02EBDE
:10B9A0008303484613F8524C13F8515C13F8506C5B
:10B9B00006F008FBE400AD00F6006428E4B205F0F0
:10B9C000F805F6B237D0002835DB07EE900AB8EE5E
:10B9D000E78A07EE904A28EE288AF8EEE77AFF22F7
:10B9E00067EE887A0021FDEEE77A17EE903A18B2FA
:10B9F00003F0A2F907EE905AF8EEE77AFF2267EE1D
:10BA0000887A0021FDEEE77AC4B217EE903A18B2B8
:10BA100003F092F907EE906AF8EEE77AC5B227EEE6
:10BA2000888AFF22BDEEC88A002118EE103A18B2AB
:10BA300003F082F9C6B233462A4621464046FFF754
:10BA40008BFF0137A5E717B0BDEC028BBDE8F08393
:10BA50000AD7233C10B58CB0044601A9104601F06A
:10BA600045FC70B99DF804200DF10601204601F057
:10BA7000EBF99DF8043084F840360BF05FFDC4F814
:10BA80003C060CB010BD000030B5A1B0054601A9C0
:10BA9000104601F0D3FB0446F0B99DF80420E3B250
:10BAA0009A4219D920AA02EBC30313F8772C1AB1D2
:10BAB000042A09D00134F0E713ED1D0A13F8781CAD
:10BAC000284601F0DFF9F5E713ED1D0A13F8781C9D
:10BAD000284601F0E1F9EDE721B030BD10B5C4B062
:10BAE00004466946104601F06DFAF0B9BDF8003021
:10BAF000B3F5007F04F5D4630FD1BDF802209FEDAC
:10BB00000C7A07EE902AF8EE677A67EE877A9FED57
:10BB1000097A67EE877AC3ED007ADDE9420143E9ED
:10BB200002010BF00BFDC4F8A40644B010BD00BF29
:10BB30000AD7233C35FA8E3C38B5084615461C46D4
:10BB400012F0E2FC60B99DF81030022B07D1012CF5
:10BB500005D137A3D3E90023C5E90023012038BD6F
:10BB600040F206439C425AD015D80B2C0BD884B116
:10BB7000601E0A280DD8DFE800F02E0C0C0C360CE5
:10BB80000C0C0C3E3A00282C29D040F2F2339C4297
:10BB900049D00020E3E740F24C439C4237D00ED816
:10BBA000B4F5876F2BD040F239439C4233D040F23A
:10BBB0002E439C42EDD120A3D3E90023CCE744F6E9
:10BBC00020639C421FD044F627639C42E1D11CA312
:10BBD000D3E90023C0E71CA3D3E90023BCE71CA3DF
:10BBE000D3E90023B8E71CA3D3E90023B4E71CA3DF
:10BBF000D3E90023B0E71CA3D3E90023ACE71CA3DF
:10BC0000D3E90023A8E71CA3D3E90023A4E71CA3DE
:10BC1000D3E90023A0E71CA3D3E900239CE71CA3DE
:10BC2000D3E9002398E71CA3D3E9002394E700BFDE
:10BC3000401DA12026812A0B55340C8B2636A0A14D
:10BC4000ECFD51169C2A1F639E6AC421818A46EE30
:10BC500026417272DF25D7B7F017304A39059E5654
:10BC6000D5A4D139F922B6A7CDD269EBC51A133BB9
:10BC7000525DB1C2FEA99EBEA1A6A1951A7065E94A
:10BC800003806A5575F30087C41EDD8B3CD93120D3
:10BC90001D95ECD7875C7F21F33AEC386248A7D832
:10BCA00013B59DF81040CDE9003413460A4601460D
:10BCB000806AFFF741FF02B010BD000070B500F5CB
:10BCC00080560D46D6F8744E7CB90C21012015F033
:10BCD000FFFFC6F8740E08B9002070BD05608460CF
:10BCE0000430FAE72646A46824B12368AB42F9D1B0
:10BCF000201DF2E70C21012015F0EAFFB0600028BA
:10BD0000EAD00560B3689C60B068E9E72DE9F041CE
:10BD100090B000F5F451BDF8587004461646043151
:10BD200040F2434201A8984602F0B0F9012F0ED12B
:10BD300046EA07412046FFF7C1FF054670B90024D7
:10BD400001A802F0C5F9204610B0BDE8F08104F268
:10BD5000D46012F0D9FB0028EAD1F0E738220021A4
:10BD600002A816F0EBFE02238DF808309DF85C3037
:10BD70008DF82030189B0993BDF86430ADF8283059
:10BD8000CDE90468ADF8187007950BF0D9FB0D4BA1
:10BD9000C01841F10001CDE90C0104F2D46002A900
:10BDA00012F0B4FB084B0028D5BF9A881A680132FC
:10BDB0001218D4BF9A801A600028D4BF002401242E
:10BDC000BEE700BF40420F00F02E002030B58FB01C
:10BDD00014460D4638220021684616F0AFFEDDE914
:10BDE0001223CDE90223BDF85030ADF8103004F134
:10BDF00019030593A37E8DF81830159B0793BDF8A2
:10BE00005830ADF820300BF09BFB0D4BC31841F1BF
:10BE100000016A46CDE90A312846E17E12F0BAFBFC
:10BE2000084B0028D5BF9A881A6801321218D4BF6F
:10BE30009A801A600028D4BF002001200FB030BDC6
:10BE400040420F00F02E0020F0B591B005460E469E
:10BE5000104608A9144601F0CBFD38BB9DF82030F0
:10BE6000012B07D104F02EFF02F0AEFF04F064FBBB
:10BE700004F0A4FC1022002106AF0CA816F05EFE10
:10BE8000012239460CA88DF8382001F0D5FD0A238F
:10BE9000029307A3D3E9002380B2CDE90370CDE973
:10BEA0000023314622462846FFF790FF11B0F0BD2F
:10BEB000CDD269EBC51A133B2DE9F041ADF5487DB4
:10BEC00066AC05460E46174600214FF4C472204664
:10BED00016F034FE0BF032FB2F4B4FF47A72B0FBAE
:10BEE000F2F0186093E8070084E8070001F036FFDD
:10BEF000037C237401F032FF437C63740323A37437
:10BF0000264B5A6962610DF5DD709A68DB68A261A3
:10BF1000E361FFF783FC42F20463EA692384204B68
:10BF2000002A18681F4B29DDCDE900320DF2CB2124
:10BF30001D4BC06A502202F0FBF950210DF2CB20BC
:10BF400017F0E8FA0DF11C0884F83201414601228D
:10BF5000204601F04DFB012302930DA3D3E90023FA
:10BF600080B2CDE90380CDE9002331463A46284628
:10BF7000FFF72CFF0DF5487DBDE8F08100935022BE
:10BF80000A4BC06A0DF2CB2102F0D2F9D5E700BF0F
:10BF90009E6AC421818A46EEE42E0020D0A10008CA
:10BFA00030100020EF6F0208E86F020822C102087B
:10BFB0002DE9F0411546ADF5866D06460F4616F0A3
:10BFC000CDF808A9284601F04DFD0446002840F0B0
:10BFD0009F8001464FF4D072A4A816F0AFFD9DF8E3
:10BFE000B880B8F1100F7ED808F1FF330F2B2BD893
:10BFF00042460DF1B9010DF2D13016F077FD4246FF
:10C0000051490DF1B90017F05DFA0246B0B94F4839
:10C010000DF11F0103F0F4FB0446002C63D09DF8E2
:10C02000B83073B39DF828305BB39DF81F20013AF8
:10C03000032A6DD8DFE802F01C2E384122460DF1AC
:10C040001F010DF2D130E5E7BDF82000479447AA63
:10C050000DF11F0103F03EFF0446002843D00123E9
:10C0600000930DF2D132112347A903F005FBD4E769
:10C07000012B4DD10C9B8DF81C3147A9204604F0B3
:10C08000B3FD9DF81F30013B032B41D8DFE803F0DF
:10C090001C444A4F012B3BD10C9BADF81C3147A9E6
:10C0A000204604F0DDFDECE7012B31D10C9B4793DA
:10C0B00047A9204604F0F6FDE3E7022B28D10CA99E
:10C0C000204604F055FDDCE701238DF8903294F909
:10C0D0000030DA17CDE9A6325C210DF2D13017F02D
:10C0E00019FA8DF8D00347AC01222146A4A801F02B
:10C0F000E1FD0B23029312A3D3E9002380B2CDE923
:10C100000340CDE9002339462A463046FFF75EFE5C
:10C110000DF5866DBDE8F08101238DF89032B4F9FC
:10C120000030D6E701238DF890322368D1E702234F
:10C130008DF890322368A693CEE700BFAFF300805E
:10C14000D5A4D139F922B6A71070020819700208D7
:10C150002DE9F04FDFF8D8A08BB0804608F2D46903
:10C16000484612F053FA0546002858D00024007EB5
:10C170000694CDE90744ADF8244001F00DFF2A7E76
:10C180008DF8240005F1100107A816F0AFFC2B680C
:10C1900043F0004306930BF0D3F9224B0390C218EF
:10C1A000DAF804000E4641F1000308F5805760B349
:10C1B0000168009409690D4606A9A847A04224DC3D
:10C1C000DAF8040003689B6A9847D0E90A23CDE9AE
:10C1D00004230BF0B5F9DDE90423801A61EB0301B8
:10C1E000114B834274EB01030FD397F87D3E072B6D
:10C1F00012D90E4A87F87D4E9388013393804846C2
:10C20000039A334612F010FA09E0484612F002FA97
:10C21000002387F87D3EA1E7013387F87D3E0BB010
:10C22000BDE8F08F40420F007F841E00F02E0020FA
:10C23000102F00202DE9F0414FF00053DFF8E0808F
:10C240001B684345FCB005460C46164604D03148F1
:10C25000DC22002116F072FC4FF0005749A9C7F804
:10C260000080304601F048FB002849D19DF8243178
:10C270003B750BB9F37E3B759DF8252126480DF5DE
:10C28000937116F033FC204612F03EF94FF0005344
:10C2900007AF58758122002128A816F04FFC3946B7
:10C2A000012228A801F06EFB2823029317A3D3E9EB
:10C2B000002380B2CDE90370CDE900232146324648
:10C2C0002846FFF783FD154F3326013E16F0FF0683
:10C2D000284608D0FFF73CFF3B68986A03680121B5
:10C2E0005B689847F1E7FFF703F9204612F00CF975
:10C2F00040F0304040F4002015F030FEFFF77CFAAB
:10C300007CB0BDE8F08100BFAFF3008026417272BF
:10C31000DF25D7B7040000201600002030100020D1
:10C320009AAD44C5F0B5044689B008460E46154698
:10C3300012F0EAF868B92B7E022B26D1EB8A012B8A
:10C3400023D12A463146204609B0BDE8F040FFF728
:10C350007BBAEB8A40F20642934200F0A18016D8E5
:10C360000B2B0BD88BB1013B0A2B0ED8DFE803F067
:10C37000370D0D0D470D0D0D0D706800282B36D0B3
:10C3800040F2F232934200F0938009B0F0BD40F2E7
:10C390004C42934274D012D8B3F5876F60D040F20C
:10C3A0003942934274D040F22E429342EDD12A4654
:10C3B0003146204609B0BDE8F04000F0E7BD44F644
:10C3C0002062934254D044F627629342DDD12A463C
:10C3D0003146204609B0BDE8F040FFF77FBB2A4652
:10C3E0003146204609B0BDE8F040FFF765BD2A465A
:10C3F0003146204609B0BDE8F040FFF71BBF07AF4C
:10C4000032480AF0AFFA0122394606A88DF8182002
:10C4100001F0C8F9052302932AA3D3E9002380B2CF
:10C42000CDE90023CDE903702A4631462046FFF7C7
:10C43000CDFC0BF083F804F58054C4F8800EA4E71B
:10C440002A463146204609B0BDE8F040FFF7B0BDAE
:10C450002A463146204609B0BDE8F040FFF7F4BC5B
:10C460002A463146204609B0BDE8F040FFF742B900
:10C470002A463146204609B0BDE8F040FFF746BAEB
:10C480002A463146204609B0BDE8F040FFF74CBAD5
:10C490002A463146204609B0BDE8F040FFF768BAA9
:10C4A0002A463146204609B0BDE8F040FFF7D2BA2F
:10C4B0002A463146204609B0BDE8F040FFF7E4BA0D
:10C4C000AFF30080F017304A39059E5624700208F9
:10C4D0000A460146806AFFF725BF000049421B4B10
:10C4E000112912D8DFE801F00911110D11111111F4
:10C4F00011111519151D2125292D9A6801329A60EF
:10C5000070479A8901329A817047DA890132DA815B
:10C5100070475A8B01325A8370471A8B01321A8343
:10C5200070471A8A01321A8270475A8A01325A8237
:10C5300070479A8B01329A8370479A8A01329A82A5
:10C540007047DA8A0132DA82704700BFF02E00208D
:10C550002DE9F04F374E97B00023CDE90B330A9306
:10C56000ADF8343073680446002B5FD0324D01279C
:10C570004FF0000A4FF0000B70688DF814704FF008
:10C5800000088DF815800368CDE900AB0DF11502A8
:10C59000D3F8089005A94346C8479DF81430002BEE
:10C5A00044D0414620220EA816F0C8FA70680368ED
:10C5B00006AAD3F814800AA90DF11603C047002873
:10C5C00034DD9DF8340001F003FD0BA902468DF81F
:10C5D000500012A816F08AFA04F2D4680A9B0E934F
:10C5E0000EA9DDE90623404612F06EFA10F10D0F98
:10C5F000014603D02046FFF771FFBDE70E9812F009
:10C6000053FA03900E9812F049FA039BCDE9000704
:10C6100008AA41462046FFF78FFA18B12B8A01334A
:10C620002B82A9E76B8B01336B83A5E717B0BDE8BD
:10C63000F08F00BF102F0020F02E002007B500F271
:10C64000D461684612F0D2F9BDF80400642358435F
:10C65000BDF80030B0FBF3F080B203B05DF804FB2E
:10C66000F0B597B004460AF069FF4FF47A73B0FB57
:10C67000F3F0434B434D1B682860D86A03685B6D39
:10C6800098474FF6FF73984228BF184628810EA995
:10C690000122284601F05EF80EAB80B20293182208
:10C6A00040F255130025CDE9003203902EA3D3E9C3
:10C6B000002304952046FFF729FB237E59074ED51A
:10C6C00001220EA93048314F00F030FD0EAB80B290
:10C6D00002931F264FF4AB73CDE90036039024A3D9
:10C6E000D3E9002304952046FFF710FB7868036820
:10C6F0009B6A9847002832D03A788DF83820026833
:10C700000F924268ADF840208268ADF84220C268BE
:10C71000ADF844200269ADF846204269ADF84820E2
:10C7200082691392C269ADF85020026AADF85220B6
:10C7300007AF436AADF85430012239460EA800F025
:10C740009FFC40F2571380B2CDE90270009304952C
:10C7500009A3D3E9002301962046FFF7D7FA17B0C3
:10C76000F0BD00BFAFF30080F1C6A7C1D068080FCD
:10C77000D1F886A9B8E33A76753CA33CAE0C08CE56
:10C7800030100020E42E0020F02E0020102F00207A
:10C79000F0B506468DB000F2D46011F0B5FE2E4D16
:10C7A00020B100232B7001200DB0F0BD0AF0C6FEB1
:10C7B0002B7804463BB13046FFF740FF012102468B
:10C7C00026480AF0CFF802F0BFFA4FF4C87306F516
:10C7D0008057B0FBF3F202FB130304F5167010FA56
:10C7E00083F000238DF8183097F87C3EC7F8780E58
:10C7F00023B901228DF8182087F87E3E08A8FFF79C
:10C800000DF897F87C1EC1F11004E4B2062C28BF85
:10C81000062408AB224619440DF1190016F066F9FA
:10C82000013406AB0025029318220123E4B2CDE9BE
:10C830000032049506A3D3E9002303943046FFF7A2
:10C8400065FA87F87C5E2846AEE700BFAFF300804C
:10C85000401DA12026812A0B000E00203470020802
:10C8600070B5244D244E4FF4807386B0AB800446DF
:10C870000AF064FE4FF47A73B0FBF3F0286062882C
:10C88000B4F902307F2A98BF33700DF117010023ED
:10C8900004F108008DF8173004F0A6F941F23810C1
:10C8A00001F060FA054608B109F07CFB134B1D60EE
:10C8B000134B00225D601A702DB12B6861685B68B4
:10C8C0000122284698470F4B009304F2D46004F2EB
:10C8D00004710D4B019441F27072039011F0E0FD70
:10C8E0003178039821B106B0BDE8704011F004BE64
:10C8F00006B070BDE42E0020252F0020182F002048
:10C90000102F0020A1BC0008D1C40008082910B5D0
:10C910000C460BD8064A106801EB810310EB83002C
:10C9200004D004F099FD431C18BFC4B2204610BDCA
:10C93000E42F00202DE9F04F2DED028B00F14C0586
:10C9400093B00746284608F053FE0FF2F809D9E9DC
:10C950000089DFF8F8A09FED398A0646002E66D0E0
:10C9600096FAA6F4B4FA84F40123A3401822002115
:10C970000CA826EA030616F0E1F821463846FFF730
:10C98000C5FF0DAA8DF845002146284608F0B0FEE7
:10C9900008B9CDF834A00EAA2146284608F090FE2A
:10C9A00008B9CDF838A00DF11A022146284608F042
:10C9B0006FFE88B3BDF91A30DFED217A07EE103A29
:10C9C000B8EEC77AE7EE087ACDED0F7A07AA2146CE
:10C9D000284608F037FE28B1DDED077AFDEEE77A4C
:10C9E000CDED107A08AC4FF0000B012221460CA8C7
:10C9F000CDF830B000F0B8FC40F20A4380B2182203
:10CA0000CDE90032CDE90240CDF810B042464B46A8
:10CA10003846FFF77BF9A1E70DF11A0221462846B7
:10CA200008F01EFE0028C5D1CDF83CA0CEE713B01B
:10CA3000BDEC028BBDE8F08FAFF300800AD7233C3A
:10CA40003393884354B2FBA2AE28AFA90000C07F45
:10CA500030B50628134698BF1D4AC7B098BF155C6D
:10CA600007930C464FF07C024FF0000127A888BFC7
:10CA7000002516F063F8079B22465A210DF1BE00EF
:10CA800009F026FF5A2828BF5A2008AC8DF8BD00AF
:10CA90002146012227A88DF89C5000F08DFE00232E
:10CAA000049380B243F6FF731822CDE90240CDE92A
:10CAB0000032084804A3D3E90023FFF727F947B061
:10CAC00030BD00BFAFF30080759D040C8EA454D61A
:10CAD000F0700208381000200EB403B503AA52F813
:10CAE000041B0192FFF7B4FF02B05DF804EB03B042
:10CAF000704700000FB407B504AA072052F8041BC2
:10CB00000192FFF7A5FF03B05DF804EB04B0704796
:10CB100037B5044600F2D46011F086FD2046FFF7D9
:10CB20008DFD462802D92B4809F01CFF2046FFF74F
:10CB300097FD94F90850002D38D0002304F1080027
:10CB4000EDB201A98DF8043004F04EF82A2D224CE4
:10CB50000AD1224D2846FFF7CDFF2368986A036863
:10CB600064215B689847F5E72B2D04D11C48FFF73B
:10CB7000C1FF1C4B98474FF4FA6101A801F06CFA11
:10CB80002468A06A03684FF47A715B689847E06A8A
:10CB900003689B6A984718B1012816D0124800E034
:10CBA0001248FFF7A7FF01A801F062FA104B00221C
:10CBB0005A710AF0C3FC47F23053984207D90D4826
:10CBC00003B0BDE8304015F0C9B90B48E9E703B040
:10CBD00030BD00BF6C700208301000208A7002085F
:10CBE0009B70020838ED00E0D6700208AB700208B6
:10CBF000E42E0020263A09B0C07002082DE9F34166
:10CC000004460AF09BFC3C490B68C31A322B0546CC
:10CC10001AD93A4B1B78BBB13948027801239340AB
:10CC200023F4AA4323F055031B041B0C002B0EBF57
:10CC300001260026082343EAC6430132314E02F0A2
:10CC40001F02B36102700D6004F580560AF076FC95
:10CC5000D6F8783E984202D92046FFF799FD2A4A35
:10CC60001368EB1AB3F57A7F07D315600AF068FCF6
:10CC700002460B462046FFF74BFF2046FEF79AFD83
:10CC8000204600F031F90AF051FC04F5F455DFF8C4
:10CC90007C80074604350AF049FCC01BB0F57A7F5A
:10CCA00017D2D8F80030986A03684FF480619B6807
:10CCB000984740F2D772294601A801F0E7F92046CB
:10CCC000FFF746FA2046FFF743FC01A801F000FAFF
:10CCD000E1E7D6F8803E63B10AF030FCD6F8803E3A
:10CCE000C01AB0F57A7F04D92046FEF701FCFEF7A2
:10CCF00083FD02B0BDE8F081202F0020000E00204F
:10CD0000242F0020000400481C2F00203010002099
:10CD1000072802D82130C0B270470B2801D84A300A
:10CD2000F9E794307047000038B5044604F03CFF42
:10CD300004F054FD002504F52F74E8B2FFF7E8FF76
:10CD400001350146204604F0C3FD202DF5D138BD44
:10CD50002DE9F7433A4B1E680446706A0368DB6CA2
:10CD6000984794F91010002907DB4FF4E1331022A3
:10CD7000C9B204F1280004F0C9F9002505F1330116
:10CD8000E8B209B2013504F01FFE092DF6D13325B2
:10CD900028B201354FF47A71ADB204F095FC532DF1
:10CDA000F6D100252F464FF001095FFA85F840467D
:10CDB000FFF7AEFF41F6FF7104F09AFC4046FFF723
:10CDC000A7FF0DF1070104F061FD20B19DF80730C8
:10CDD00009FA03F31F430135202DE6D12046FFF762
:10CDE000A3FF184D706A2A68036892F85913D3F8A4
:10CDF000AC309847706A6289036839465B68984727
:10CE000004F0D2FE227B394604F032FE706A2968B3
:10CE1000036891F85813D3F8A0304FF4C8729847BC
:10CE200060694FF47A72012101F076FF4FF47A7352
:10CE300093FBF0F0C4F8B80203B0BDE8F08300BF84
:10CE400030100020982F0020F8B507460E46C1B1DB
:10CE5000202AA8BF202214460025E8B284420DD91A
:10CE6000FFF756FF36F9153023EAE37307EE903AE1
:10CE7000B8EEE70A04F014FC0135EEE7012387F869
:10CE80003836F8BD10B5044601F1320004F07EFDDD
:10CE9000012384F8383610BDF6EE007A30EE270A0A
:10CEA00010B5BCEEC00A044610EE103A0846323007
:10CEB00099B204F04FFD012384F8383610BD00000C
:10CEC00010B5084B1B680446586AFF29036805D152
:10CED0001B6D9847012384F8383610BDDB6C9847EA
:10CEE000F8E700BF301000202DE9F041044682B081
:10CEF00000AF0AF023FBB4F90E20002A054642DDFC
:10CF0000D4F83C36C31A934234BF0023012394F86B
:10CF10004066AEB1A3B17200D31D03F47E73E84640
:10CF2000ADEB030D6B461846002115F007FE3246A7
:10CF300001462046FFF788FF012384F83836C546AE
:10CF400094F83836DBB1002384F8383604F02CFE30
:10CF5000786004F091FD786804F0F6FD04F0AEFA14
:10CF6000786804F0F9FDD4F8B432D4F8B822EB1A9A
:10CF7000934204D3C4F8B4522046FFF7DBFC0837D1
:10CF8000BD46BDE8F0810023C1E7000013B50023D2
:10CF9000044601A91046019300F034FA78B9BDF8AF
:10CFA0000620012A0BD89DF804100F2907D80A3152
:10CFB00002F00102C9B204F5D56008F00BFD02B021
:10CFC00010BD00002DE9F3410446007F0D4618B165
:10CFD000A38AB3F5857F28D200231946082200953D
:10CFE000204611F07DFB6B1C0822009311460023A4
:10CFF000204611F075FB002705F102086B78FE0052
:10D000009F4206F1100113D305F5847500230095A6
:10D010004022204611F064FB237FA08A5736F60891
:10D0200083B9B0422CBF0020012002B0BDE8F081DE
:10D0300008EB0703009308220023204611F050FB61
:10D040000137DBE7801B18BF0120EEE713B504466C
:10D05000007F10B1A38A012B0CD800230091082275
:10D060001946204611F03CFB237FA08A23B9B0FA71
:10D0700080F0400902B010BD013818BF0120F9E767
:10D0800070B50C461926054632460021204615F09B
:10D0900055FD2B4620460822002111F05FFC2B1D78
:10D0A00020462022082111F059FC05F108032046F2
:10D0B0001022282111F052FC05F10A03204610220B
:10D0C000382111F04BFC05F10C03204610224821B9
:10D0D00011F044FC05F10E0320461022582111F0F6
:10D0E0003DFC05F1100320461022682111F036FCAA
:10D0F00005F1140320462022782111F02FFC05F1C0
:10D10000180320461022982111F028FC05F11A037B
:10D1100020461022A82111F021FC204605F11C0315
:10D120001022B82111F01AFC304670BD70B50C46C3
:10D130001C26054632460021204615F0FFFC2B46F2
:10D1400020462022002111F009FC2B1D2046102230
:10D15000202111F003FC05F1080320462022302194
:10D1600011F0FCFB05F10C0320461022502111F0B8
:10D17000F5FB05F10E0320461022602111F0EEFBB5
:10D1800005F1100320461022702111F0E7FB05F194
:10D19000120320461022802111F0E0FB05F1140358
:10D1A00020461022902111F0D9FB05F116032046EC
:10D1B0001022A02111F0D2FB05F118032046102205
:10D1C000B02111F0CBFB05F11A0320461022C0213B
:10D1D00011F0C4FB2046AB191022D02111F0BEFB88
:10D1E000304670BD7FB50C46009215460968002395
:10D1F0000822064611F074FA21686B1C0831216080
:10D20000009308220023304611F06AFA21680DF1DC
:10D210000E0308312160009310220123304611F0E3
:10D220005FFABDF80E0011F017FC85ED010A2368C6
:10D2300000201033236004B070BD00002DE9F043DE
:10D24000067F85B005460C4636B1838A3D2B03D94F
:10D25000012005B0BDE8F08300230393002E3BD1ED
:10D260003346009404223146284611F039FA039BD4
:10D270000433039323780F2BEAD8271D23789E428B
:10D280001BD23A4603A92846FFF7ACFF083700280F
:10D29000DED10136F2E7013FDAD0227819FB0282B3
:10D2A000224403A92846FFF79DFF0028D0D1237808
:10D2B00001332370039B9E42EDD8039B2A7FA88AEB
:10D2C0000733DB0822B9834294BF00200120C0E766
:10D2D000181A18BF0120BCE72370AE8AF600073E7B
:10D2E00010274FF008094FF00408E3E72DE9F34158
:10D2F000037F04460D4633B1838A242B10D90120C5
:10D3000002B0BDE8F08100910522194611F0E8F95C
:10D310002B78142BF3D8052700264FF00E080FE0CA
:10D32000DB000E220027B3FBF2F30B70F4E70136AB
:10D3300005EB460300930E220123204611F0D0F99D
:10D340002B789E4208FB0671F1D3237FA08A073118
:10D35000C90823B9814294BF00200120D0E7081AF0
:10D3600018BF0120CCE7000073B50C460E26054619
:10D3700032460021204615F0E1FB2B4620220021F9
:10D38000204611F0EBFA95ED010A11F037FB0DF193
:10D390000603ADF8060010222021204611F0DEFA27
:10D3A00095ED020A11F02AFB0DF10603ADF8060017
:10D3B00010223021204611F0D1FA95ED030A11F028
:10D3C0001DFB0DF10603ADF806001022204640219A
:10D3D00011F0C4FA05F1100320461222502111F079
:10D3E000BDFA05F1140320460722622111F0B6FAB6
:10D3F000204605F115030522692111F0AFFA3046E8
:10D4000002B070BD37B50446007F0D4610B1A38A47
:10D41000032B15D800231946009508222046023513
:10D4200011F05EF90023009510220821204611F02A
:10D4300057F9237FA08A2BB902288CBF0020012036
:10D4400003B030BD033818BF0120F9E77FB50446AB
:10D45000007F0D4610B1A38A042B22D80DF10E06D1
:10D460000123102200210096204611F039F9BDF861
:10D470000E0011F0F1FA1022012385ED000A114689
:10D480000096204611F02CF9BDF80E0011F0E4FAD8
:10D4900085ED010A237FA08A2BB903288CBF0020C9
:10D4A000012004B070BD043818BF0120F9E7000066
:10D4B000F7B50C4600921546096800230822064677
:10D4C00011F00EF921686F1C0831216000970023CC
:10D4D0000522304611F004F92168AF1C05312160A6
:10D4E000009700230622304611F0FAF82168033530
:10D4F00006312160009500230522304611F0F0F836
:10D50000236800200533236003B0F0BD2DE9F0430C
:10D51000067F85B005460C4636B1838A3D2B03D97C
:10D52000012005B0BDE8F08300230393002E3BD11A
:10D530003346009405223146284611F0D1F8039B6A
:10D54000053303932378142BEAD8671C23789E4273
:10D550001BD23A4603A92846FFF7AAFF0437002842
:10D56000DED10136F2E7013FDAD0227819FB0282E0
:10D57000224403A92846FFF79BFF0028D0D1237837
:10D5800001332370039B9E42EDD8039B2A7FA88A18
:10D590000733DB0822B9834294BF00200120C0E793
:10D5A000181A18BF0120BCE72370AE8AF600073EA8
:10D5B00015274FF004094FF00108E3E713B50446BF
:10D5C000007F10B1A38A012B0CD800230091082200
:10D5D0001946204611F084F8237FA08A23B9B0FAB7
:10D5E00080F0400902B010BD013818BF0120F9E7F2
:10D5F0002DE9F3470D46044600219046284640F2A7
:10D60000791215F09BFA234620220021284611F0BA
:10D61000A5F9231D02222021284611F09FF9631D40
:10D6200003222221284611F099F9A31D0322252166
:10D63000284611F093F904F1080310222821284606
:10D6400011F08CF904F1100308223821284611F05A
:10D6500085F904F1110308224021284611F07EF9D2
:10D6600004F1120308224821284611F077F904F149
:10D67000140320225021284611F070F904F11803F8
:10D6800040227021284611F069F904F12003082294
:10D69000B021284611F062F904F121030822B821D3
:10D6A000284611F05BF904F12207C0263B463146BB
:10D6B00008222846083611F051F9B6F5A07F07F187
:10D6C0000107F3D194F832308DF8073031460DF16F
:10D6D00007030822284611F041F9002604F1330A15
:10D6E0009DF807304FEAC6099E4209F5A47720D37A
:10D6F00094F83231502B28BF50238DF80730B8F101
:10D70000000F08D139460DF107030722284611F012
:10D7100025F909F24F17002604F233149DF807305B
:10D720009E4207EBC6010DD30731C80802B0BDE821
:10D73000F0870AEB060308223946284611F00EF955
:10D740000136CDE7A3190822284611F007F9013662
:10D75000E4E7000013B504460846002101602346B3
:10D76000C0F803102022019011F0F8F80198231D51
:10D770000222202111F0F2F80198631D03222221D8
:10D7800011F0ECF80198A31D0322252111F0E6F811
:10D79000019804F108031022282111F0DFF8072076
:10D7A00002B010BD08B503460846002101700122F1
:10D7B00011F0D4F8012008BD2DE9F3410D460446CF
:10D7C0000021164628467B2215F0B8F9234603228D
:10D7D0000021284611F0C2F863781F2B28BF1F23B1
:10D7E0008DF8063005220DF106030321284611F0BD
:10D7F000B5F801239DF80620DF0003F10108013B85
:10D800009A421CD894F821305A2B28BF5A238DF8FD
:10D8100007303EB939460DF107030722284611F0BB
:10D820009DF80737002622349DF807309E4207EB0B
:10D83000C6010DD30731C80802B0BDE8F08104EB82
:10D84000080308223946284611F088F84346D1E7F4
:10D85000A3190822284611F081F80136E4E70000F8
:10D86000F7B5047F05460E462CB1838A122B02D9E8
:10D87000012003B0F0BD0023194607220096284678
:10D8800010F02EFF731C009301220023072128466D
:10D8900010F026FFD4B9B31C0093052223460821BB
:10D8A000284610F01DFF0D24B378102BE0D8374622
:10D8B000B278BB1B934210D32B7FA88A0734E408AD
:10D8C000B3B9844294BF00200120D2E7AB8ADB00C9
:10D8D000083BDB08B3700824E6E7FB1C00932146F5
:10D8E00000230822284610F0FBFE08340137DFE74A
:10D8F000201A18BF0120BCE7F7B5047F05460E4685
:10D900002CB1838ACA2B02D9012003B0F0BD0023B9
:10D91000194600960822284610F0E2FE731CD4B97E
:10D920000822009311462346284610F0D9FE102401
:10D930007378C82BE8D8012372785F1C013B9342AF
:10D9400010D32B7FA88A0734E408B3B9844294BF6C
:10D9500000200120D9E7AB8ADB00083BDB087370AD
:10D960000824E5E7F31900932146002308222846FE
:10D9700010F0B6FE08343B46DEE7201A18BF01203F
:10D98000C3E70000F7B50D460446002116462846B9
:10D99000812215F0D3F8234608220021284610F0F2
:10D9A000DDFF94F901206378002AB8BF7F238DF84A
:10D9B00007309EB90DF1070307220821284610F011
:10D9C000CDFF0F27002602349DF807309E4207EB5B
:10D9D000C60105D30731C80803B0F0BD0827F1E739
:10D9E000A3190822284610F0B9FF0136ECE7000021
:10D9F00037B50446007F0D4610B1A38A072B15D812
:10DA000000231946009508222046083510F068FECC
:10DA10000123009530220821204610F061FE237F6B
:10DA2000A08A2BB906288CBF0020012003B030BD8E
:10DA3000073818BF0120F9E738B50C4600212160EE
:10DA40000546C4F8031003463022204610F086FF36
:10DA5000204605F108030122302110F07FFF072046
:10DA600038BD00002DE9F04390F81C8085B00646D3
:10DA70000D46B8F1000F06D0838AE02B03D90120B0
:10DA800005B0BDE8F083002319460D22009530460D
:10DA900010F026FE0DF10F030093032200230D2149
:10DAA000304610F01DFE9DF80F30042BE7D82B7286
:10DAB000013B032B03D8DFE803F025303B4610245D
:10DAC000B8F1000F5FD105F198030093214643465A
:10DAD0000722304610F004FE073495F898305C2B8E
:10DAE000CDD82F4695F898207B1B934252D3337F95
:10DAF000B08A0734E408002B58D1844294BF002038
:10DB00000120BDE705F110030093402201231021FD
:10DB1000304610F0E5FD5024D2E705F110030093E4
:10DB2000202201231021304610F0DAFD3024C7E70F
:10DB300005F110030093082200231021304610F055
:10DB4000CFFD1824BCE705F1100300930822002341
:10DB50001021304610F0C4FD2B7C802B8FD800277D
:10DB600005F111092B7CFC009F4204F11804A7D297
:10DB700009EB07030093082200232146304610F0EA
:10DB8000AFFD0137EEE7B38AC4EBC303DB0885F8CA
:10DB90009830A2E707F19903009321460023082259
:10DBA000304610F09DFD083401379BE7201A18BF5E
:10DBB000012065E7F7B50C46137809688DF8063043
:10DBC00015460DF106030322064610F0C7FE216834
:10DBD000033121602B78013B032B0CD8DFE803F0E5
:10DBE000020D161F05F108034022304610F0B6FE64
:10DBF00023684033236003B0F0BD05F10803202201
:10DC0000304610F0ABFE23682033F3E705F108033C
:10DC10000822304610F0A2FE23680833EAE72B7A88
:10DC2000802B28BF80238DF8073008220DF10703D1
:10DC3000304610F093FE236808332360002709352F
:10DC40009DF807309F42D6D2EB1921680822304652
:10DC500010F084FE2368083323600137F0E70000EA
:10DC600073B50C46137809688DF8073015460DF129
:10DC700007030222064610F071FE2168023121607E
:10DC80002B78012B03D0022B0BD002B070BD05F115
:10DC900008034022304610F061FE236840332360C1
:10DCA000F3E705F108032022304610F057FE236801
:10DCB0002033F4E773B50D46044600211646284686
:10DCC00040F2731214F03AFF0523224601A92846B8
:10DCD0000193FFF76FFF019B04F19002053301A947
:10DCE00028460193FFF766FF019B04F59072063307
:10DCF00001A928460193FFF7B3FF019B04F5987231
:10DD0000063301A928460193FFF7AAFF94F8403192
:10DD10005C2B28BF5C238DF803304EB90DF1030353
:10DD200001990722284610F019FE019B0733019341
:10DD3000002604F241149DF8033001999E4203D35A
:10DD40000731C80802B070BDA3190822284610F098
:10DD500005FE019B083301930136ECE7004870474C
:10DD6000407102080121884238BF084613F0B0BF55
:10DD7000FFF7F8BF08B113F0AFBF7047FFF7FABF66
:10DD800010B4026854681A4623465DF8044B1847DD
:10DD90000020704701207047002070470020704726
:10DDA0000020704770470000002070470020704737
:10DDB000704700007047000037B505460C468322C7
:10DDC000011D01A800F062F9611EC9B202299EBFBF
:10DDD00005EBC1010023C1E9073301A800F078F980
:10DDE00003B030BD2DE9F7431E461B885B0705468F
:10DDF000884620D4011D422201A800F047F92C4694
:10DE000005F118094C4513D0E3696BB12B6828461E
:10DE10005B6C98473388276AC1B243F00403E0691A
:10DE20004246B8470834EDE7236A002BEED1F9E704
:10DE300001A800F04DF9012003B0BDE8F083000017
:10DE40007FB56D4685E806000446011D712203A8D2
:10DE50001E4600F01BF921460022C869D3B288B9DA
:10DE6000086A78B995E8030004EBC2021C3201335A
:10DE700082E803000124337003A800F029F920464A
:10DE800004B070BD0132032A01F10801E5D100247C
:10DE9000F2E700002DE9F04F2DED028B8BB0044628
:10DEA0008B465322011D01A8BDF858809FED258B9C
:10DEB00000F0ECF8254604F11809002708F0040AE0
:10DEC000A94536D0EB690BB92B6A63B1BAF1000FE3
:10DED0000BD1236820465B6C98474346C1B25A4633
:10DEE000D5E90706B0470835EAE7002FFBD18DEDED
:10DEF000028BADF810705B4605AA0BF1080C186890
:10DF00005968174603C7083363453A46F7D118687E
:10DF100038609B88BB8009F013FB0423ADF81030F8
:10DF20002368CDE902019B6C02A92046984701278E
:10DF3000D9E701A800F0CCF801200BB0BDEC028BB2
:10DF4000BDE8F08F000000000000000030B503685D
:10DF50000968DD0FB5EBD17F23F0604421F060420A
:10DF60004FEAD1700BD0002BB8BFA40C0029B8BF6A
:10DF7000920C944202D034BF0120002030BD944264
:10DF800005D1C1F38070C3F380738342F6D194420C
:10DF90002CBF00200120F1E7082817D90C280CD944
:10DFA00010280CD914280CD918280CD920280CD9E1
:10DFB00030288CBF0F200E207047092070470A20A0
:10DFC00070470B2070470C2070470D2070470000F1
:10DFD000082817D909280CD00A280CD00B280CD0F7
:10DFE0000C280CD00D280CD00E2814BF4020302057
:10DFF00070470C207047102070471420704718207D
:10E00000704720207047000043681847836818470E
:10E0100010B5024C8260C0E9004110BDD871020801
:10E02000007B00F001007047704700008160828033
:10E0300070470000826838B504465AB1037B13F07C
:10E04000010507D143F0010303739047237B65F378
:10E050000003237338BD000010B5044B1B68044651
:10E06000986A03681B699847204610BD301000204D
:10E0700010B5054B1B680446986A036800211B69AC
:10E080009847204610BD00BF30100020F8B50C4B5B
:10E0900001601E680446B06A03681B6C1746984707
:10E0A000054610B1F36AA3F84270206803689B68C4
:10E0B00098471DB1F36A0022A3F842202046F8BD1C
:10E0C0003010002010B50446FFF7E0FF204610BDD9
:10E0D00010B5044600680368DB689847204610BD09
:10E0E000C181B1FA81F0400970470000C0897047D2
:10E0F0007047000000207047704700007047000024
:10E100000020704700207047704700004FF4B45063
:10E1100070470000002070470020704700207047C3
:10E120000020704700207047007B70477047000058
:10E1300007B503688DF80710DB6801220DF10701B0
:10E14000984703B05DF804FB08B5036801225B6AD9
:10E1500098470028D4BF0020012008BD07B50368F8
:10E160000DF10701DB69984720B19DF8070003B066
:10E170005DF804FB4FF0FF30F9E7000013B50446EB
:10E1800008460191FCF7C2FF23680199DB6802464B
:10E19000204602B0BDE810401847000009F0D0B991
:10E1A00010B444682CB903685DF8044BD3F8803090
:10E1B000184700205DF8044B7047000082681AB9C8
:10E1C0000368D3F8903018470020704782681AB966
:10E1D0000368D3F8943018470020704730B445687E
:10E1E00025B90468E46FA44630BC604730BC704772
:10E1F00000231A46FFF7F2BF436813B18B4200D0E9
:10E2000041B9836813B1934200D01AB9C0E9011231
:10E21000012070470020704710B484680CB19C4204
:10E2200006D103685DF8044BD3F8843092B21847E6
:10E2300000205DF8044B70470023FFF7EDBF00009E
:10E24000013901298CBF0020012070470020704750
:10E2500000207047002070477047000000230B70BB
:10E2600070470000704700007047000000207047B2
:10E2700000207047002070474368C26893423CBF4B
:10E280008268D15443680133436001207047000025
:10E29000F8B505460C468F180026BC4207D02B68FF
:10E2A00014F8011B9B68284698470644F5E730465A
:10E2B000F8BD000000207047002070470020704724
:10E2C0000020704738B590F89C308B4204460D46CC
:10E2D0000CD080F89C1009F031F92368C4F8A00034
:10E2E0005B682046984708B984F84D5038BD000057
:10E2F0007FB50D461446194600267AB1531E0B4AC7
:10E300006846CDE90026089ACDE9025300F08EF860
:10E310000198844204D92E5404B070BD1346EEE730
:10E32000002CF9D02C4404F8016CF5E7FC710208CC
:10E3300008B410B585B007AC54F8043B00940394BE
:10E34000FFF7D6FF05B0BDE8104001B070470000F0
:10E3500070B5044602F002FF5E224FF4000102F0A5
:10E36000E9FE0D4E0D4B1D6833783BB9E86A042277
:10E370002146483009F0E6F801233370EB6A2A227F
:10E3800083F84620EB6A93F89C301BB90448214679
:10E3900009F0A6F870BD00BF262F00203010002025
:10E3A000E071020807B503680DF10701DB699847C2
:10E3B00020B19DF8070003B05DF804FB4FF0FF307B
:10E3C000F9E70000F8B506460F4614460025AC42B2
:10E3D0000AD0336830469B699847431C01D12846D0
:10E3E000F8BD78550135F2E72046F9E70EB403B5DC
:10E3F00003AA036852F8041B5B680192984702B0B5
:10E400005DF804EB03B0704700F010B813B5044694
:10E4100008460191FCF77AFE23680199DB68024601
:10E42000204602B0BDE81040184700002DE9F04F2B
:10E430002DED028B06468DB0904691F80090B9F113
:10E44000000F00F0DE82B9F1250F08D04B1C0393BA
:10E45000336849469B68304698470399EDE791F841
:10E4600001908B1CB9F1250F0393F1D00025AA462A
:10E470002C461F2C3BD8B9F12B0F2DD01CD8B9F14D
:10E48000200F2BD0B9F1230F2ED0A9F13003DBB22E
:10E49000092B36D860064BBF05EB85050AEB8A0AC7
:10E4A00003EB450503EB4A0A4EBF05F0FF050AF0F2
:10E4B000FF0A44F0200407E0B9F12D0F11D0B9F1A3
:10E4C000300FE2D144F00104039B13F8019B039346
:10E4D000B9F1000FCDD126E044F0020444F0040469
:10E4E000F2E744F00804EFE744F01004ECE77F2C77
:10E4F000CBD9230617D5B9F16C0F14D144F480742D
:10E50000E2E7B9F12E0F05D1620600F17A8244F0FC
:10E510004004D9E7B9F16C0F02D144F08004D3E78D
:10E52000B9F1680FD0D0A9F14503022B61D809F1E8
:10E53000200944F010045FFA89F908F1070828F06F
:10E540000708F8E80201FCF709FB14F0400F08BFC8
:10E55000062524F0C004B9F1650F08EE100AA4B234
:10E5600050D144F0400427060DD59FED977AF0EE88
:10E57000C87AF4EEC77AF1EE10FAC2BF4FF63F73D5
:10E58000234043F0400414F0800346D03B2DA946BD
:10E5900028BF4FF03B0909F101095FFA89F9072704
:10E5A0001722002106A8029314F0C8FA4A463946F9
:10E5B00006A8B0EE480A09F0FBFA9DF8183001935E
:10E5C00003F00902012A029B83462FD0A0072FD413
:10E5D00014F0040F0CBF00222022019911F00C0747
:10E5E00058D0002A40F0AB82BAF1030F50D817463A
:10E5F00037E0A9F16503022B00F25B8124F01004DF
:10E60000A4B29AE7B9F1660F02D144F08004AAE7F8
:10E61000002DA8D0013DEDB2A5E70A2D83BF0A2544
:10E6200099462F462F4698BF9946B9E72D22D4E741
:10E630002B22D2E70427AAEB07072107FFB20AD44F
:10E64000336802929B6820213046013F984717F0BB
:10E65000FF07029AF4D122B1336811469B68304615
:10E660009847019B594D13F0080F594B08BF1D46A1
:10E67000013D04F0100415F8011F002900F0B580D9
:10E680000CB12039C9B2336830469B689847F2E72D
:10E690000327D0E7CDF808B0002B36D0019BD94432
:10E6A000DB065FFA89F907D59DF81930312B04BFD5
:10E6B00009F1FF395FFA89F94FFA89F3002B44DD3C
:10E6C000B9F1080F28BF4FF0080914F08003049334
:10E6D0001ABF2BEAEB730133052302B101330DB1ED
:10E6E000691C0B449A45C4BFAAEB0303DFB214F0C4
:10E6F000090F2FD177B3336805929B6820213046EC
:10E70000013F9847FFB2059AF4E76006DDD45D4506
:10E7100004DB1BF1040FA8BF44F080046B1C06A9A6
:10E720000B4435B113F80119302902D1013DEDB286
:10E73000F7E72106C9D505F101095D455FFA89F9B9
:10E7400006DDA5EB0B05EDB2BFE74FF00109BCE715
:10E750000025BAE722B1336811469B6830469847D6
:10E76000220708D43FB1336830219B683046013F0F
:10E770009847FFB2F6E7049B002B47D02BEAEB74D7
:10E78000ABEB040A06AB9A44ABEB09096D42A34517
:10E7900017DBA14515DA9AF80110013CA54219DCF6
:10E7A000002900F0D281336830469B689847631C8B
:10E7B00004D133682E219B68304698470AF1010A3C
:10E7C000E5E73021E9E700BF7F96184B2C7202087D
:10E7D00028720208A34507D19DF81930352B0FD8B0
:10E7E00002D1019BDD060BD559B9002F3FF435AEA0
:10E7F000336820219B683046013F9847FFB2F4E719
:10E80000312133689B6830469847EEE79DF8191030
:10E8100031291EBF019B03F0EF030193336830469B
:10E820009B689847E5B9336814F0100F14BF452171
:10E8300065219B6830469847BBF1000F29DACBF180
:10E84000000302932D21336830469B68984730219E
:10E85000029B092B23DD01310A3BC9B20293F7E782
:10E8600033682E219B68304698470235EDB24FF051
:10E8700002094B460CAA1A44336812F8181C9B680C
:10E8800009F101095FFA89F930469847A945F0D1A5
:10E89000C9E702D1019BDC06D1D42B21D3E7336831
:10E8A00030469B6898470299336830319B68C9B2FB
:10E8B000A9E7B9F1630F37D0B9F1730F4FD0B9F1B0
:10E8C000640F63D124F0900714F4807FBFB20DF180
:10E8D00018097BD008F1070222F007029046516820
:10E8E00058F8080B002904DA404261EB410147F077
:10E8F00080070A234A4600F07BF9A0EB0900C4B266
:10E900007B0640F19F8027F00109AC421FFA89F98C
:10E9100080F0D28007F01403102B03D127F01107E9
:10E920001FFA87F9AB468FE058F8043B8DF8183092
:10E9300001250DF11809200701D4AA451CD84D4422
:10E940005746A9453FF451AF336819F8011B9B683E
:10E9500030469847002FF4D0013FFFB2F1E758F856
:10E96000049B14F0400F14BF29464FF0FF31484676
:10E9700014F0D0FD0546DEE7336820219B68304661
:10E980000AF1FF3A98475FFA8AFAD6E7B9F1690FB8
:10E9900098D0B9F1750F27D124F01004A7B20A233B
:10E9A00017F4807FDBB20DF1180944D008F1070895
:10E9B00028F00708F8E802014A4600F019F9A0EB30
:10E9C000090027F08007C4B2BFB299E758F8040BDA
:10E9D0000028B8BF40424FF00A024946B8BF47F08E
:10E9E000800700F0B7F888E724F00607B9F1700F48
:10E9F000BFB214D00AD8B9F1580F13D0B9F16F0FC4
:10EA000017D00DB0BDEC028BBDE8F08FB9F1780FD7
:10EA1000F7D1F90601D547F004071023C0E747F006
:10EA20001007F6E7E20601D547F006074FF4047336
:10EA3000B6E70823B4E758F8040B1A46494600F035
:10EA400089F8BCE7A346B94619F0100F41D00CABCA
:10EA5000234413F8193C302B30D129F016091FFA42
:10EA600089F919F0080744D119F0010F35D0DA45BA
:10EA700045D904EB0A05A5EB0B05EDB2336819F097
:10EA8000100F9B683FD030213046984719F0040F93
:10EA900008D0336819F0020F9B6814BF5821782101
:10EAA000304698473368AC429B6839D230213046B3
:10EAB000013D9847EDB2F5E7A346C5E719F0040F0D
:10EAC00002D10BF1010B01E00BF1020B5FFA8BFBA2
:10EAD000C7E719F0860FC4D0F3E73368DA459B68BF
:10EAE0000FD9202130460BF1010B98475FFA8BFBC1
:10EAF000F3E7DA4505D9AAEB0B07FFB2BEE72546D7
:10EB0000BCE70027BAE719F0860FCBD019F0020F47
:10EB100014BF2B21202119F0800F18BF2D21BFE732
:10EB2000651E06AB53FA85F5336815F801199B6825
:10EB3000013CE4B230469847002CF5D155E6BAF1D5
:10EB4000040F3FF677AD002786E5A3457FF44DAE71
:10EB500042E600BF082A30B505D10346C008FCD103
:10EB600030330B700DE0102A0DD100F00F0202F1CE
:10EB70003003392B88BF02F13703000901F8013B4C
:10EB8000F3D1084630BD03460022DCB223F0010376
:10EB9000023342F10002580840EAC270C31842EB47
:10EBA0005202180940EA0270C01842EB1212030A1E
:10EBB00043EA0263181842EB1222030C43EA0243B1
:10EBC0001B1842EB1242D31842F100001B0943EA22
:10EBD0000073C3EB4315C3EB85053034020904EB26
:10EBE000450453EA101001F8014BCED1C9E70000EB
:10EBF000082B30B50AD10346C00840EA4170C90865
:10EC000050EA0104F7D13033137013E0102B13D105
:10EC100000F00F0404F13003392B4FEA101088BFC5
:10EC200004F1370340EA0170090902F8013B50EA98
:10EC30000103EDD1104630BD20F00104023441F152
:10EC40000003610841EAC3710C1943EB5303210926
:10EC500041EA03710C1943EB1313210A41EA0361E2
:10EC60000C1943EB1323210C41EA0341091943EB2F
:10EC70001343591843F10003C5B2080940EA037071
:10EC8000C0EB4014C0EB84043035190905EB440592
:10EC900050EA131302F8015BCED1CBE770EE600AA5
:10ECA000DFED057AF0EEE00AF4EEE70AF1EE10FA95
:10ECB0004CBF0120002070470000003410B5B4EEB6
:10ECC000400AF1EE10FA2DED028B0446B0EE608A98
:10ECD000F0EE418A0FD702F041FAA2B24FF4806100
:10ECE00002F028FA38EE288AB6EE000A28EE000A6A
:10ECF000BDEC028B10BDB4EEE00AF1EE10FA07D4C1
:10ED0000B4EE410AF1EE10FAC8BFB0EE410AEFE7E7
:10ED1000B0EE600AECE70000884203DB9042014657
:10ED2000A8BF114608467047884203D39042014667
:10ED300028BF114608467047884203DB90420146CF
:10ED4000A8BF114608467047094A136849F269008E
:10ED500099B21B0C00FB01331360064B186844F298
:10ED6000506182B2000C01FB0200186080B2704753
:10ED7000080E0020040E00207047000038B505681A
:10ED800004462DB1284608F097FD2846FEF7F2FF0D
:10ED9000204638BD13460246014801F0CDBF00BFF2
:10EDA0007A2F002013B50422054B01930446014637
:10EDB0000DEB0200FFF7EEFF024B1C8002B010BD0E
:10EDC000FFFF3F006C2F002007B5502304228DF871
:10EDD0000430412300210DEB02008DF8053006239D
:10EDE0008DF806308DF80710FFF7D4FF0420FFF7E9
:10EDF000D9FF03B05DF804FB00EB0212907B20B951
:10EE00001BB19289120758BF3F20984008447047B1
:10EE1000430608D4000A08D0054B1B88184214BFCB
:10EE2000012000207047002070470120704700BF7C
:10EE3000702F002010B50B4B1A880B4B01301B684C
:10EE400080B2142404FB0033824207D9DC898C424F
:10EE500003F1140304D0013080B2F5E7002010BDA7
:10EE60000120FCE77E2F0020802F0020828983680C
:10EE7000D20648BF1B681846704700008289836825
:10EE8000D20648BF1B6818467047000007B5042328
:10EE900000220DEB03010B48019201F02DFF9DF8BC
:10EEA0000430502B07D19DF80530412B03D19DF83C
:10EEB0000630062B01D0FFF787FF012003B05DF875
:10EEC00004FB00BF7A2F002082894368920705D592
:10EED0001B68181E18BF01200B6070470120FBE75C
:10EEE00037B58B891446DA070D4605D523684A687D
:10EEF00013442360012012E09B07FBD50A4B1B68DB
:10EF0000142201A902FB0030FFF7DEFF48B101998E
:10EF100022686B680A44D3581BB15B1A236003B0A4
:10EF200030BD0020FBE700BF802F00202DE9F04F0F
:10EF30008BB01F469DF854800691142353430593CC
:10EF400008F10603DBB2054616464FF0000B0793A7
:10EF50005FFA8BFA07EB0A1999F80F40002C4CD096
:10EF6000062C28D1B8F10B0F21D84846FFF77EFFB9
:10EF70000446C8B1169B099309AA49463046FFF7D3
:10EF8000AFFF88B11499434652463846FFF734FF25
:10EF9000099B0293079B0699CDE90003324623465D
:10EFA0002846FFF7C3FF18B90BF1010BD0E700208B
:10EFB0000BB0BDE8F08F1499434652463846FFF730
:10EFC0001BFFB0EB953FEFD1C5F30423A342EBD178
:10EFD0000B4C059B206809A91844FFF775FF002812
:10EFE000E2D0D9F80430099A1344169A1344069AC9
:10EFF00013602068059B1844DAE72046D8E700BF75
:10F00000802F00202DE9F04F1F4B5FFA80F8B3F8F6
:10F0100000A0C0F3403348EA03281C4B1E680F468B
:10F0200087B00546C0F3042B00211FFA81F9CA45B9
:10F0300027D9F3894345344620D1337C062B0FD1A1
:10F040003046FFF71BFFC8B10023CDE90133009321
:10F050004A46034639462846FFF768FF044609E05A
:10F060009B450BD105A93046FFF72EFF0028F5D0B0
:10F07000059B3B60204607B0BDE8F08F0131143698
:10F08000D3E70024F6E700BF7E2F0020802F00206A
:10F090002DE9F04F98468DB0142353430693484B07
:10F0A0009DF85890DDF868B004461868069B0E4637
:10F0B00018440AA91746FFF707FF00287DD0002350
:10F0C000079309F10603DBB209939DF81CA006EB38
:10F0D0000A15EB7B002B70D0062B3BD12846FFF79F
:10F0E000C5FE0890002831D0B9F10B0F65D8179BE9
:10F0F0000B930BAA29463846FFF7F2FE30B39BF874
:10F100000030012B59D85A1C0BEB83038BF80020DD
:10F1100041465D6052464B463046FFF76DFE1B9AF6
:10F120000899CDE904B2199A0392189A02920B9A9F
:10F130000192099A009203463A462046FFF7A8FF3B
:10F1400000BB9BF80030013B8BF80030079B01337C
:10F150000793BAE7179A686810440A9A1044A042C5
:10F1600013D14B46524641463046FFF745FE189BA9
:10F170001B9A1860199B1D6000231370104B1868B0
:10F18000069B18440DB0BDE8F08F052BDED1031DA2
:10F190009C4203D000F108039C42D7D11B9B201A4C
:10F1A0008008187052464B4641463046FFF724FE11
:10F1B000189B1860199B1D60E0E70020E2E700BF84
:10F1C000802F00202DE9F04F8BB00025DFF8A4A0A0
:10F1D000079306460F4690461560254B1B881FFA7D
:10F1E00085FB5B4541D9DAF80000142303FB0B04CF
:10F1F00009A9204694F81090FFF766FE98B3B9F17C
:10F20000060F17D12046FFF739FE014658B3149B6D
:10F210000593079B0297CDE903830023CDE90033D3
:10F220005A463046FFF734FF0446E0B120460BB0A3
:10F23000BDE8F08F0998B04204D1149A00233B60D6
:10F240001370F3E7B9F1050F0DD1031D9E4203D0F2
:10F2500000F108039E4206D1149B301A80081870F2
:10F2600000233B60E2E70135B7E70024DEE700BF9B
:10F270007E2F0020802F00202DE9F04798460D8832
:10F28000234B0446C5F30809186809EB890588B0C3
:10F2900000EB850507A92846119E95F810A0174692
:10F2A000FFF712FE20B90025284608B0BDE8F08718
:10F2B0000021BAF1060FC8F8001013D12846FFF755
:10F2C000DDFD0028EFD0109B0091CDE90383CDE94F
:10F2D00001170B46059601464A462046FFF7D8FE21
:10F2E0000546E1E70798A04202D139603170DBE7BB
:10F2F000BAF1050FD7D1031D9C4203D000F10803DA
:10F300009C42D0D1241AA408002334703B60CBE780
:10F31000802F00200138C0B204289ABF014B185C2E
:10F3200000207047107302082DE9F04F2DED028B7D
:10F3300083B000240093931DDBB208EE103A05461B
:10F340000E461746A246A0464FF0010BE0B201015F
:10F3500005EB001090F80F90B9F1000F5AD0837BA5
:10F360003F2B02D92E4808F0BBF817B1002B08BF7D
:10F370003F23C3F1200EA3F1200C2AFA03F208FA6E
:10F380000EFE28FA0CFC42EA0E0242EA0C0212F0CF
:10F39000010FC3F1200CA3F12002E3D10BFA02F21A
:10F3A0002BFA0CFC42EA0C020BFA03F3B9F1060F3C
:10F3B00043EA0A0A42EA080813D10B2FD2D8FFF712
:10F3C00055FD814658B16858FBF7A0FE009B1844D4
:10F3D000C3B218EE102A31464846FFF7A5FF0134A4
:10F3E000B4E74846FFF796FF01900028BAD0685866
:10F3F000FBF78CFE009B1844C0B2B9F1050F04BFA7
:10F400000230C0B21028019BACD8308804300344CD
:10F410003380E4E703B0BDEC028BBDE8F08F00BFA2
:10F42000307202082DE9F04F85B00423DFF8989080
:10F43000ADF80E3000244FF0140A214B1B881FFA40
:10F4400084F8434539D9D9F800300AFB08F15D1832
:10F450002F7CB5F80EB0062F23D1B8F1000F02D1E2
:10F46000184808F03DF828460193FFF707FD0646C7
:10F47000A8B1019B5858FBF749FE0022C3B20DF119
:10F480000E013046FFF750FF59464046FFF7D2FCC9
:10F490000028E5D1062F02D0AB899B07E0D40134C8
:10F4A000CBE73846FFF736FF0028D9D0BDF80E303D
:10F4B00004331844ADF80E00E6E705B0BDE8F08F60
:10F4C0007E2F002030720208802F0020437803F046
:10F4D0001F021F2A0FD00278C3F3401342EA03230E
:10F4E00040F2FF12934206D000680138C31C94BF5B
:10F4F0000020012070470120704700002DE9F341F2
:10F50000224FDFF8908006460D4604247B88A342F4
:10F5100037D904230DEB03012246384601F0ECFBFA
:10F520009DF80510737881EA0302D20618D196F887
:10F5300000C09DF80400C3F34013C1F340124CEA2D
:10F54000032340EA022293420AD13268019B5340CE
:10F5500013EA080F04D12C80012002B0BDE8F0812D
:10F5600001A8FFF7B3FF20B1094B2C801C800020BD
:10F57000F3E701F01F00FFF7CDFE031D1C44A4B20A
:10F58000C4E74FF6FF732B80F1E700BF7A2F00200E
:10F590006C2F002000C0FFFF70B50C4620461146BE
:10F5A00015461E4613F0B6FF831CAB420AD85F22F5
:10F5B000225422180330A84206F1580656709CBF08
:10F5C0000022E25470BD00002DE9F74FDDE90D5433
:10F5D00007468A46164609689DF830809B462246B3
:10F5E0009DF83C300093284613F080FF4FF000094F
:10F5F0009BF800105FFA89F29142019212D92146DC
:10F60000284613F087FFC0B28442019A07D90BEB5A
:10F6100082025168221A0968284413F067FF09F131
:10F620000109E5E7E6B12146284613F073FFC3B2AE
:10F630009C4204D93168E21AE81813F057FF009B86
:10F6400013B9B8F1000F13D0F37B052B10D143464B
:10F6500022462946384603B0BDE8F04FFFF79CBF6D
:10F66000009B13B9B8F1000F02D09AF81030ECE704
:10F6700003B0BDE8F08F0000F0B58BB007AC1F46BB
:10F680000023C4E9013307930DF11303CDE90043CF
:10F69000154606AB05AA0646FFF7EEFD014610B972
:10F6A00028700BB0F0BD9DF84030069A0195CDE969
:10F6B00002739DF81330009330462346FFF784FF12
:10F6C000EFE700002DE9F04F984689B014234B4333
:10F6D000DFF828A1039204460E4604934FF0000978
:10F6E0005FFA89F52B0108EB0515059395F80FB026
:10F6F000BBF1000F7FD0BBF1060F58F803702AD181
:10F700003846FBF703FD39460246204613F0B8FEA3
:10F71000002869D12846FFF7A9FB0746002863D0D7
:10F72000039B079307AA29463046FFF7D9FB002819
:10F730005AD0059B58F80300FBF7E8FC129B009396
:10F74000079A3B4631462044FFF7BCFF00284BD0C8
:10F7500009B0BDE8F08F3946204613F061FE88B944
:10F76000DAF80000049B07A91844FFF7ADFB002856
:10F770003AD0129B83F800B06868079B1844039B3B
:10F780001844E5E7BBF1050F2ED11021384613F0E0
:10F79000C1FE5FFA80FB5A463946204613F092FEBE
:10F7A00010BB14F90B305F2B1ED10BF1010B14F8B9
:10F7B0000B30583B022B17D8DAF80000049B07A93E
:10F7C0001844FFF781FB78B16868079B129A1844C8
:10F7D000039B18440423137014F90B30592B06D0E3
:10F7E0005A2B06D0582BB3D009F1010978E7043021
:10F7F000AEE70830ACE75846AAE700BF802F0020EC
:10F800002DE9F04F8BB0DFF8C8B0029104461746DF
:10F8100000252E4B1B881FFA85FA534552D9142216
:10F8200053465343DBF8002002EB0309D35899F801
:10F830001080B8F1060F33D110211846039313F04E
:10F8400069FE039B5FFA80F842461946204613F092
:10F8500039FE0646002833D14846FFF70FFB034622
:10F8600070B3029A009204EB080032465146FFF74B
:10F8700029FF804620B37FB10DF11303009306AA40
:10F8800007AB05A9CDE9076605960996FFF79AFC2F
:10F89000069B0BB19B893B8040460BB0BDE8F08FC7
:10F8A0001946204613F0BCFD50B9029B07A983F806
:10F8B00000804846FFF708FB20B1DDF81C80EBE72D
:10F8C0000135A6E74FF00008E6E700BF7E2F0020D5
:10F8D000802F002010B590B00023CDE908330693A7
:10F8E0000A930DF11703009306A908AB07AA044673
:10F8F000FFF768FC014668B111230122CDE902320D
:10F900000BAB01939DF817300093079A08AB204684
:10F91000FFF75AFE10B010BDF0B5304D87B040F281
:10F92000A51202908DF80C1006460C4601A8291D60
:10F93000FEF7ACFB052204A9286808F011F9074678
:10F9400001A8FEF7C5FB052F06D1049BB34203D1E6
:10F950009DF81430A3423ED0214E224F4FF4B07296
:10F96000314601A8FEF792FB286808F00FF804283A
:10F9700021D92868052202A908F08CF8431F5C42AF
:10F980005C4101A8FEF7A4FB2CBB3C68E36A93F83A
:10F990009C3093B9A06A036801211B699847A06A4B
:10F9A00003684FF4FA719B689847A06A03680021C6
:10F9B0001B699847D2E70024E3E7A06A03681B6C41
:10F9C00098470028E6D001F0C9FB40F2FA424FF414
:10F9D000801101F0AFFB07B0F0BD00BF442F002045
:10F9E000482F0020301000202DE9F341154E164F0E
:10F9F000C92406F10408013CA4B2FCB140F24B1248
:10FA0000414601A8FEF742FB306807F0A5FF054616
:10FA100001A8FEF75DFB042D10D93D68A86A0368B4
:10FA20000A211B699847A86A03680A215B689847FE
:10FA3000A86A036800211B699847DCE702B0BDE8AB
:10FA4000F08100BF442F00203010002000B58BB0A3
:10FA50000023CDE90733049309930DF10D030093BF
:10FA600005AA07AB04A9FFF7ADFB10B3059B23B3B1
:10FA7000DB7BC2898DF8182003F01F03C2F300223C
:10FA80001B0243EA4233049A43EA82339DF818206A
:10FA90000DF10E01134306A80693FFF72FFD40B1A9
:10FAA0009DF8193003F01F03052B03D09DF80D308E
:10FAB00003B100200BB05DF804FB037CD9E7000024
:10FAC000F0B5144F3B8889B006460D46FBB10DF1E9
:10FAD0000B030024009304AA05AB03A9CDE9054458
:10FAE00003940794FFF76EFB88B10B4B38881B68B3
:10FAF000A2B290420BD91A46013411688E4203F12A
:10FB00000C03F5D1137A2B70012009B0F0BD002051
:10FB1000FBE700BF742F0020682F002013B50DF104
:10FB200007010446FFF7CCFF10B92046FFF78EFF10
:10FB300002B010BD07B5074B1B884BB10DF1070193
:10FB4000FFF7BEFF08B19DF8070003B05DF804FBA6
:10FB50001846FAE7642F002010B50C46FFF7EAFFBD
:10FB600040B9A30608D5054B1B6813B1186AC0F34A
:10FB7000800010BD0020FCE70120FAE7E4460020E9
:10FB80000138032816D8DFE800F002080E13FDEE56
:10FB9000C07A17EE903A0B707047BDEEC00A10EEB7
:10FBA000103A0B807047BDEEC00A81ED000A704725
:10FBB00081ED000A7047000037B5036803F0004389
:10FBC00003600A4B1B880C4613B9002003B030BDFC
:10FBD000074D01A92868FFF777F90028F5D014B17F
:10FBE0002B681B7C23700198F0E700BF7E2F00205C
:10FBF000802F00202DE9F04F8FB09B469DF870308C
:10FC00000B93142343439DF860901A9D0A93074673
:10FC100088460892002307939DF81CA008EB0A165B
:10FC2000F47B002C00F0BC80B089FFF7F1F80028CD
:10FC300000F0B380062C2FD13046FFF717F90446A9
:10FC4000002800F0AA80199B0D930DAA3146384672
:10FC5000FFF746F9002800F0A0804B46524659466F
:10FC60004046FFF7C9F81D9A05920B9A04921B9A19
:10FC7000CDE902520D9A019209F10602D2B2034671
:10FC800000922146089A3846FFF7B4FF002800F09A
:10FC900084800FB0BDE8F08F089B1B780993002B80
:10FCA0003CD02B8867F308032B8052464B465946BD
:10FCB0004046FFF7A1F83B4B03EA40302B6823F0A6
:10FCC000FF4323F4FF0323F4FC4318431B9B2860EA
:10FCD00003B11C70344B18680A9B0DA91844FFF738
:10FCE000F3F8002859D00D9A73681344199A98189C
:10FCF0000B9A002ACDD02D4A1278002AC9D0F27B67
:10FD0000012AC6D1B2895207C3D5199A9B56002B36
:10FD1000BFD1EB7843F08003EB70BAE74B46524615
:10FD200059464046FFF768F82B68C3F351339842B1
:10FD300033D1089A0123137095F90330002B06DAAA
:10FD4000EB78099A62F3C713EB701046A1E7052C14
:10FD500023D16B78C3F34302022A1ED8013262F327
:10FD600044036B701B9B13B11B9A042313700E4B3F
:10FD700018680A9B0DA91844FFF7A6F868B17068C7
:10FD80000D9C95F801B0199B2044CBF3430B18440C
:10FD90000BF1FF3B00EB8B007BE7079B01333AE75E
:10FDA000204676E700E0FF7F802F00200C0E002029
:10FDB0002DE9F04F8BB0DFF8EC9004880792002219
:10FDC0008DF82720B9F800201F46C4F308039A4293
:10FDD00005460E461C4662D9DFF8CC801BB2D8F827
:10FDE000001003EB83039A0001EB83031B7C052BBC
:10FDF00018D14378C3F34301022915D8013161F3C7
:10FE0000440343700EB104233370D8F800106878AF
:10FE10000A44C0F34300431E506800EB83000BB05C
:10FE2000BDE8F08F062B04D001340123A4B28DF875
:10FE300027304FF0140B4FF0000AB9F80030A342FE
:10FE40002DD9D8F800200BFB04229089FEF7E0FFA3
:10FE5000B8B1117C062917D11046FFF70FF80146FB
:10FE600078B1079B0597CDE90363CDE901A5CDF8EE
:10FE700000A000230DF127022046FFF7BBFE00285B
:10FE8000CDD10134A4B2D8E72B68C4F3080403F041
:10FE9000004323432B6006B131705068BFE7002058
:10FEA000BDE700BF7E2F0020802F002073B50546E0
:10FEB0000C461646334601220DF107012846FFF78E
:10FEC00077FF28B19DF80730042BF3D804B12370D5
:10FED00002B070BDF8B514460746002220460E4613
:10FEE000FFF76AFE002540B1BD4206D00022314630
:10FEF0002046FFF7DBFF0135F5E7F8BD013903299F
:10FF00000BD8DFE801F00204060800F079BE00F02B
:10FF1000B3BE00F0D1BE00F03BBE9FED010A7047BA
:10FF20000000C07FB4EE400AF1EE10FA10B50446AE
:10FF30000CD69FED327AF0EEC07AF4EE477AF1EE0D
:10FF400010FA03DC042902D180ED000A10BD032958
:10FF500019D1B5EEC00A9FED2A7ADFED2A7A9FED1E
:10FF60002A1ADFED2A0AF1EE10FA58BFF0EE477AAE
:10FF700030EE270A40F6C900FEF7A0FEBDEEC00A2B
:10FF800084ED000AE2E702291AD1B5EEC00A9FED1E
:10FF90001C7ADFED1C7A9FED1E1ADFED1E0AF1EED2
:10FFA00010FA58BFF0EE477A30EE270A40F6CE003E
:10FFB000FEF784FEBDEEC00A10EE103A2380C5E7BE
:10FFC0000129C3D1B5EEC00A9FED0D7ADFED0D7AA0
:10FFD0009FED111ADFED110AF1EE10FA58BFF0EEA5
:10FFE000477A30EE270A40F6D300FEF767FEFDEEB3
:10FFF000C07A17EE903A2370A8E700BFFFFF7F7F1B
:020000040801F1
:100000000AD7233C0AD723BC0000004F000000CFD2
:1000100000FEFF46000000C70000FE42000000C3D3
:100020002DE9F3411D4690F90030232B0F469046F1
:100030004FF000042CD01749019401AA14F01CF9C8
:10004000064618B9002002B0BDE8F081FBF75EF863
:100050001028F7D80F4901AA204614F00DF90028FE
:10006000F0D0214614F084F80A4988ED000A01AA6C
:100070003E60204614F000F930B10749FBF73CF828
:1000800010B901202870DEE700232B700120DAE789
:100090002046D8E7447202084B72020830B5044685
:1000A0009DB00D4603F04EFB01232146002203F0D4
:1000B000D7FA431C044624D003F044FB23466322B2
:1000C00003A903F005FBA0B10DF1020302AA01A9E7
:1000D00003A8FFF7A5FF0028EED0019800220DF13C
:1000E0000301FFF78DFB0028E6D02B8801332B801E
:1000F000E2E703F027FB214603F0DCFA01201DB004
:1001000030BD0020FBE700002DE9F0479EB015460A
:10011000019003F017FB01230199002203F0A0FADC
:10012000431C064602D1334807F0DAF9DFF8CCA0C9
:10013000DFF8CC80DFF8CC90012703F003FB3346D7
:10014000632205A903F0C4FAF0B10DF10A0304AA71
:1001500003A905A8FFF764FF0028EED0039800224A
:100160000DF10B01FFF74CFB044600283FD02A8815
:10017000BAF80030934212D800F0F0FF40F64C126B
:100180004FF4801100F0D6FF03F0DCFA314603F0A3
:1001900091FA194B01201F701EB0BDE8F0870C20AA
:1001A000D8F8001042438C502A88D8F800300499BF
:1001B00000FB0232516029889DF80A2000FB0133C0
:1001C0001A7222B1B9F800300133A9F800302B8837
:1001D00001332B802046FFF739FC0028ADD19DF874
:1001E0000B109DED040A2046FFF79CFEA5E707468D
:1001F000A3E700BF58720208782F0020762F002056
:10020000682F0020642F00202DE9F7430D46064695
:1002100000286DD011F088FD074610B9354807F069
:100220005FF900233449ADF8003001AA019314F0BE
:1002300023F8DFF8C48088B16946FFF72FFF044632
:1002400030B9384611F048FD204603B0BDE8F083D0
:1002500001AA4146002014F00FF8ECE7DFF8A8905F
:10026000384611F039FDD9F8000008B1FDF786FDD8
:10027000224BDFF89880224F00241C80BDF800300C
:10028000A8F800400C2058433C80FDF771FDC9F8E8
:10029000000008B91B48C2E7BDF80030A8F80030DC
:1002A00023B33046019411F03FFD06460028B5D037
:1002B0001149ADF8024001AA13F0DEFFDFF83880E3
:1002C00070B10DF102022946FFF71EFF044608B97E
:1002D0003046B7E701AA4146002013F0CDFFEFE713
:1002E000304611F0F9FCBDF800303B800124ABE74B
:1002F0000446A9E784720208B0720208642F002045
:10030000742F0020B2720208682F0020762F002080
:1003100010B50446FFF778FF28B921460248BDE82A
:10032000104006F01FBB10BDDC7202082DE9F0433F
:100330004FF000089DB005460E461746A2F8008013
:10034000002E35DDB2B200239CB2A24203F10109B6
:1003500002D9EB5C0A2B29D1632C28BF63242246E7
:10036000294603A812F0C2FB1CAB1C44A6EB0906ED
:1003700004F8648C9DF90C30232B4D44E0D0002B05
:10038000DED00DF1020302AA01A903A8FFF748FE7F
:100390000028D5D0019800220DF10301FFF730FAB3
:1003A0000028CDD03B8801333B80C9E74B46CBE7E3
:1003B00001201DB0BDE8F0832DE9F04FDFF8288162
:1003C0000546D8F800009FB00E4608B1FDF7D6FCF0
:1003D000434FDFF818A1DFF8189100240DF10A024D
:1003E00031462846C8F800403C80AAF80040A9F8E9
:1003F0000040ADF80A40FFF799FF00286DD0BDF826
:100400000A300C205843FDF7B3FCC8F8000010B9BF
:10041000344807F065F8BDF80A303B80A346BDF8C4
:100420000A30A34257D9002E55DDB1B2002297B24F
:10043000B94202F1010302D9AA5C0A2A49D1632F09
:1004400028BF63273A46294605A8019312F04EFBC0
:100450001EAB1F44019B07F864BCF61A1D449DF9AE
:100460001430232BDBD0002BD9D002AB04AA03A974
:1004700005A8FFF7D5FD0028D1D0039800220DF183
:100480000901FFF7BDF907460028C8D00C2303FB7C
:1004900004F2D8F800309850D8F800301344049A89
:1004A0005A609DF808201A7222B1B9F80030013361
:1004B000A9F8003001343846A4B2FFF7C7FA002883
:1004C000ADD19DF809109DED040A3846FFF72AFDCD
:1004D000A5E71A46ABE7AAF800301FB0BDE8F08FD9
:1004E000762F0020B2720208682F0020742F00209F
:1004F000642F002002460248418A1430FFF75CBF97
:100500001873020810B50A4B1B680446D86A0368C2
:100510005B69984710B12146FFF7FAFE054B5B8AED
:1005200023B12046BDE81040FFF7E4BF10BD00BF77
:10053000301000201873020830B5002085B0FFF796
:10054000E1FF214B1A7872B901221A701F4B204A21
:100550001B680292986A1F4A0368039204AA12E970
:1005600006009B6A98471C4D04246B88A34229D936
:10057000042322466946284600F0BEFB6846FEF783
:10058000A5FF18B1154B1C8005B030BD009801A91E
:10059000FEF738FD60B19DF8010000F01F00FEF786
:1005A000B9FE221D0346019992B2284600F0A4FB31
:1005B0009DF8010000F01F00FEF7ACFE043004447B
:1005C000A4B2D2E70020DFE7792F0020301000200E
:1005D000272F0020010B01087A2F00206C2F00200C
:1005E00070B50E4B1E880E4B1B68002294B2A642BB
:1005F00009D91C4601322568854203F10C03F5D167
:1006000094ED010A70BD8B891B0649BF8B6891ED83
:10061000020AC01A90ED000AF4E700BF742F002010
:10062000682F00202DE9F04105460F464FF00008E5
:100630005FFA88F307EB0311CC7BDCB1042C0BD8F9
:100640004E682E443046FFF7CBFF31462046FFF779
:1006500097FA08F10108EBE7052CFAD14C682C4415
:100660002046FFF7BDFF84ED000A84ED010A84ED0A
:10067000020AEEE7BDE8F08170B50E4B1E880E4B06
:100680001B68002294B2A64209D91C460132256893
:10069000854203F10C03F5D194ED010A70BD8B89FD
:1006A0001B0649BF8B6891ED020AC01A90ED000A43
:1006B000F4E700BF742F0020682F00202DE9F041DF
:1006C0008AB00023CDE90733039309930DF10903A1
:1006D000009304AA07AB03A90446FEF773FD054681
:1006E00020B9002630460AB0BDE8F081049B002BFB
:1006F0003AD0DB7BEA898DF8142003F01F03C2F3A4
:1007000000221B0243EA4233039A43EA82339DF8F4
:1007100014200DF10A01134305A80593FEF7EEFE20
:10072000064658BB06A92846FEF7CEFB0028D9D0BE
:100730009DF815700499DDF8188007F01F07B9B10E
:100740009DF81C3093B1089A012B556802D0099B83
:100750005B681D442046FFF743FF49684144294434
:100760003846FFF70DFABDE7037CC3E73546F1E7EE
:1007700029462046FFF780FF4146F1E79DF8150026
:100780009DF8093000F01F02052A0FD0002BA8D1D8
:1007900000F01F00FEF7BEFDBDF80A20043203463C
:1007A00092B22146044800F0A7FA9BE7002BEFD055
:1007B000A4EB8304ECE700BF7A2F00202DE9F0437F
:1007C00085B0FEF763FB134E134F00254FF014085E
:1007D0003288ABB29A4219D91C463B6808FB0434F4
:1007E00094F81090B9F1040F0ED803A92046FEF733
:1007F0006BFB48B1039801902146FFF73DFF01983C
:1008000001464846FFF7BCF90135E1E705B0BDE810
:10081000F08300BF7E2F0020802F00202DE9F347BA
:10082000DFF88C901F4940F678226846FDF72EFCD1
:10083000B9F800702FB11C4B1A881C4B1B889A42C8
:1008400028D0194E194D05244FF00008B9F8007052
:100850001FB132882B889A421CD0013C14F0FF044F
:1008600018D00022114601A83788CDF80480FFF780
:10087000A3F94FF0000A1FFA8AF30AF1010A28B11E
:100880000022114601A8FFF711FBF4E7A9F8003098
:100890002F80DBE76846FDF71BFC384602B0BDE859
:1008A000F08700BF282F0020622F0020722F002029
:1008B0006E2F0020024A138801331380704700BF57
:1008C000622F00202DE9F0412DED028B90B0002326
:1008D000CDE9083305930A930DF1110300930E46F9
:1008E00008AB06AA05A90446FEF76CFC0546D8B17C
:1008F0000699F1B1CA7BEB898DF81C3002F01F021A
:10090000C3F300201302059A9DF8117043EA4033A7
:1009100043EA82339DF81C201A43C3F30423052BBA
:10092000079200F0868037B110B0BDEC028BBDE8B5
:10093000F081027CDFE7012B05D121B18B895B07B8
:1009400001D5FFF7B7FF274677E0BDF812204FF635
:10095000FF739A420AD14C4B83F800804B4B4C49B1
:100960001B68986903681B689847DDE79DF81D10B0
:1009700001F01F01042925D99DF81D00BDF81220A2
:10098000444900F01F00FEF7C5FC498813180833DE
:100990008B424AD20432104480B2FEF703FA9DF82B
:1009A0001D0000F01F00FEF7B5FCBDF81210043169
:1009B000024689B23846FEF7EDF9BDF8121004225E
:1009C00007A85EE02046FFF799FA0699F0EE408A04
:1009D00071B12046FFF704FEB0EE408AF0EE400A07
:1009E000B0EE680AFEF75AF938B1002EC4D19BE781
:1009F00029462046FFF740FEEEE7002EBCD19DF8C9
:100A00001D3003F01F03032BB6D09FED230A38EEF1
:100A1000C88AF0EEE88A68EE808AB0EEC88AB4EE42
:100A2000E88AF1EE10FAA7D57EE7174B01221A707B
:100A300094E7002F87D0A4EB870711234FF001081C
:100A4000CDE902380BAB01939DF811300093294694
:100A50002046069A08ABFEF7B7FD0DF1120107A874
:100A6000FEF74CFD00283FF470AF9DF81D0000F02C
:100A70001F00FEF74FFCBDF812100431024689B288
:100A80003846FEF787F94FE7602F0020301000202E
:100A9000007302087A2F002017B7D1387FB5164DA2
:100AA0002E1D40F27F12314601A8FDF7EFFA2868AB
:100AB00006F052FF042812D92868052202A907F07F
:100AC0006BF8431F5C425C4101A8FDF701FB44B198
:100AD0009DF80C1002980122FFF7F4FEE1E70024D4
:100AE000F2E7064B1B68986A03685B6B984708B18E
:100AF000FFF794FE04B070BD442F0020301000209A
:100B0000FFF7CCBF10B50446FDF734F9204610BD01
:100B100038B51148114D05F0A3FE114A11490E4890
:100B200011F0FCFE2846002340F8043B05F098FE37
:100B30001420FDF717F9044610B19B2106F0AAFE18
:100B40000949074A05482C6011F0E8FEBDE8384025
:100B50000648002100F0C8B8282F0020442F0020AC
:100B6000E046002079ED00087DED00087A2F002096
:100B7000D1ED007A90ED007AF4EE477AF1EE10FABA
:100B800004D0C0ED007A0121FEF7C6BE7047000018
:100B900090ED000A7047000091F900300370704733
:100BA00091F9002090F90010914202D00270FEF7F6
:100BB00091BE704791F9001090F900309FED097ACD
:100BC00001705B1A07EE903AF8EEE77AF0EEE77AFA
:100BD000F4EEC77AF1EE10FA4CBF01210021FEF7C6
:100BE0009BBE00BF0000003491F9002090F9001076
:100BF000914203D002700121FEF78EBE70470000C3
:100C000090F9003000EE103AB8EEC00A70470000CC
:100C100038B504460D46FEF781FF10B9B5F900302E
:100C2000238038BDB1F9003003807047B1F900105E
:100C3000B0F900309FED097A01805B1A07EE903A17
:100C4000F8EEE77AF0EEE77AF4EEC77AF1EE10FA12
:100C50004CBF01210021FEF75FBE00BF0000003441
:100C6000B1F90020B0F90010914203D002800121B7
:100C7000FEF752BE70470000B0F9003000EE103AA7
:100C8000B8EEC00A7047000038B504460D46FEF7BE
:100C900045FF08B92B68236038BD00000B6803606E
:100CA000704700000A6801688A4203D0026001218F
:100CB000FEF732BE7047000090ED000AB8EEC00AA1
:100CC0007047000008B5064B1B68586903685B68ED
:100CD000984720B9BDE80840024805F043BE08BD6A
:100CE000301000202C750208017011B100234380E0
:100CF00070474FF44873FAE770B51C460378A3B900
:100D0000B2F5487F11D212FA84F3B3F5487F094B4C
:100D10001B685869C8BFC2F548750368D4BFA5B23F
:100D2000ADB29E682B46B047641BB4FA84F040090C
:100D300070BD00BF3010002070B51C460378A3B909
:100D4000B1F5487F11D211FA84F3B3F5487F094B0E
:100D50001B685869C8BFC1F548750368D4BFA5B200
:100D6000ADB2DE682B46B047641BB4FA84F040098C
:100D700070BD00BF3010002010B5044B044918604E
:100D80000446FFF74FFC204610BD00BF842F002013
:100D9000BC75020890F8233063B9012380F8233032
:100DA000054800684FF40073006C80224FF4E13175
:100DB000FDF714BA704700BF30100020002850DD46
:100DC0006F2846D01BDC132845D00EDC431E082BB1
:100DD00011D8082B33D8DFE803F041053236323220
:100DE000323239004FF416607047392839D0642800
:100DF0003AD026283AD04FF47A7358437047B0F56A
:100E0000FA7F36D010DCB0F5807F34D006DC732852
:100E100034D0E628EFD14FF461307047B0F5E67F6B
:100E2000E9D14FF4E120704740F2DC53984228D0DA
:100E3000B0F5FA6F27D040F29933984225D0B0F53B
:100E4000FA6FD8DD70474FF4965070474FF4165044
:100E500070470F4870474FF4964070474FF49660C4
:100E600070474FF4614070470A4870474FF416408E
:100E70007047094870474FF47A3070474FF4E130BB
:100E8000704706487047064870474FF46120D9E71D
:100E9000FCB10100A086010020A1070060E316005C
:100EA00080841E000068FFF789BF0000914215D0C2
:100EB000CBB2581E012801D92B2905D1511EC9B228
:100EC00001290BD92B2A09D0053B012B08D8501F2B
:100ED000C0B201288CBF002001207047012070475C
:100EE000002070472DE9F84300250446894617463F
:100EF0002E4600F1060818F9352049462046FFF72E
:100F0000D5FF38B1B74203D104EBC500BDE8F88383
:100F10000136F6B20135042DEDD10020F6E70000D0
:100F200010B5FFF7DFFF78B1C379092B0CD8074A5A
:100F30001033126852F8234024B1236881885B6B18
:100F400020469847204610BD0024FBE730100020C3
:100F50000E4B70B51D68CBB2092B0C4612D810335E
:100F600055F8232000EBC103116810464E6B998899
:100F7000B04750B9A8690649036822461B68BDE816
:100F80007040184700231B68FFDE70BD3010002042
:100F90004C7502082DE9FF41FF23804603A921304B
:100FA0008DF80C30FFF720FE4046FFF7F3FE564B5E
:100FB0001B68019308F1080401267327019A06F1C2
:100FC000100352F82350E6717DB3B1B24046FFF7EB
:100FD000BFFF94F906300133332B00F28C80DFE839
:100FE00003F0241A1A1A2C3335353D478A338A52B6
:100FF0008A8A245A8A8A698A8A4C8A7D8A8A8A8A53
:101000008A248A8A8A8A8A8A8A8A8A8A8A8A1A8A16
:101010008A8A8A8A8A242046FFF744FF4FF4807325
:10102000014680222846FDF7D9F80136042E04F146
:101030000804C3D104B0BDE8F081092303A9204608
:101040000393FFF72BFEF0E73923F7E72046FFF77E
:1010500029FF102301464FF48072E3E703A92046DD
:101060000397FFF71BFE80231A464FF4E131D9E7BF
:1010700003A920460397FFF711FE2046FFF712FF52
:1010800080230146CDE7092303A9A01D8DF80C306C
:10109000FFF790FDC9E703A920460397FFF7FEFD80
:1010A0002046FFF7FFFE1E2301461A462846FDF79D
:1010B00095F80DE02046FFF7F5FE802301461A461D
:1010C0002846FDF78BF82B680121DB6C28469847F2
:1010D0002B680021DB6B28469847A6E703A920462A
:1010E0000397FFF7D1FD2046FFF7DCFE10230146F2
:1010F0004FF40072DAE72046FFF7D4FE0146284697
:10110000FDF776F891E700BF30100020032973B592
:1011100005461E460CD8CC00A01D01A928448DF818
:101120000420FFF739FD01A928190196FFF7B6FD44
:1011300002B070BD10B503680281194343680160B5
:1011400001334360044B1B68DC6AA162D96A4068C2
:101150008885DB6ADA8510BD3010002000487047B2
:10116000882F002010B509490446F9F7C5FF28B1BA
:1011700007492046F9F7C0FF28B90120054B142282
:1011800002FB003010BD0020FCE700BF4C760208D7
:101190006FD8020834BD020810B50C46FFF7E2FF15
:1011A00010B183682360006910BD00007047000023
:1011B0002DE9F74F07460E46F9F7A8FFDFF874B0A0
:1011C00005464FF0140A00F101083488012C2BD891
:1011D000174A0AFB04F3384652F803902A46494658
:1011E00012F070F9E8B919F9052015B12F2A00D0CD
:1011F000BAB909EB08022F211046019212F02AF920
:101200004CB138B1019A821A42445946484611F00D
:101210005DFC30B1012401343480484603B0BDE8A0
:10122000F08F01343480D0E74FF00009F5E700BFBC
:1012300034BD02084C76020810B50C46FFF792FF49
:1012400010B183682360012010BD000010B505496E
:101250000446FFF7E7F9044B4FF0FF321A602046CF
:1012600010BD00BF7CBD0208942F002010B5B0F95E
:101270000030B0F902209A42044626DDC28922B32A
:1012800007EE902ADFED140AB8EE671ABE20FDF7CC
:1012900015FDE28994F9063007EE102ABBB9B4F9BE
:1012A0000030B4F90220D21A07EE902AF8EEE77A5D
:1012B000B8EE477A27EE800AC0EE077AFCEEE77AAE
:1012C00017EE900A184480B200E098B210BDF8EE14
:1012D000C77A37EEC00AE2E70000000010B5C38904
:1012E00004460BB9808810BD90F906200AB1B1EE12
:1012F000400A5A4207EE903A00EE902AB8EE671A7A
:10130000F8EEE00ACE20FDF7D9FCE389B5EEC00A7D
:10131000F1EE10FA07EE103AB4F9043013DDB4F927
:101320000220D21A07EE902AF8EEE77AB8EE477A52
:1013300027EE800AC0EE077AFCEEE77A17EE900AF5
:10134000034498B2CFE7B4F900209A1A07EE902A26
:10135000F8EEE77AB8EE477A20EE670AC0EE077A31
:10136000FCEEE77A17EE900A1B1AEAE7037BDB072D
:1013700001D5FFF7B3BFFFF779BF0000C37C03B10E
:101380003AB1044A4181417B01238B4011680B43F0
:1013900013607047942F002010B5C38907EE903A70
:1013A000F8EEE77A044627EE800AFFF7DFFF002217
:1013B00001462046BDE81040FFF7E0BF037BC18136
:1013C00023F0030343F0030303737047037BC181DE
:1013D00023F0030343F0020303737047552813DC23
:1013E000442806DC1E3880B20A288CBF0020012069
:1013F00070474538012380B203FA00F0044B1842CD
:1014000014BF012000207047A03880B21328ECE7F9
:1014100033F0010010B5427B012393400B4A126860
:101420001342044609D1B0F90800FFF7D7FF10B105
:10143000074B1B7813B9E37C13B110BD9FED050A70
:101440002046FFF793FF6081F7E700BF942F00204D
:10145000C42F002000000000B0F90800552808DC67
:1014600051280DDC213883B2072B0AD94FF0FF3009
:101470007047A0F1A0039BB2132BF7D86C3000E0AB
:101480004A3840B27047000010B40A4A417B1268E3
:1014900001238B4013420AD1074B1B685B6A1A6811
:1014A00054694289184623465DF8044B18475DF895
:1014B000044B7047A82F00203010002038B5054D90
:1014C0000024286820441434FFF7DEFFB42CF8D140
:1014D00038BD00BFE42F002008289FBF054B1B68C4
:1014E00000EB800003EB800094BFB0F908000020FF
:1014F000704700BFE42F0020037B9B0729D4B0F97D
:1015000008305C2B32DC452B0BDC1A2B22DC172B32
:1015100037DC0B2B4BD018DC032B13DC012B46DC08
:101520007047463B162B14D8DFE803F041131341F4
:10153000412B2B2B2B2B2B44131313132B2B13135C
:1015400013134400042B1CD07047103B9BB2052B97
:1015500017D97047292B2DD004DC1F3B9BB2012BE0
:1015600028D970472D3B9BB2022BF1E77F2B08D087
:1015700011DC7D2B0CDC7B2B03DC6D2B05DC5D2B68
:10158000E7D041F29411FFF719BF6E2B0FD07047CF
:101590007E2B0FD070479C2B09D003DC8C3B9BB279
:1015A0000F2BD5E7B43B9BB2032B03D970476421C3
:1015B000FFF70CBF4FF47A71FAE700002DE9F04F06
:1015C000324D334E2A68334F336802432A603A68FB
:1015D0001943316085B002F1B4010124B2F9083039
:1015E0007B2B06DC772B08DD537B04FA03F31843CF
:1015F00003E0813B9BB2032BF6D914328A42EDD132
:10160000254B1B685B6A1A680146D2F88C20184685
:101610009047224B4FF0000B18604FF001094FF03C
:10162000140A4FF47A782A6809FA0BF3134224D08B
:101630003C6801930AFB0B440DF10E012046ADF806
:101640000E80FFF7EFFA4FF4FA620DF10E01A01CC5
:10165000ADF80E20FFF7E6FA019B3268134218BF7F
:1016600040F2DC5304F104000DF10E0114BFADF89B
:101670000E30ADF80E80FFF7D5FA0BF1010BBBF180
:10168000090FD0D105B0BDE8F08F00BFA02F00201A
:10169000C82F0020E42F002030100020A82F0020A9
:1016A00083B2B72B0BD8064B03EBC00282ED010AC5
:1016B000044A53F83010136823EA0103136070479B
:1016C000E82F0020942F0020F8B5084F054600248D
:1016D0000EB23B681819B0F90830AB4202D131465E
:1016E000FFF76CFE1434B42CF3D1F8BDE42F0020C6
:1016F000F8B5084E05460F46002433681819B0F9AE
:101700000830AB4202D13946FFF760FE1434B42CE6
:10171000F3D1F8BDE42F0020B72908B508D9FFF7A9
:101720001DFDBDE80840A2224FF40031FFF702BDC5
:101730004A09012301F01F0103FA01F150F8223098
:101740000B4340F8223008BD2DE9F74FDFF88880C1
:10175000D8F800303BB318221B481C4E002111F072
:10176000EDF900231A4646F833200133B82BFAD19D
:10177000174FDFF854903A6000244FF0140A4FF0EE
:10178000010BD8F800000AFB04000BFA04F30589EA
:10179000B72D0BD93A6813433B600134092CF0D1C3
:1017A0000C4B01221A7003B0BDE8F08F0193FFF7D4
:1017B000A3FE29464846FFF7AFFF56F83520019BA8
:1017C000134346F83530E8E7AC2F0020E82F00201F
:1017D000A42F00209C2F0020E42F0020274B2DE970
:1017E000F0471F68264BDFF89C801A68DFF898A046
:1017F000B2F856130646786A0368D3F890309847D3
:10180000FFF7A2FF00254FF00109D8F80040786AE1
:101810002C44D0F800C02389617BB72B20D8DAF89C
:10182000003009FA01F21A421AD1DCF80C3098475C
:10183000B4F90830862B16D1218800222046FFF704
:101840009DFD2046FFF720FE1435B42DDDD1786ACA
:1018500003685B6A9847301DBDE8F04703F00ABC97
:10186000DCF81030E3E7872B02D1A1880022E5E7FE
:10187000882BE9D161880022E0E700BF301000200A
:10188000982F0020E42F0020A82F002038B50E4B01
:101890001B7804460D460BB9FFF756FFA3B2B72BD2
:1018A0000FD80A4B53F83420002A92FAA2F3B3FA65
:1018B00083F308BF4FF0FF33581C01D02B70012079
:1018C00038BD0020FCE700BF9C2F0020E82F00203F
:1018D00007B508460DF10701FFF7D8FF78B1094BAE
:1018E00009491B6809685A6A9DF8073003EB8303AE
:1018F00001EB830031F8233040881081D38003B09E
:101900005DF804FB30100020E42F002010B50F4BD1
:101910001B7804460BB9FFF717FFA3B2B72B08D902
:10192000FFF71CFCA2224FF40031FFF703FC00205C
:1019300010BD074A5B09012052F8233004F01F0450
:1019400000FA04F41C4208BF0020F1E79C2F00209D
:10195000AC2F0020F8B505460E46FFF7D7FF90B133
:10196000094F00243B681819B0F90830AB4207D181
:1019700000223146FFF702FD38682044FFF784FD5E
:101980001434B42CEED1F8BDE42F002070B52DED49
:10199000028B0546B0EE408AFFF7B8FF70B1094EE2
:1019A000002433681819B0F90830AB4203D1B0EE07
:1019B000480AFFF7F1FC1434B42CF2D1BDEC028BD1
:1019C00070BD00BFE42F00200828F7B50C461AD8D8
:1019D0000E4DADF806102B6800EB8000870003EB7E
:1019E00080000DF1060130F9086FFFF711F92B683F
:1019F0003B44B3F908309E4205D09C4203D10448D1
:101A0000A1B2FFF789FE03B0F0BD00BFE42F0020B4
:101A1000AC2F0020F8B50446043002F09DFF04F519
:101A20002876354604F5557728461435FFF70EFC21
:101A3000BD42F9D104F5597004F012FF094D0A4B6B
:101A40000A491C6020462E60FEF7ECFD2A68002340
:101A50000D32142000FB03F153540133092BF9D14B
:101A60002046F8BDE42F0020982F00202CBE02084D
:101A7000043003F09DBB00002DE9F0412DED028BF9
:101A80002B4B9FED2C8A1C682B4E82B004B3D4EDF7
:101A9000027AF4EEC87AF1EE10FA11DBB4F90050D4
:101AA000D4ED010A06EBC50537EEA01A95ED010A43
:101AB00070EEE70A40F29710FDF700F985ED010A94
:101AC000B4F9003006EBC3035B686360E468DDE7EC
:101AD0001A4B1B4D19681B4EDFF85C804FF4CE7219
:101AE00001F5597101A8FCF7D1FA0127306835F8E2
:101AF000023B2044B3B9C3740289B0F90830B72A55
:101B000005D808EBC30393ED010AFFF783FC1434F7
:101B1000B42CEBD101A8FCF7DBFA02B0BDEC028BD0
:101B2000BDE8F081013BC77425F8023CE4E700BF43
:101B3000E02F002000000034E82F0020982F002024
:101B4000CC2F0020E42F0020024B1B68586A03684A
:101B50001B6B18473010002010B5064B1B6804465D
:101B6000586A03685B6B9847201DBDE8104003F07E
:101B7000A1BC00BF3010002010B50446FFF7ACFC3C
:101B800001300CD0074B186840B1012202FA04F36F
:101B9000D0F85C23134214BF0120002010BD0120A7
:101BA000FCE700BF982F0020014B1868704700BF6A
:101BB000982F002002481822002110F0BFBF00BF5C
:101BC000AC2F002010B506490446FEF72BFD054B4F
:101BD0001A6812B1044805F083FC1C60204610BD51
:101BE000B0BF0208A83500202CBF020838B50D4C44
:101BF0000D4D237845F82310486055F823000368FD
:101C00009B689847237850B955F8230010B10368B2
:101C10005B6898472378002245F8232038BD0133BC
:101C20002370FBE7AC350020D03500202DE9F04FC4
:101C3000A64D2B7885B00446002B00F0788105B0C6
:101C4000BDE8F08FA3680AEA0303802B00F0B080A0
:101C500047D8082B00F0D2802ED8022B7CD0042B42
:101C600000F08B80B9F101094FEA4A0AEAD1142049
:101C7000FCF778F8064640B11422494610F05EFFA2
:101C8000934B336044F62063338231462046FFF79E
:101C9000ADFF2B78052BD2D81C20FCF763F801464A
:101CA00020B18C4B036040F6E4430383204605B02B
:101CB000BDE8F04FFFF79ABF402BD3D13B6858687F
:101CC00003689B6898474FF0000B804606FA0BF3B9
:101CD00013EA080F59D10BF1010BBBF1200FF5D11D
:101CE000C0E7B3F5804F00F0B7801AD8B3F5006FA6
:101CF00000F08D80B3F5005FB4D13B68586803688D
:101D00009B6898474FF00008834606FA08F313EAE9
:101D10000B0F40F08C8008F10108B8F1200FF4D1CE
:101D2000A0E7B3F5004F00F0BE80B3F5803F99D136
:101D30003B6858680368DB6898474FF000088346A3
:101D400006FA08F313EA0B0F40F0DC8008F10108F3
:101D5000B8F1200FF4D185E75820FCF703F880464E
:101D600010B1002101F006FC41462046FFF73EFF7E
:101D70002B78052B7FF676AF61E75820FBF7F2FF53
:101D800080460028F0D00121ECE75820FBF7EAFF5D
:101D9000034628B15FFA8BF1039001F045F8039BED
:101DA00019462046FFF722FF2B78052B93D946E7EB
:101DB0003B6858680368DB6898474FF0000B804623
:101DC00006FA0BF313EA080F05D10BF1010BBBF177
:101DD000200FF5D146E75820FBF7C4FF034628B192
:101DE0005FFA8BF1039001F01FF8039B1946204620
:101DF000FFF7FCFE2B78052BE7D920E75420FBF7F3
:101E0000B1FF80460028AFD001F0F6F8ACE74C20D7
:101E1000FBF7A8FF80460028A6D001231A460096AB
:101E2000002101F0DDF92C4BC8F800309CE75C2064
:101E3000FBF798FF034630B130225FFA88F1039038
:101E400000F00CFF039B19462046FFF7CFFE2B78CE
:101E5000052B7FF660AFF2E63B6858680368DB68E5
:101E600098474FF00008834606FA08F313EA0B0F71
:101E700005D108F10108B8F1200FF5D1F2E65C2098
:101E8000FBF770FF034630B130225FFA88F1039010
:101E900000F0E4FE039B19462046FFF7A7FE2B78CF
:101EA000052BE6D9CBE63B68586803689B689847E2
:101EB0004FF00008834606FA08F313EA0B0F0DD122
:101EC00008F10108B8F1200FF5D1CBE6AC350020C0
:101ED0000CC3020858C0020884C002085820FBF74F
:101EE00041FF034630B154225FFA88F1039000F0BD
:101EF0006BFE039B19462046FFF778FE2B78052BD7
:101F0000DED99CE65820FBF72DFF034630B1542262
:101F10005FFA88F1039000F057FE039B19462046B4
:101F2000FFF764FE2B78052B7FF610AF87E64FF0A6
:101F3000010A024F4FF01109564693E63010002077
:101F4000FFF774BE70B5094D094E00242A78E3B23C
:101F50009A4207D956F8230010B10368DB68984706
:101F60000134F3E7034B00221A6070BDAC3500204A
:101F7000D0350020CC3500202DE9F74FDFF83C901C
:101F8000DFF83CA005460E4617469846002499F80F
:101F90000020E3B29A420DD95AF8230040B10368F9
:101FA000CDF80080D3F814B032463B462946D847D6
:101FB0000134ECE703B0BDE8F08F00BFAC35002082
:101FC000D03500200378013BDBB2022B9ABF024AD6
:101FD000D0560020704700BFACBF02087047000019
:101FE0007047000070470000704700007047000015
:101FF0007047000010B50446FBF7BCFE204610BD3C
:1020000038B5294B1B780446D80702D54FF000435A
:102010002FE005F093FA6369C01A238B984241D3ED
:10202000224D237A2A7FC3F34011914207D062F3F5
:10203000451323721E4BE36005F080FA6061AB79B3
:1020400053B1237A590607D443F040032372194B46
:10205000E36005F073FA6061237A2A79C3F38001A3
:1020600091420BD062F382035A072372CED56FF0F0
:102070000303E36005F062FA606113E0EA7BC3F3F7
:102080000011914206D062F304132372DB0609D5D6
:10209000094BEEE7EB7D13B14FF02043E9E7EB7A14
:1020A000002BB3D138BD00BFCC350020AD350020AA
:1020B000002049920000FFAB000040ED10B4037A0D
:1020C00003F001028A4216D061F3000303724368F1
:1020D0001A7B0A4B1B68DB6919680C69017C007A62
:1020E000C00758BFB2FA82F2184658BF52092346B9
:1020F0005DF8044B18475DF8044B70473010002022
:1021000010B5436893F9022004460AB9002010BDB7
:1021100093F9051001740029F8DD0C4B1B68D86990
:10212000036801225B68C9B2984700212046FFF787
:10213000C5FF074B227A197961F382022272DA7A9B
:10214000237A62F3C30323720120E0E730100020FA
:10215000AD35002010B5C368044663B105F0EEF953
:102160006369C01AB0F5486F06D300212046FFF717
:10217000A5FF0023E36010BD6423B0FBF3F04FF034
:10218000004323FA00F0E368184218BF01212046FB
:1021900008BF0021BDE81040FFF790BF10B504460E
:1021A000FFF72EFF2046BDE81040FFF7D3BF000029
:1021B000012070472DE9F7431F46244B1C68E36A52
:1021C00093F89C300D4616461BB1002003B0BDE8C5
:1021D000F083606A0368D3F8B030984701282DD1A6
:1021E000606A0368002D4FF00A084FF0000514BF25
:1021F00017211B21D3F8B490FF222B46CDE900858F
:10220000C847606A0368AE4214BF18211C21D3F886
:10221000B490FF222B46CDE90085C847606A036869
:10222000AF42D3F8B4404FF0FF02CDE900852B4612
:1022300014BF16211A21A0470120C7E7606A03686E
:10224000D3F8B03098470328BFD1C9E73010002039
:102250007047000010B50446FBF78CFD204610BD0A
:10226000012303FA01F1837C23EA010181747047A1
:102270007047000010B50446FBF77CFD204610BDFA
:102280002DE9F84F9246134A03EB830380468946B3
:10229000002402EB030B052C09EB040714BF1BF809
:1022A000046000260025BFB2D8F808000368F107D3
:1022B0000AEB05024CBF5B689B6892B23946013558
:1022C0009847082D4FEA5606EED10134062CE2D18C
:1022D000BDE8F88F28C10208F8B506460C46174637
:1022E0005D1E15F9011F69B12039C9B25E2994BF7D
:1022F0004BB2002321463A4630460734FFF7C0FF71
:10230000A4B2EEE7F8BD000070B5054686B01446ED
:102310000E46F1B1052A1CD8012303FA02F2837C90
:10232000134383741322202101A810F007FC13210A
:10233000304611F0EFF804EB84040246314601A860
:1023400010F0D4FB620001AB063200212846FFF7F3
:10235000C3FF06B070BD0000064B01EB81014A00CF
:102360001979063219B1044B0021FFF7B5BF034BB1
:10237000FBE700BFAD350020B0C00208C3C00208B3
:10238000064B01EB81014A009979063219B1044BE1
:102390000021FFF7A1BF034BFBE700BFAD350020D5
:1023A000D8C00208EBC00208064B01EB81014A00CD
:1023B000D97B063219B1044B0021FFF78DBF034BC7
:1023C000FBE700BFAD35002000C102080DC10208C7
:1023D00030B54368094A87B00C4605464833132197
:1023E00001A804EB840404F05DFA620001AB06323C
:1023F00000212846FFF770FF07B030BD1CC102085E
:1024000070B5002686B005460C460F22314602A85C
:1024100010F094FB04EB84041222202101A810F098
:102420008DFB6200AE8101AB063231462846FFF7D4
:1024300053FF06B070BD000070B5002594B004468F
:102440000F220E4603A82946029510F077FB2F2293
:10245000294608A8079510F071FB05F06FF863682E
:102460005A6C801A228A904205D331462046FFF7E3
:10247000C7FF14B070BD627B12B1013A6273F8E716
:102480000F33144A332107A804F00CFA122220213A
:1024900002A810F053FB257B07AB591908460191A0
:1024A000F8F734FEC2B2122A28BF1222019906465A
:1024B00002A810F01BFB122E95BF4FF4806301356C
:1024C000A381257302AB062200212046FFF704FFFB
:1024D000CFE700BF22C1020810B5817C11F00101D5
:1024E000044601D1FFF7A8FFA37C990703D401217B
:1024F0002046FFF76DFFA37CDA0603D404212046B3
:10250000FFF73EFFA37C9B0605D420460521BDE8CE
:102510001040FFF749BF10BD10B5164A1378182BAD
:10252000044602D80133137010BD00231370124A01
:10253000837B12798AB1012BF6D080680368DB684F
:10254000984703212046FFF707FF0123A373A068E4
:102550000368BDE810401B681847022B05D080684F
:102560000368DB6898470223A3732046FFF7B4FF94
:10257000EDE700BFE8350020AD35002010B504467A
:10258000006810B103685B689847204610BD0000E2
:1025900010B50446006810B103685B689847204690
:1025A00010BD00002DE9F04F856887B0044645BB9B
:1025B0002E4B1E68706803685B6898472C4B074673
:1025C0004FF0010A4FF004090AFA05F23A4207D126
:1025D0000135202DF8D1A06860B907B0BDE8F08FB3
:1025E000626892F90320012A0DD0022A2AD0A2683B
:1025F000002AEDD02046FFF76FFFA06803681B6834
:1026000098470120E9E770684FF000080268CDF8AC
:102610000490CDF80080D2F800B0E9B23C22D8474F
:10262000039003A8CDE9048800F012FAA06003A883
:10263000FFF7AEFF04A8FFF7ABFF05A8FFF79EFF6B
:102640000B4BD4E770684FF000080268CDF8049097
:10265000CDF80080D2F800B0E9B23C22D847039010
:1026600003A8CDE9048800F0E7F8DFE73010002088
:10267000801A0600012380F8283470474FF48462E2
:102680000021083010F05ABAF0B5234B8DB005AADE
:10269000044603F11807164618685968154603C51D
:1026A0000833BB422A46F7D119889B782980AB7042
:1026B0004FF48462002104F1080010F03FFA6068D2
:1026C00018B9002528460DB0F0BD03689B6A9847ED
:1026D00003689B6898476068002302680093156947
:1026E00031461B22A8470546606803689B6A9847E5
:1026F0000368DB689847002DE3D0606803940123EA
:1027000084F828340368DE6A044B0493224644F6B6
:102710002061B047D6E700BF106C02080928010805
:10272000832910B50ED83F2A0CD8D308842404FB83
:1027300003110844012302F0070203FA02F2037AAC
:102740001A43027210BD0000832910B50ED83F2A2B
:102750000CD8D308842404FB0311084402F00702B8
:1027600001239340027A22EA0302027210BD0000A4
:102770002DE9F04190F8283494B00446002B3ED067
:102780002049002580F82854D1F81B0002904322EC
:102790001F3103A810F0AAF904F1080765F04F03F0
:1027A00060688DF80B30002603680096D3F810801F
:1027B0000422334602A9C047394642220DF10D00DA
:1027C00010F094F9606803680096D3F810804322F3
:1027D000334603A9C0474222B9180DF10D0010F08D
:1027E00085F9606803680096D3F810804322334669
:1027F00003A90135C047082D07F18407CED114B0D5
:10280000BDE8F081106C0208FFF7B2BF10B5044BB1
:10281000044640F8043BFFF7BBFE204610BD00BF56
:1028200038C3020810B50446FFF7F0FF2046FBF757
:10283000A1FA204610BD000037B5002503680560E9
:1028400040F22C400193FBF78DFA044620B10B4B6C
:102850000360019B4360019501A8FFF799FE54B105
:10286000236820469B699847054620B9236820467F
:102870005B6998472C46204603B030BD38C3020838
:10288000012380F8083470474FF48062002108303B
:1028900010F054B9F0B5214B8DB004AA044603F1F1
:1028A0002007164618685968154603C50833BB4209
:1028B0002A46F7D14FF48062002104F1080010F09D
:1028C0003DF9606818B9002528460DB0F0BD0368D1
:1028D0009B6A984703689B68984760680023026872
:1028E0000093156931462022A847054660680368B1
:1028F0009B6A98470368DB689847002DE3D06068BF
:102900000294012384F808340368DE6A044B0393BD
:10291000224644F62061B047D6E700BF746C020837
:10292000212A01087F290DD83F2A0BD8D30801EBB3
:10293000C3110844012302F0070203FA02F2037AEA
:102940001A430272704700007F290DD83F2A0BD826
:10295000D30801EBC311084402F00702012393409E
:10296000027A22EA03020272704700002DE9F04366
:1029700090F8083497B00646002B4CD02749002524
:102980008A8C80F80854086A91F826300390ADF8D4
:1029900010202731412205A88DF8123010F0A6F83A
:1029A00006F10807A84670688DF811500368CDF845
:1029B00000801C690722002303A9A0473C460DF1B3
:1029C000150307F1400254F8041B43F8041B94421A
:1029D000F9D170680368CDF80080D3F810904122D7
:1029E000002305A9C8470DF1150304F1400254F86E
:1029F000041B43F8041B9442F9D170680368CDF8B6
:102A000000801C694122002305A90135A047082D3B
:102A100007F18007C7D117B0BDE8F083746C0208D6
:102A2000FFF7A4BF10B5044B044640F8043BFFF782
:102A3000AFFD204610BD00BF5CC3020810B50446C0
:102A4000FFF7F0FF2046FBF795F9204610BD000088
:102A500037B500250368056040F20C400193FBF791
:102A600081F9044620B10B4B0360019B4360019543
:102A700001A8FFF78DFD54B1236820469B69984754
:102A8000054620B9236820465B6998472C462046B6
:102A900003B030BD5CC3020810B5054B03600446AB
:102AA000C06C10B103685B689847204610BD00BF3A
:102AB00080C3020880F85530012380F8531080F855
:102AC000542080F85230184670470000F0B5364B5D
:102AD0001F680446786894F85010036887B0042291
:102AE0000026CDE9006294F851201D682F4BA847BD
:102AF0000546E064C0B103689B6A98473D220146E1
:102B000003A8FBF7DFFAE06C03680A21DB6C984747
:102B1000E06C01230DF10B02314604F021FE30B9C7
:102B2000002503A8FBF7D4FA284607B0F0BD9DF8AE
:102B30000B3094F85120B3EB420FF1D1E06C3346E7
:102B4000C5225F2104F0E8FD0028E9D0B86A0368D7
:102B500064219B6898470123E06C0DF10B02194634
:102B600004F0FEFD0028DBD09DF80B30F02BD7D110
:102B7000E06C3346F122012104F0CEFD0546002829
:102B8000CED0E06C03680121DB6C9847E06C0494C4
:102B90000368DE6A064B059306AB13E90C0044F6A6
:102BA0002061B047BDE700BF30100020801A06004A
:102BB000412C010810B50446FFF76EFF2046FBF7D5
:102BC000D9F8204610BD000073B555230E461546B2
:102BD0000093FF22AA230021044600F001FB044BCE
:102BE0002360204684F8506084F8515002B070BDD4
:102BF00080C3020870B590F852300446FBB100253E
:102C000090F8532080F852502B461021C06C04F0ED
:102C100083FD94F85420E06C2B46212104F07CFDC8
:102C200094F85520E06C2B46322104F075FDE06CE1
:102C30002B46C522BDE87040502104F06DBD70BD2B
:102C4000FFF7D8BF80F85330012380F8542080F874
:102C5000551080F8523018467047000073B5552360
:102C60000E4615460093FF22AA230021044600F0D9
:102C7000B7FA054B236020460023E36484F85060D4
:102C800084F8515002B070BDB4C30208F8B590F892
:102C900052300546C3B1002380F8523000F1560689
:102CA000022416F8037C3378BB4206F1010607D0F4
:102CB000E86C00233A46214604F02EFD06F8017C1C
:102CC0000134E4B2052CECD1F8BD0000FFF7DEBF03
:102CD00010B5044B044640F84C3BFFF74FFC204630
:102CE00010BD00BFB4C3020810B50446FFF7F0FFE3
:102CF0002046FBF73FF8204610BD0000F0B5414BE1
:102D00001F680446786894F85010036887B000255F
:102D10000422CDE9005294F851201E683A4BB04786
:102D2000E36C0495E0641BB11A681846526890473A
:102D300004AE3046FFF722FCE06C002860D0036848
:102D40009B6A98473E22014603A8FBF7BBF9E06C5B
:102D500003680A21DB6C9847E06C0023FF220D21F9
:102D600004F0DAFC30B9002503A8FBF7B1F92846D6
:102D700007B0F0BDB86A036864219B6898470525D1
:102D8000E06C01233246294604F0EAFC0028EAD030
:102D90009DF81030AF2BE6D10135EDB2082DEFD103
:102DA0000023E06C4022194604F0B6FC0028DAD07B
:102DB000B86A03684FF4FA719B689847E06C002387
:102DC0000122294604F0A8FC0028CCD00023E06CA6
:102DD0001A46702104F0A0FC05460028C3D0E06C20
:102DE00003680121DB6C9847E06C0368DF6A074BDE
:102DF0000494059396E80C0044F62061B847B3E7C5
:102E00000546B4E730100020801A0600CD2C0108DA
:102E100080F85230012380F8501080F8512080F85B
:102E2000533018467047000037B50F230D46009306
:102E30001F2218230021044600F0D2F9044B23601E
:102E400020460023E36484F8545003B030BD00BF33
:102E5000E8C302081FB51F2301F0E001C2EB022204
:102E6000B2FBF3F21A40C06C0A438DF80C200268E2
:102E700000230093146903A90122A04704B010BDE8
:102E800070B506464D1E402415F8012F21463046E8
:102E9000FFF7E0FF18B12034E4B2A02CF4D170BDEC
:102EA00090F8533001462BB1002380F85330503155
:102EB000FFF7E6BF70470000FFF7F2BF10B5044B05
:102EC000044640F84C3BFFF759FB204610BD00BFBD
:102ED000E8C3020810B50446FFF7F0FF2046FAF7F2
:102EE00049FF204610BD00002DE9F04B88B043F6A5
:102EF0003813ADF81030374BDFF8E0B01B680393A0
:102F000004460DF110094FF002080427039B94F8C2
:102F10005410586800250368019700951E6819F839
:102F2000012B5B46B047E36C0695E0641BB11A6861
:102F300018465268904706AE3046FFF71FFBE06C1C
:102F4000C0B103689B6A984703689B689847E06C28
:102F500003680A21DB6C98471F2220212046FFF7D7
:102F600079FF054670B9E06C03689B6A984703686F
:102F7000DB689847B8F1010F01D1002526E04FF03A
:102F80000108C3E7E37A8DF8143005A920468DF8CF
:102F900015308DF81630FFF773FF0746E06C0368B5
:102FA0000121DB6C9847E06C03689B6A98470368D3
:102FB000DB68984757B1E06C0368DF6A064B0694FC
:102FC000079396E80C0044F62061B847284608B0FD
:102FD000BDE8F08B30100020B92E0108801A0600E1
:102FE00080F85230012380F8501080F8512080F88A
:102FF000533018467047000013B54F23009300224A
:103000007F23FF21044600F0EBF8034B23602046AA
:103010000023E36402B010BD1CC4020830B590F870
:10302000533087B043B390F8502090F8511090F887
:1030300052400023CDE90233120109012401CDF8E9
:103040000F3080F853308DF80B40C06C8DF80F10A6
:10305000240A090A8DF813200625120A8DF80C405F
:103060008DF810108DF808508DF814200268009328
:10307000146902A90D22A04707B030BDFFF7CEBFEB
:1030800010B5044B044640F84C3BFFF777FA204656
:1030900010BD00BF1CC4020810B50446FFF7F0FFC6
:1030A0002046FAF767FE204610BD0000F0B5364B0B
:1030B0001B680646586887B0002404220368CDE9DF
:1030C000004201211D68314B4022A847F36C049453
:1030D000F0641BB11A6818465268904704AF38462E
:1030E000FFF74CFAF06C00284CD003689B6A9847B5
:1030F00003689B689847F06C03680521DB6C00252A
:103100009847F06C8DF80B5001230DF10B02294606
:1031100004F026FB0446F06C44B903689B6A9847A8
:103120000368DB689847204607B0F0BD9DF80B3078
:103130008DF80C5023F0300343F020038DF80D3050
:10314000036800951C6902222B4603A9A047044688
:10315000F06C0368002CE1D00121DB6C9847F06C27
:1031600003689B6A98470368DB689847F06C0368BC
:10317000DD6A074B0496059397E80C0044F620613E
:10318000A847D0E70446CEE730100020801A06009A
:103190007D3001082DE9F0411D46037A8B4204463B
:1031A0000F46164605D1437A934202D1837AAB4249
:1031B0000BD023683246D3F8248039462B4620466C
:1031C000C04710B127726672A572BDE8F081000099
:1031D00010B59DF80840C47401744274837410BD26
:1031E00030B543739DF80C308373144B836103F146
:1031F000764303F5AB43C361114B0362A3F1DB5389
:10320000A3F558234362A3F1DB53A3F5582383624C
:103210000C4B027346F6B652C0E90B230A4D0B4B1A
:10322000C1720B4905600B4DC0E90D1342F2924388
:10323000C0E90F5341F24923436430BD0CC3300C45
:10324000B6EDFF3F9224491250C4020836600300D5
:10325000499224098220080230B4456895F901504A
:10326000012D04D00468A46AA44630BC604730BC79
:103270007047000038B54368057B93F90030012B97
:10328000044610D0022B10D003B9C57A084B1B6836
:10329000D86903689B6B984718B1A37B9D4228BFF0
:1032A0001D46284638BD857BF0E7457BEEE700BF2D
:1032B00030100020174B1A780AB1806970471A7ACB
:1032C0002AB95A7A1AB99A7C0AB9DA7E0AB1C0695F
:1032D0007047997ADA7C51B9197B41B9D97A31B9F9
:1032E000D97B69B9597D71B912B9406C70470AB17F
:1032F000006A7047DA7B42B1406A7047C06A704723
:10330000002AF9D0F4E7002AF2D15B7D002BF5D03A
:10331000806A7047AD35002010B5104C2378C3B9D2
:103320002379C3B90E4B1B68D86A0368DB699847D9
:103330000128A37906D00B4846F6B652002B18BFD9
:10334000104610BD084A42F29240002B08BF1046BA
:10335000F7E70648F5E744F62410F2E7AD3500201C
:1033600030100020866118068220080254A85001FF
:1033700070B5C37C044643B90368427C9D6A017CF6
:10338000837CAC46BDE8704060474FF47A75B5FB6E
:10339000F3F504F0D3F86369C01AB0FBF5F305FB4D
:1033A00013002368B0EB550F9D6A83BF627CA37C3A
:1033B000217C00239CBF1A4619462046E1E7000005
:1033C00070B5436893F901300446032B46D8DFE813
:1033D00003F006020A42BDE87040FFF7C9BFFFF7DD
:1033E00069FF054606E01E4B1E4D1B791E48002B4B
:1033F00018BF05462046FFF73DFF064604F09EF83D
:103400000A2394F848106422B0FBF2F2B2FBF3F006
:1034100003FB1022D2B2914207D04A1CB2FBF3F157
:1034200003FB1122D2B284F8482002EB420225FAB3
:1034300002F2D3B2510754BFE17A31469A0754BF22
:10344000E27A3246DB0758BFE67A20463346BDE8CB
:103450007040FFF701BFFFF75FFFC2E70025C9E734
:10346000AD350020922449122449922410B5054B11
:1034700003600446C06C10B103685B68984720463F
:1034800010BD00BF84C4020880F85330012380F8C7
:10349000511080F8522080F85030184670470000D4
:1034A0002DE9F0412B4B1B680546586895F85410E0
:1034B000036886B000260427CDE9006755221C6802
:1034C000254BA0470446E864B8B103689B6A984757
:1034D0003822014602A8FAF7F5FDE86C03680A21D4
:1034E000DB6C9847E86C33460322394604F014F944
:1034F00038B9002402A8FAF7EBFD204606B0BDE873
:10350000F081EB7AE86C8DF80D304FF001088DF802
:103510000C808DF80E308DF80F30036800961C6912
:1035200003A933463A46A0470446E86C036841467F
:10353000DB6C9847002CDCD0E86C04950368DE6AED
:10354000064B059306AB13E90C0044F62061B04727
:10355000D0E700BF30100020801A0600E1350108D6
:1035600010B50446FFF782FF2046FAF703FC204619
:1035700010BD000037B511230D460093FF228023B4
:1035800000210446FFF72CFE034B2360204684F8FD
:10359000545003B030BD00BF84C402081FB590F87A
:1035A0005030DBB101228DF80C2090F85320120925
:1035B0008DF80D2090F8522012098DF80E2090F809
:1035C0005120002380F850301209C06C8DF80F2074
:1035D00002680093146903A90422A04704B010BD37
:1035E000FFF7DCBF704700002DE9F3410C68144D74
:1035F00094F900302F2B0F4608BF0134012655F8EF
:10360000361001910846F7F781FD5FFA80F80199BD
:10361000424620460FF056FF68B904EB08033B60B2
:1036200014F908202F2A04BF01333B6005EBC600C4
:1036300002B0BDE8F0810136042EE0D10048F7E782
:10364000C4C402080B680548B3F5806F3FBF1A0A6F
:10365000DBB20B6000EBC200704700BFC4C40208BD
:1036600030B585B0CDE9022103A90193FFF7BCFF76
:10367000044640680168DDE901320D680399A847F6
:10368000011E09DBFF290ADD606803685B68984753
:103690000FF016FA222303604FF0FF3005E00448D4
:1036A000201AC0F3C70001EB002005B030BD00BFF9
:1036B000C4C4020807B5019101A9FFF7C3FF406820
:1036C000019903685B68984703B05DF804FB00004C
:1036D0002DE9F3410E4601A990460193FFF7B2FF91
:1036E000054640680199036800225C690123A047F0
:1036F000071E03DA002002B0BDE8F0816868019976
:10370000036832469C684346A0470028F2DD002348
:10371000DCB2844256FA83F106DA32570D2A03D01E
:103720000A2A03F10103F3D100230B7068680199A1
:1037300002683C44013455692246A847231A58427E
:103740005841D8E700487047E935002010B5094CCA
:10375000094B204640F8043B03F082F8074A084929
:1037600020460FF0DBF8074B074A1A60074B084A60
:103770001A6010BD843700206CC50208E0460020A6
:10378000E53501082037002008C50208EC36002086
:10379000A0C60208002070474FF0FF3070470000BD
:1037A0004FF0FF3070470000002070470020704746
:1037B0004FF0FF30704700004FF0FF3070470000BF
:1037C00000207047002000217047000000200021E9
:1037D00070470000002070470120704770470000CC
:1037E00000207047002070470329F7B506460D46B4
:1037F00017461C4604D8182303FB01031A793AB96B
:103800000FF05EF9092303604FF0FF3003B0F0BD05
:10381000D3F818C0BCF1000FF2D0D96846F21B7281
:10382000ADF80020C1B1182202FB05629069D3688F
:1038300082682344934227D8182303FB0565224658
:10384000AB691868EB68394618440FF04FF9EB681C
:103850002344EB602046D9E7052CE4D93868009072
:1038600080B2B7F804E0DCF80830ADF804E090422C
:10387000D9D1BDF804209A42D5D9D21A604603F0B6
:10388000D3FE0028CFD1BFE79A1A002103F0CCFE67
:103890000028D1D1B8E70000032938B504D818248E
:1038A00004FB0104257935B90FF00AF909230360F7
:1038B0004FF0FF3038BD012B08D0022B09D003B9DF
:1038C000E260182303FB0100C068F3E7E3681A44D1
:1038D000F6E70FF0F5F81623E9E700002DE9F04FC1
:1038E0002DED028B8DB05568984600238A4614460C
:1038F0008DF82C30ADB915870DF1170106AA2046B9
:10390000FCF75AF9BAF80420ABB29A42064612D92B
:103910000135F0B106AA0DF117012046FCF7C6FAF1
:10392000F0E7138F013313870DF1170106AA204624
:10393000FCF7BCFA0646BAF8063056B1ABB1228F96
:103940009A4212D3002528460DB0BDEC028BBDE88B
:10395000F08FBAF80650002DF4D1248FFCF75EFFEB
:103960008442EFD0FCF7A6FFEDE70123009307AAFE
:10397000102321463046FBF77FFE04F1080308EED2
:10398000103A07A9E51D002215F9010F8B4611F920
:10399000017BD3B2B842039302D101320028F3D1A4
:1039A0005846F7F7B3FB10F0FF0706D1039B5A1EEA
:1039B000D3B203930BF1FF3B01279DF81700FBF7F0
:1039C000A9FC3D18023501288146EDB215D964687D
:1039D000BAF8022006342C44B4FBF2F102FB114485
:1039E0005CB1A04209D9041BE4B240462246002142
:1039F0000FF0A4F82544A044EDB29DF81720039BD6
:103A000088F800207A1E43EA021288F801205946FD
:103A10003A4608F102000FF069F8B81C31464A46F0
:103A200040440FF063F818EE100A07A90FF020FDCC
:103A300089E700002DE9F04F064689B00F461C4685
:103A4000154642B93C22294618460FF077F8012066
:103A500009B0BDE8F08F5B68934204D93C22002195
:103A600020460FF06BF894F81990B9F1000F1AD0B6
:103A7000D4F804A0A5EB0A08C84528BFC8465FFAD9
:103A800088FBD94508D008F11A01A9EB08022144A6
:103A900004F11A000FF038F8A9EB0B0908EB0A0340
:103AA00084F81990636004F11A086368AB421BD074
:103AB000A5EB030A22466B4639463046FFF70EFF58
:103AC00090B18245D14628BF8146824508D2A0EBFD
:103AD0000A03DAB262760DEB090140460FF006F8F0
:103AE00063684B446360E0E76068431B5842584199
:103AF000AEE700002DE9F04F2DED028B03298BB0CE
:103B00008046894692461D4604D818234B43C61862
:103B100032795AB90EF0D4FF092303604FF0FF3415
:103B200020460BB0BDEC028BBDE8F08F0433C31808
:103B300008EE103AB3691BB10EF0C2FF1623ECE792
:103B4000F3880BB905B1F580F3880BB1AB42F3D123
:103B5000182202FB098213693BB1D2689342C0F07C
:103B6000AB809B1A9D4228BF1D46182303FB098387
:103B7000DB68052B00F2A28046F21B73ADF808301B
:103B8000FCF74CFE3389ADF80C009842D4D9C01A2A
:103B9000738980B2ADF80A001BB1984288BFADF8B6
:103BA0000A30182303FB0983D9687379C1F106042D
:103BB000AC4228BF2C461BB146F21C73ADF808304E
:103BC000E4B202AB2246194450460EF08FFF182390
:103BD00003FB09832D1BDA682244DA60A0D0A244DB
:103BE000182303FB098301275E69DA687068063AC7
:103BF0000023022F06D0316C914203D381424FF053
:103C000002075DD3C3EB031306EB8306736893428D
:103C100008D018EE101A33464046FFF70BFF002875
:103C20003FF47EAF002D3FF47BAF777E2FB3AF42E2
:103C300028BF2F46FBB2009306F11A0319465046DF
:103C40003A4601930EF052FF96F819B0009B9B453F
:103C5000A5EB0705BA4408D0019B07F11A01ABEBAD
:103C60000702314418460EF04FFF009BABEB030BED
:103C7000736886F819B03B44736006F11A0308EEC6
:103C8000903A7DB118EE101A02AB32464046FFF76B
:103C900025FEE8B9182303FB0983DA6819693A4459
:103CA00089B91A61182101FB09883C44D8F80C3005
:103CB0003B44C8F80C3033E7002556E700248FE773
:103CC0000846012395E78A4294BF1A611961E9E722
:103CD000A842834628BFAB46A84208D9401BC2B2BF
:103CE00002AB18EE900A727659190EF0FFFE5A4692
:103CF000504602A90EF0FAFE726802EB0B03A5EB28
:103D00000B05DA445F447360BBE7000010B50C4656
:103D10000922084920460FF0D5FB38B994F909006B
:103D200030B1A0F13F035842584110BD0020FCE7DC
:103D30000120FAE7E4C402082DE9F84F0646894657
:103D40009246FFF7E3FF40B90EF0BAFE022303608C
:103D50004FF0FF352846BDE8F88F0AF0030A4FF010
:103D600000081823321D03FB08F74546D15D0029E2
:103D700070D0032D08F10108F5D10EF0A1FE172334
:103D8000E5E7182303FB086300240122DC60C7E990
:103D900001241C619C61BAF1000F12D01020F9F7C8
:103DA000E1FF18B1C0E9004484608481182303FB5B
:103DB0000863986128B9336841465B683046984784
:103DC00052E048463F210FF045FBDFF8A490DFF8B2
:103DD000A4A00446002CBDD094F90030002BB9D02B
:103DE00004F1010B4946062258460FF06BFB0146D1
:103DF00080B907340A22204610F0B4FA4FF6FE7359
:103E000098421AD83881262120460FF023FB83469A
:103E10005C46DFE75146062258460FF053FB014649
:103E20000028F5D107340A22204610F09BFA4FF6FD
:103E3000FE73984201D87881E5E7182000FB0866F8
:103E4000706908B1F9F79AFF00233B710EF038FE54
:103E500016237CE73744BAF1000F92D17820F9F7A6
:103E600087FF786100288CD10EF02AFE0C236EE7C4
:103E7000F0C40208F7C4020810B51446FFF746FF65
:103E800030B90EF01DFE022303604FF0FF3010BD6D
:103E90005822002120460EF051FEFCF7BFFC0C23F7
:103EA000584320610020F2E72DE9F04F00251570FE
:103EB00093464A699368052B91B040F2C18014681B
:103EC0002068A2880490ADF8142080B246F21B72DC
:103ED000904240F0B580BDF814209A4240F0B08086
:103EE0000D22294607A8063406950EF027FEBDF8D8
:103EF0001220ABB29A4240F2A780277807F00F0653
:103F00003F0940F09D8094F8018008F00F0A4FEAC5
:103F1000181808F101030AEB0309B9F1100F019316
:103F200000F38E80524606A90BA80EF0DFFD019B20
:103F30001A460BABA11C03EB0A000EF0D7FD10AB29
:103F400099440DF12C0E09F8147CBEE80F000DF118
:103F5000180CACE80F00DEF800308CF800300DF1E2
:103F60000E020DF10D010BA88DF80D70FBF748FC4A
:103F700008F103084444804620B9012E2AD10134B7
:103F80000135B4E7BDF80E10FBF7E6FD0028F4D0CC
:103F9000BDF80E309DF80D1013F004031FD11F461D
:103FA0008E4224D1032E22D154F8043BC8F80030AD
:103FB000002211464046FCF785FC002FE0D001238B
:103FC0008BF80030214B1B68986A036864215B689A
:103FD0009847D5E7022E0CBF02340434D0E70129FC
:103FE00002BF98F90070B7FA87F77F09D8E7012E6A
:103FF0000ED1237817B11F1E18BF01275BB200EE48
:10400000103A4046B8EEC00AFBF78CFF0134CFE708
:10401000022E09D134F9023B00EE103AB8EEC00A84
:104020004046FBF77FFFC3E7032E02D154F8043B61
:10403000F2E7042EBCD154F8043B00EE103AEFE74F
:10404000002011B0BDE8F08F0120FAE73010002009
:1040500073B505460E460524013C14F0FF040CD050
:104060000DF1070231462846FFF71EFF18B19DF8F3
:104070000730002BF0D102B070BD0120FBE700003B
:104080000329F8B504460D4604D81821694346189B
:1040900033793BB90EF014FD092303604FF0FF376D
:1040A0003846F8BDB369DBB9002700233371182601
:1040B00006FB0543586908B1F9F760FE06FB0546A3
:1040C00000237361B6692EB1304603F0CFFA304653
:1040D000F9F750FE182101FB05440023A361DFE737
:1040E00004310144FFF7B4FF0028DDD10EF0E8FCF5
:1040F000162303604FF0FF37D7E70000002070471A
:1041000000200021704700000020704708B50EF025
:10411000D7FC1E2303604FF0FF3008BD032938B5DC
:1041200004D80C2404FB0104E56935B90EF0C8FC81
:10413000092303604FF0FF3038BD012B08D0022B5C
:1041400012D063B9002A05DA0EF0BAFC1623F0E7A4
:10415000636A1A44236A9A4294BF626263620C23C0
:1041600003FB0100406AE7E7236A6362F7E70000A8
:1041700008B50EF0A5FC1E2303604FF0FF3008BD0C
:104180002DE9F34112F0030504460F4609D00EF065
:1041900097FC1E2303604FF0FF35284602B0BDE8B0
:1041A000F081011D242201A8F9F770FF2A460C2393
:1041B00004F11C0103FB02F6154651F80680B8F124
:1041C000000F0DD0032D02F10102F3D10EF078FCA7
:1041D000172312E0C4F8248001A8F9F779FFDCE77F
:1041E00006F1200121443846FCF7D6FF3444E06153
:1041F0000028EFD10EF064FC022303604FF0FF357E
:10420000EAE700004868FCF7D1BF00000329F8B5D1
:104210000646104604D80C2202FB0166F76937B93E
:104220000EF04EFC092303604FF0FF30F8BDD6E9D5
:1042300008516C1A9C4228BF1C4634B122463944AE
:104240000EF054FC736A234473622046EEE70000CC
:104250002DE9F341912207460E46011D01A8F9F709
:1042600015FF00234FF4847207F14C0102FB03F8A1
:1042700051F8084044B10133042BF7D10EF020FC73
:1042800017230360002413E007EB08053046A5F868
:1042900050400DF049FDE86450B108F15001394437
:1042A000FCF786FFA5F8504010B108F14C043C44DF
:1042B00001A8F9F70DFF204602B0BDE8F08100002B
:1042C00000F14C032DE9F041CE1A04462048F710C6
:1042D000B6F5467F00FB07F707D90EF0F1FB09237F
:1042E000036000252846BDE8F0814FF4847808FB80
:1042F000074806F15001D8F84C002144FCF758FF5C
:1043000005460028EED0D8F84C00F6F7FFFE08B1BD
:104310000130054452362644FF22294630460FF02C
:10432000E5F82F2128460FF095F84FF4847303FB2E
:10433000074418B984F851013546D3E70123401BDF
:1043400084F851310444002384F85230F4E700BF6C
:10435000E1830F3E70B506460C200D46F9F702FDCD
:10436000044670B1866001462846FCF715FF0546F5
:10437000606030B9204600F08FFA2046F9F7FAFC69
:104380002C46204670BD000000F14C0337B5C91A19
:1043900004461148CD10B1F5467F00FB05F507D95D
:1043A0000EF08EFB092303604FF0FF3003B030BDE9
:1043B000211DDD2201A8F9F769FE4FF4847000FB8E
:1043C00005440025E06C0DF087FCE56401A8F9F7D1
:1043D0007FFE2846EAE700BFE1830F3E13B508469B
:1043E00001A91446FCF728FF38B90EF069FB022337
:1043F00003604FF0FF3002B010BD5822002120466C
:104400000EF09CFB019B23610020F4E7032937B5E4
:1044100004D80C2404FB0104E3693BB90EF050FB03
:10442000092303604FF0FF3003B030BD011D3F2270
:1044300001A8F9F72BFE0025E069FCF7B7FEE5615E
:1044400001A8F9F745FE2846EEE700004FF0FF30DF
:1044500070470000032910B504D80C2404FB0101A7
:10446000087930B90EF02CFB092303604FF0FF30C0
:1044700010BD012B0AD0022B11D02BB9CB689B6841
:104480009342D4BF8B608A608868F1E78B681A44D6
:10449000CB689B689A4294BF8A608B60F4E70EF009
:1044A0000FFB1623E1E7000091F9003010B533B19E
:1044B0000EF006FB022303600024204610BD4FF4DB
:1044C0008270F9F74FFC04460028F6D10EF0F8FA96
:1044D0000C230360F1E70000032970B5064610467F
:1044E00004D80C2202FB0166327932B90EF0E8FAE8
:1044F000092303604FF0FF3070BDD6E902129568C2
:104500006C1A9C4228BF1C461368224619440EF0C0
:10451000EDFAB3682344B3602046EDE738B50B6885
:104520000B2B0C464FF000050CD881F803510D1DE4
:104530000549FF2251F82310284603F003F82368A9
:1045400001332360284638BD68C60208032970B5C8
:1045500004460D4604D80C2303FB01031A7932B933
:104560000EF0AEFA092303604FF0FF3070BDDE6835
:1045700000221A712EB1304603F078F83046F9F770
:10458000F9FB0C2101FB05440020E060EEE7000090
:1045900008B5084631B90EF093FA162303604FF0C0
:1045A000FF3008BDF9F7E6FB0020FAE770B5084ECA
:1045B0000D46002456F8041B2846F6F79DFD08B961
:1045C00060B270BD01340C2CF4D14FF0FF30F8E72D
:1045D00068C602082DE9F74F12F0030405460F469E
:1045E00004D00EF06DFA1E230360E4E00C23021DDC
:1045F00003FB04F9A04612F809A0BAF1000F00F07D
:10460000C280B8F1030F04F10104F1D10EF058FAA1
:104610001723E9E739462846FFF7C8FF00280CDAD8
:10462000304603F023F83046F9F7A4FB0023CAF81C
:104630000C300EF045FA0223D6E760493846F6F70B
:104640005BFD30B95E4B1B68D86A03683146DB6D91
:1046500098475C493846F6F74FFD48B9584B1B68F8
:10466000D86A0C23026803FB0453126ED968904782
:1046700055493846F6F740FD48B9514B1B68D86A92
:104680000C23026803FB0453526ED96890474F49CC
:104690003846F6F731FD48B9494B1B68D86A0C23F8
:1046A000026803FB0453126FD968904748493846A3
:1046B000F6F722FD50B9424B1B68D86B30B10C2382
:1046C000026803FB0453526AD9689047414938464F
:1046D000F6F712FD48B93A4B1B68D86A0C230268FA
:1046E00003FB0453926ED96890473B493846F6F76E
:1046F00003FD98B9324B1B68CDE900005869036887
:1047000001AA9B696946984740B10C20019B00991A
:1047100000FB04501A46C06802F0B2FF2F49384629
:10472000F6F7EAFC50B90C2000FB04504FF480234C
:10473000C0681A464FF0006102F0A2FF0C2606FB8B
:104740000456F3689A68AAB91B7B002B14BF0C2788
:1047500002270EF0B5F90760F6682EB1304602F078
:1047600085FF3046F9F706FB0C2000FB04540023BC
:10477000E36020E04D440023AB6001232B714046F1
:1047800003B0BDE8F08F1020F9F7ECFA064628B127
:10479000C6E900AAC6F808A0A6F80CA04FF00C0BBA
:1047A0000BFB045ACAF80C60002E7FF433AF0EF0F6
:1047B00087F9C0F800B04FF0FF38E0E7C8C502083D
:1047C00030100020D4C50208DCC50208E7C5020885
:1047D000F2C5020801C6020811C602081DC6020879
:1047E00070B5064615460C4619B112B191F9003064
:1047F00033B90EF065F9162303604FF0FF3070BD3A
:104800005822002128460EF099F92046F6F77EFC42
:10481000012894F9003003D12F2B04D10020EEE7BA
:104820002F2B08BF013421463046FFF7BFFE00287A
:1048300003DA0EF045F90223DEE706492046F6F7D3
:104840005BFC18B94FF448732B61D8E7024B2B611E
:10485000E4E700BF11C60208A08601004FF0FF3058
:10486000704700004FF0FF30704700004FF0FF30FE
:10487000704700004FF0FF30704700004FF0FF30EE
:1048800070470000486810B50C4618B10DF024FAC6
:104890000023636010BD000010B50446806818B1A5
:1048A000036821469B6D9847204610BD2DE9F043D3
:1048B000036899B09B6902AA05468846984707464F
:1048C00020B10024204619B0BDE8F0830C20F9F790
:1048D00049FA04460028F4D08560069801300DF0AE
:1048E000B3F9064630B92046FFF7D6FF2046F9F760
:1048F00041FAE6E72B684146D3F800903A463B463A
:104900002846C847431C014603D130460DF0E4F960
:10491000E9E72B680190D3F80880069B32462846C9
:10492000C047069B019998422B6828465B6801D0D6
:104930009847EAE79847069BC4E90036C2E70000BB
:1049400030B1044B1B6830EA03030CBF0120002088
:10495000704700BFA02F002010B5044600F070FF84
:104960004FF46B43A4F8303220460549FBF75AFE5A
:10497000044B1C60FF2384F89832204610BD00BF12
:10498000D0CB0208F03B002007B543682BB10844A8
:1049900090F87A0203B05DF804FB07298DF8073020
:1049A00008D82131C8B20DF10701FCF76FFF9DF85F
:1049B0000700EFE70B2901D84A31F3E701F1940032
:1049C000F1E7000070B50A4400204AF201068A426D
:1049D00014D011F8014B082384EA000515F0010FEB
:1049E0004FEA500018BF704003F1FF3318BF80B288
:1049F00013F0FF034FEA5404EED1E8E770BD000066
:104A000090F82E228118002381F8FE3102F18201F4
:104A100000EB810100EB82008B7180F80F32704750
:104A20002DE9F347154690F82E3290F840229A422D
:104A3000044689465FD903444FF47A7101A893F87C
:104A4000FE81F9F709FB2D4B1E68B06A03686421EB
:104A50009B689847776A94F82E123B682046D3F8F3
:104A60006CA0FFF791FFD4F8843201464FF49642D0
:104A70003846D04750B90F2384F82F32002501A8BB
:104A8000F9F7F6FA284602B0BDE8F087B06A036885
:104A900064219B689847D4F86C321BB902F04EFD34
:104AA000C4F86C0204F1F0072A46494638460EF075
:104AB0001DF82A4649462046FFF784FF6319B8F1DE
:104AC000000F83F8F0004FEA102083F8F100706ABD
:104AD00018BF0222036808BF00222A441B6F92B24B
:104AE0003946984705460028C5D0B06A03681A21A0
:104AF0009B689847C3E70025C4E700BF301000203B
:104B00002DE9F34790F82E320344044693F8FEA1B2
:104B1000BAF1000F14BF03260126884601A84FF4FE
:104B20007A7116441546F9F797FA344B1B68586AA0
:104B30000368B6B2D3F8749004F1F0074FF47A73B7
:104B4000734332463946C84794F916308146002BE4
:104B500038D003462A492A460620F7F7BDFF4E45BE
:104B600032D094F916301BB126490620F7F7B4FF6E
:104B70000F2384F82F32002401A8F9F779FA204690
:104B800002B0BDE8F08796F8F220302A12D094F9EE
:104B90001630002BECD01C490620F7F79DFFE7E705
:104BA00096F8F020302A05D094F91630002BDFD08B
:104BB0001649F1E725B12A46394640460DF096FFE1
:104BC0000124D9E78642D3D16619BAF1000FE7D0A4
:104BD0002A4639462046FFF7F5FE96F8F020C3B284
:104BE0009A4205D196F8F120C0F30F239A42CAD019
:104BF00094F91630002BBBD00549B6E730100020E1
:104C000060C7020879C7020896C70208AAC7020847
:104C100089C7020837B501A80C46F9F71DFA0B4BF6
:104C20001B68586A03685D6F4FF47A73634301220F
:104C30000DF10701A847012801A80CBF9DF8074006
:104C4000FF24F9F715FA204603B030BD30100020DC
:104C500013B5B0F8EA204FF6FF739A42044624D009
:104C600090F916301BB112490620F7F735FF0023E3
:104C70008DF80530FF238DF80430B4F8EA308DF854
:104C800007301A0A8DF8062004220DEB0201204697
:104C9000FFF7C6FE38B102212046FFF7BBFFA0F1A7
:104CA00030035842584102B010BD0120FBE700BF5D
:104CB000C0C702082DE9F04188B006468846144670
:104CC0001F46FFF7C5FF054678B1B7F5807F14BFD3
:104CD0003B460023022207A930468DF81C808DF840
:104CE0001D30FFF79DFE20B90025284608B0BDE81D
:104CF000F0813A4621463046FFF702FF054600287C
:104D0000F2D0102FF1D1B6F8EA20B6F830329A423C
:104D1000EBD196F91630002BE7D0E3680493A37823
:104D200003936378029323780193A3680093E27856
:104D3000636802490620F7F7CFFED6E7E4C702080A
:104D4000F0B590F916308FB004467BB190F82E2262
:104D500090F84032039311460292FFF715FEDDE909
:104D6000022300905B490620F7F7B6FE2046FFF7C6
:104D700047FE594B08AA03F11007164618685968F0
:104D8000154603C50833BB422A46F7D118681B797C
:104D900028602B71152231462046FFF741FE18B9D5
:104DA000002528460FB0F0BD082205A92046FFF7D0
:104DB000A7FE05460028F3D04849032205A80EF0B7
:104DC00081FB064618B10F2384F82F32E8E794F8E8
:104DD0002E329DF817109DF8190004EB830282F81B
:104DE00010129DF8181082F80F1203F1820204EBE2
:104DF00082022344907183F80662D28894F9167077
:104E00004EF6B206B24240D84EF6B006B24247D88D
:104E100049F20F36B24227D849F20636B24227D9B4
:104E200002F5D94679364FF0010CB6B20CFA06F607
:104E300040F2091C16EA0C0F1AD0022283F806224F
:104E40001FB127490620F7F747FE94F82E022318D2
:104E500004EB800493F8062284F81122002AA0D0E3
:104E6000012283F8FE219CE749F20B46B242E4D0CE
:104E70000139C9B28E2922D8062820D1042283F80C
:104E80000622002FE1D01749DDE74FF29036B242FB
:104E900006D00CD822F020064FF2103C6645E7D130
:104EA000012283F80622002FCFD00F49CAE74FF224
:104EB0001046B242F4D04FF65006B242EFE70F234D
:104EC00084F82F32002FC0D008490620F7F704FEDF
:104ED000BBE700BF10C80208DC6C02082EC802083D
:104EE00032C802086EC8020850C802088CC80208FE
:104EF00007B50023ADF8043090F82E3200EB8303A1
:104F0000012283F80E2201A90222FFF789FD03B0D6
:104F10005DF804FB10B5064B1B680446586AD4F8CC
:104F2000841203689B6F98470023C4F86C3210BD4D
:104F3000301000202DE9F041C6B004460D464FF078
:104F4000000806A911308DF81880FBF729FE424BA6
:104F50001B689B69C4F8383294F84032AB4207D8DA
:104F60003E492A46062046B0BDE8F041F7F7B4BDF9
:104F700094F82E723A4984F82E522A460620F7F702
:104F8000ABFD052640F6B83101A8F9F765F82046D3
:104F900084F82F82FFF734FD2046FFF7D1FE054647
:104FA000002850D094F82E32234406AA93F80632F3
:104FB000022B14BF4FF4F8430023A4F8EA3018BFC3
:104FC00003214FF4807308BF07212046FFF772FECC
:104FD00094F82E322344054693F80632042B01D16F
:104FE00000BB00252046FFF783FF01A8F9F740F832
:104FF0002046FFF78FFF1B4BD4F874221A601A4B20
:105000001A4A1B4984F82E72002684F87062B54251
:1050100008BF1A460620F7F75FFDC4F8386246B0AD
:10502000BDE8F081B4F83032A4F8EA302046FFF74A
:105030000FFE0028D5D0102302AA03212046FFF737
:1050400039FE0546CEE701A8013EF9F711F816F042
:10505000FF0697D1CCE700BF30100020BEC8020881
:10506000D2C80208A82F0020B7C80208B0C802089A
:10507000F2C802082DE9F0470026DFF83091044617
:1050800035464FF0010A40F2DC5894F84022F3B262
:105090009A4216D92344013693F87A12A3680AFA81
:1050A00001F71F40D9F80030586A03689B6B984796
:1050B000002F14BF43464FF47A73984218BF01255E
:1050C000E3E702F03BFA94F86432002B68D094F8DE
:1050D0007832002B59D0B4F9123043B1D4F8682299
:1050E0004FF47A71821A13FB01F39A4207D8002D0C
:1050F0004BD0D4F86832C01AB0F57A7F45D9D4F8CD
:105100006C3213B12046FFF705FF94F8703233B1CB
:10511000002384F87032234BD4F874221A60D4F838
:1051200034327BB194F916301BB11F490620F7F7D2
:10513000D3FC0022D4F834021146F9F75DF80023BD
:1051400084F87832F5B1DFF864800025012740F259
:10515000DC5694F84022EBB29A4213D92344A26859
:1051600093F87A12D8F80030586A07FA01FC0368FD
:105170001CEA020F5B6914BF32464FF47A729847FB
:105180000135E6E794F8643253B194F9111000291F
:1051900006DD01392046C9B2BDE8F047FFF7CABEB7
:1051A000BDE8F087A82F0020A4C902083010002015
:1051B000F7B50123044680F864320D4600230DF153
:1051C0000701113016468DF80730FBF7E9FC6168DE
:1051D00094F917200D4326B992B2072A9CBF0132D9
:1051E000D6B2384B1F68B31E062B0DD875B1786A3E
:1051F00003683246D3F8803029469847304602F09B
:105200001DFB18B12E4602E0002DF7D10026A16843
:1052100030463140FCF7D2F9786A2B4B1A680368A4
:1052200092F85913D3F8AC309847786AA1680368AC
:1052300031409B699847786AE16803683140DB69CF
:1052400098470023012194F84022072ADFB226D98B
:1052500094F91630C4F8845233B194F840221B49B3
:1052600033460620F7F738FCA36835EA030226D058
:10527000003B18BF012384F8793294F8403263B1BF
:10528000B4F91430002B08DD114B186828B1002246
:105290001021FBF745FEC4F83C0203B0F0BD01FA53
:1052A00003F0304218BFA01803F101031EBF013202
:1052B00080F87A7284F84022102BC4D1C8E700230A
:1052C000D9E700BF30100020982F002038CB02080B
:1052D000842F00202DE9F04F2DED048B0546D0F8EA
:1052E0003C0203689BB05B6A0A220EA99847092812
:1052F0001BDD0EAC4FF0090A002114F8010B072248
:1053000002F098FD0AF1FF3A1AF0FF0A0146F4D1C3
:105310009DF8413083420DD095F916302BB195F8A8
:1053200090225F490620F7F7D7FB1BB0BDEC048B3A
:10533000BDE8F08F95F89032BDF83F4095F919001F
:105340002B4464BA93F87A72564BD3F80080A4B217
:10535000C826744394FBF0F4D8F8240003684FF097
:105360000109D3F89C3009FA07F1A4B2984707EE77
:10537000904ADFED4D0AB8EE670A3946284600F03C
:105380006DFA2422514611A80DF0D8FB9DF8383053
:10539000DFED466A03EB830303EB83039B00ADF869
:1053A0004430BDF839305BBA9BB207EE103ABDF815
:1053B0003B305BBA9BB207EE903ABDF83D30F8EE59
:1053C000677A5BBA67EEA67A9BB2CDED137AB8EE38
:1053D000477A07EE903A27EE267AF8EE677A1D2391
:1053E00011AA394628468DED127ACDED147A00F0D7
:1053F00039FA95F916304B4597DD95F890322B44E4
:1054000093F87A3209FA03F9EB6919EA030F10D01D
:10541000D8F82400036839465B6D98474FF6FF7350
:10542000984204461FBF744395F9196094FBF6F443
:10543000A4B2D8F8186095F8902233681298D3F87F
:105440000090BDF944300D920C93F5F737F8824681
:1054500013988B46F5F732F841EC180B1498F5F7D2
:105460002DF841EC190BD8F8240001688D6D3946F0
:10547000A84710EE105A02F061F80A902846F5F796
:105480001DF88DED049BCDE908018DED028BCDE972
:1054900000ABDDE90C32064906943046C84744E7C4
:1054A0005CCB020830100020000000000AD7233C2B
:1054B0006FCB02082DE9F743D0F83C32044673B3B2
:1054C0003E4B1B685BB302F031F894F89132B4F9AB
:1054D000147094F84052064643B9D4F83C024FF495
:1054E000E131F8F785FE012384F89132D4F83C02CB
:1054F00003685B6998470A2807D9D4F83C02036817
:105500001B6A03B0BDE8F0431847431E082B0CD8B4
:10551000D4F8940230B1301AB0F57A7FEDD203B0EE
:10552000BDE8F083C4F89462F9E70A2805D1204663
:10553000FFF7D0FE0023C4F89432D4F88C22204B1D
:1055400015FB07F5B3FBF5F3B3F5FA6FA6EB020213
:1055500038BF4FF4FA639A42E1D394F8908294F8FA
:10556000407208F10105B5FBF7F307FB1355EDB2E7
:105570004FF00109631993F87A1209FA01F108460C
:105580000191FFF7DDF94545019908D048B901358A
:10559000EDB2B5FBF7F307FB1355EDB2EAE70028D0
:1055A000BDD0084B1B68586A0368D3F894309847FD
:1055B00084F89052C4F88C62B1E700BFA02F00209D
:1055C00040420F003010002010B5064B1A68044608
:1055D00012B1054801F084FF04491860FBF722F876
:1055E000204610BDF43B002080CC0208ACCC020861
:1055F0002DE9F0470024054600F1D80726464FF074
:1056000024094FF0010A4FF0180809FB0453D3F89E
:10561000F0301BB908FB0453DB6853B1384600F087
:1056200025F918B108FB04531B7D13B10AFA04F3E2
:105630001E430134092C07F12407E6D13046BDE8AA
:10564000F0870000082909D8182303FB01010B7D0E
:1056500003F0FF001BB10B68136070470020704718
:105660000829F8B504460D46164601D90020F8BDB4
:10567000242707FB0100D830412100F001F9002860
:10568000F4D007FB0544B4F8D8303380EFE70000CE
:105690000829F8B504460D46164601D90020F8BD84
:1056A000242707FB0100D830822100F0E9F8002808
:1056B000F4D007FB0544B4F8EC303380EFE700008A
:1056C0000829F8B504460D46164601D90020F8BD54
:1056D000242707FB0100D830082100F0D1F800286A
:1056E000F4D007FB0544D4F8E0303360EFE7000066
:1056F0000829F8B504460D46164601D90020F8BD24
:10570000242707FB0100D830042100F0B9F8002855
:10571000F4D007FB0544D4F8DC303360EFE7000039
:10572000082970B54DD8002B4BD00124DE0780F836
:10573000654241BF242404FB0104B2F90060A4F8CF
:10574000D86003F0020535B1242404FB0104B2F94A
:105750001450A4F8EC505C0741BF242404FB01045E
:105760005568C4F8DC501E0741BF242404FB010423
:105770009568C4F8E050DD0641BF242404FB010411
:10578000D568C4F8E4509C0641BF1469242202FB8A
:105790000102C2F8E840242404FB0104B4F8F62016
:1057A000013292B2A4F8F620B4F8F42092B2134376
:1057B000A4F8F43001F0C2FE0123C4F8F00084F82C
:1057C000F83070BD2DE9F04108292DED028B04461B
:1057D0000D46F0EE408AB0EE608A29D84FF00108FD
:1057E00080F8658201F0A2FE182606FB05464045BA
:1057F00005EB450538BF404604EBC5040746F06895
:10580000236863600C4AC4ED008A6421381AF9F7F2
:105810008BFA07EE900ADFED096AF8EE677A86EEFA
:10582000A77A86ED047AF76086ED028A86F81480FE
:10583000BDEC028BBDE8F08180969800002474498D
:1058400008B5044B1B68036013B9034801F048FE18
:1058500008BD00BFF43B0020CCCC02080068FFF775
:10586000B1BF00000068FFF75BBF0000836923B190
:1058700090F8200080F00100704701207047000080
:1058800008B5838B194005D0FFF7F0FF80F00100C9
:10589000C0B208BD0846FCE710B4064B064A1B68B8
:1058A0000649986903681C68537E127EA4465DF819
:1058B000044B604730100020D0A10008DCCC020867
:1058C00070B50446054600F124062846063502F068
:1058D000B9FDAE42F9D120460349FAF7A3FE034BC6
:1058E0001C60204670BD00BFF4CC0208F83B0020CD
:1058F0007FB50D4A0346106892880290ADF80C20DF
:1059000002AE9D1C03F1260416F9013B5A1C06D079
:105910000DF106012846ADF80630FBF779F906359A
:10592000A542F1D104B070BDECCC020813B500293A
:1059300012DB0A4B1C68E0690368C9B25B6801911D
:1059400001229847E06901990368DB6898470038AD
:1059500018BF012002B010BD0020FBE7301000206E
:1059600037B50029144611DB094B1D68E869036847
:10597000C9B201915B6801229847E86901990368FF
:105980001B69224603B0BDE83040184703B030BD64
:105990003010002073B501EB410100EB41040646D5
:1059A000B4F902104B1C154612D00191FFF7BEFF4F
:1059B00094F905300199002BC8BF85F00105854297
:1059C00006D02A46304602B0BDE87040FFF7C8BF97
:1059D00002B070BD4B1E182B2DE9F04105460E4656
:1059E00090460ED80024062707FB04F3E1B2EB5CD7
:1059F000B34203D142462846FFF7CCFF0134062CC0
:105A0000F2D1BDE8F081000070B50546FFF770FFE8
:105A10002C460026B4F902300133F1B215D02278B9
:105A2000531E182B11D8A2F10A030F2B03D9531EB2
:105A30005A425A4132B1237994F90420012B04D8F7
:105A400002F001022846FFF7A5FF0136062E04F1F9
:105A50000604DFD170BD0000002070470E207047A3
:105A600000F5805090F8F000C0F34000704700004F
:105A700000F588507047000000F5805090F9F8005C
:105A80007047000000F58050C0F8F4100120704706
:105A90002DE9F3470C68BDF8288014F00054074640
:105AA0000D4696469C4640F08F800E7B082E00F2F5
:105AB0008B8000F58059D9F800610136C9F8006182
:105AC000302686F31188C66BD6F808A01AF0806FCE
:105AD00017D1B468240113D4B46814F080546FD182
:105AE000D9F808510135C9F80851D9F80C51002DE1
:105AF00068D1CDF80080F8F7CDF984F311885CE027
:105B000001242B6804F11802002B4FEA0212BABFDD
:105B1000DB0043F004035B05B3502B6813F0804FA8
:105B200023B218BF06EB031106EB03131EBFD1F817
:105B3000802142F00202C1F880212A7BC3F884212F
:105B400006EB0416AA68C6F88C216A68C6F8882194
:105B5000D3F8802142F00102C3F8802141F2900184
:105B600007EB44120A4401EB44113944C2E900EC4A
:105B700063012A46083105F10C0052F8044B41F844
:105B8000044B8242F9D13B4412880A8003F58053CA
:105B900008F0030293F8AC1021F00B010A4383F8DC
:105BA000AC20002383F31188CDF800807246634651
:105BB00029463846F8F76EF9012002B0BDE8F087B3
:105BC00002249EE7204698E74FF0FF30F5E70000FB
:105BD0002DE9F04F90F83830032B40F098800E2AD2
:105BE00000F29580002900F09480302383F311881F
:105BF000C46BD4F8003243F00103C4F80032C46B24
:105C0000D4F8003223F47C53C4F80032C46BD4F8C7
:105C1000003243F46063C4F80032C36B3E4CC3F8F7
:105C20001442C46B0023C4F80432C46B6FF078458F
:105C3000C4F80C5200F5805494F8F8509D4218BFF7
:105C40000E25DAB9C36B05F1480143F83120C36B67
:105C500003EBC1035A60C26B012303FA05F5C2F8D6
:105C60001C52C26BD2F8003223F00103C2F800329A
:105C7000002383F311880120BDE8F08F4FF0010865
:105C800001F10409EF189A42D0F83CA008FA07FE87
:105C900036DD51F833B059F833C0BBF1000F02DBE9
:105CA000BCF1000F27DB4FEACB044FEACC0644F0EF
:105CB00004041BF0804F07F1480718BF44F00204AA
:105CC0004AF83740C46BBCF1000FB8BF46F0040679
:105CD00004EBC7041CF0804F18BF46F00206666054
:105CE000C66BD6F81C424EEA0404C6F81C420133C7
:105CF0000E2BC7D1B5E74FEA4B544FEA4C56D8E7C5
:105D0000DAF81C4224EA0E04CAF81C42EFE700202D
:105D1000B2E70846B0E700BFAAAAAA0A13B500F581
:105D200080540191D4F8840001F030FE1F280BD973
:105D30000199D4F88400202201F0ACFEA0F12003E8
:105D40005842584102B010BD0020FBE708B530238F
:105D500083F3118800F58050D0F8840001F0EAFD4B
:105D6000002383F3118808BD002202608281426013
:105D70008260704710B500220023C0E90023002391
:105D8000044603810C30FFF7EFFF204610BD0000F2
:105D90002DE9F04300F580570D4697F8F03013F0E9
:105DA000040FC3F3800108BF114661F3820387F833
:105DB000F03000EB451303F58553083389B01B79A8
:105DC000D907DDE9108904464FEA45163BD5002A7C
:105DD0003BD0180739D404EB45156846FFF7CAFFD6
:105DE00005F58453183303AA05F5855518685968D5
:105DF0009446ACE803000833AB426246F6D118681B
:105E0000CCF800009B88ACF804300123ADF80830D2
:105E10002368CDE900899B6C694620469847A31901
:105E200003F5855308331A7911070ED442F008029E
:105E30001A71D7F80C3104F589540133C7F80C31C5
:105E4000C4E9028901E0002AE9D109B0BDE8F08384
:105E50002DE9F0479A4688B0074688469146302398
:105E600083F3118807F580546846FFF783FFD4F861
:105E7000840001F071FD1F282BD9D4F88400202262
:105E8000694601F089FE202823D103AD444605ABC5
:105E90002E4603CE9E4220606160354604F1080420
:105EA000F6D130682060B388A380DDE90023C9E91A
:105EB0000023BDF80830AAF80030002383F31188CE
:105EC00053464A464146384608B0BDE8F047F7F722
:105ED00089BF002080F3118808B0BDE8F08700007A
:105EE0002DE9F84F2B4B044640F8043B0F4600F0D9
:105EF000B7FC1822002104F11C000CF01FFE204604
:105F0000254B40F8403BFFF72FFF04F15000FFF70F
:105F100031FF04F1700804F58355464610353046CC
:105F20002036FFF727FFAE42F9D104F580554FF434
:105F300080534FF00009C5E91D39C5F87080012371
:105F4000C5F8846004F5885804F58556C5F87C903A
:105F500085F8803085F88830103608F110084FF049
:105F6000000A4FF0000B46E908ABA6F11800FFF756
:105F7000FBFE203646F8289C4645F4D185F8F8709B
:105F800017B1064801F0ACFA054BE3632046BDE8C3
:105F9000F88F00BF847102088CCD020864CD02081E
:105FA0000064004010B5044B197804464A1C1A706E
:105FB000FFF796FF204610BD003C00202DE9F0477A
:105FC000002950D0294B2A4FB7FBF1F599428CBFDD
:105FD0000A231123581EB5FBF3FC03FB1C53C4B268
:105FE0002BB102280346F5D80020BDE8F0870CF15C
:105FF000FF36B6F5806FF7D2C4EBC40E0EF1030383
:106000004FEAE309C3F3C703A4EB030809F1010A4C
:106010004FF47A755FFA88F009FB05555AFA88F84B
:10602000B5FBF8F5B5F5617FC1BF0EF1FF33C3F3E2
:10603000C703E01AC0B25C1C50FA84F40CFB04F4F1
:10604000B7FBF4F4A142CFD1013BDBB20F2BCBD88D
:106050000138C0B20728C7D800211071168091708E
:10606000D3700120C1E70846BFE700BF3F420F00E1
:1060700000B4C40470B505460E464FF47A74EB6B59
:106080005B6803F00103B34207D04FF47A700BF062
:10609000B3FA013CF3D1204670BD0120FCE70000BB
:1060A000F0B5C26B936913F0700F1ED000230F4E32
:1060B000936141F2A80500F5805400EB43122A4495
:1060C00011794F070ED589070CD5C16B56F823708F
:1060D0008F60117941F004011171D4F8142101325B
:1060E000C4F814210133032BE7D1F0BD78CD0208A9
:1060F00073B51D46C36B16469A68D207044609D588
:106100009A6801219960C2F34002CDE9006500213F
:10611000FFF73EFEE36B9A68D1050BD59A684FF402
:1061200080719960C2F34022CDE9006501212046CB
:10613000FFF72EFEE36B9A68D2030BD59A684FF4F3
:1061400080319960C2F34042CDE9006502212046CA
:10615000FFF71EFE04F58053D3F8F40038B1D3F8EE
:1061600030210132C3F8302103681B69984720466B
:1061700002B0BDE87040FFF793BF0000F8B50446D9
:10618000C66B002940F08D8006F10C073868850742
:1061900000F090803868C00641BF04F58055D5F8FE
:1061A00020010130C5F8200106EB011506EB0111B5
:1061B000D5F8B00110F0040FD5F8B0011ABFC0082F
:1061C00040F00040400D2064D5F8B0C11CF0020F33
:1061D0001CBF40F080402064D5F8B40100F00F00EF
:1061E00084F84C00D1F8B80184F84400D1F8B80123
:1061F000000A84F84500D1F8B801000C84F8460084
:10620000D1F8B801000E84F84700D1F8BC0184F839
:106210004800D1F8BC01000A84F84900D1F8BC015B
:10622000000C84F84A00D1F8BC11090E84F84B1018
:106230003821396004F15C0004F1400104F14C059F
:1062400051F8046B40F8046BA942F9D10988018028
:10625000C4E9142321460023A4F8583051F8503BD8
:1062600020469B6C984704F58053E8B1D3F8182179
:106270000132C3F8182193F8F020D3F8F40042F06B
:10628000040283F8F02038B1D3F830210132C3F88A
:10629000302103681B6998472046BDE8F840FFF7A6
:1062A000FFBE06F1100771E7D3F81C210132C3F8D5
:1062B0001C21E0E7F8BD000010B5044601F040F9EC
:1062C00002460B4652EA030102D0013A63F1000391
:1062D0000449086820B12146BDE81040FFF74EBFD1
:1062E00010BD00BFFC3B00202DE9F041302181F3BF
:1062F0001188DFF85C8000F584511031002441F2F0
:10630000A80E00F5805C00EB441575442E797707E4
:1063100013D4F60611D5D1E9007697429E410CD2EE
:10632000C66B58F82470B7602E7946F004062E71BB
:10633000DCF810510135CCF810510134032C01F177
:106340002001E0D1002383F31188BDE8F08100BF74
:1063500078CD020808B5302383F31188FFF7A0FE3B
:10636000002383F3118808BD2DE9F041C36B054676
:10637000986800F0E050B0F1E05F0F4623D000B322
:10638000302383F3118805F584541834002641F234
:10639000A80805EB461343441B791A0706D50136B6
:1063A000032E04F12004F4D1012007E05B07F6D4AA
:1063B00021463846F7F7CAFD0028F0D1002383F3C1
:1063C0001188BDE8F0810120FBE7000008B530230B
:1063D00083F3118800F58050D0F8840001F0BCFAF6
:1063E000002383F3118843090CBF0120002008BD5E
:1063F000F8B51D46002313700F4606461446FFF7F6
:10640000E5FF80F00100387025B129463046FFF7DE
:10641000ABFF2070F8BD00002DE9B8410C461546D1
:106420001F46804601F08CF80B462178024609B9D8
:10643000287850B14046FFF757FFFFF78BFF3B46E8
:106440002A462146FFF7D4FF0120BDE8B8810000AD
:1064500070B5302686F31188174B9A6D42F00072A2
:106460009A659A6B42F000729A639A6B22F00072FE
:106470009A63002383F3118800F5805494F8F03078
:1064800013F0010516D1A9B186F311880321132059
:106490000AF0BAF8032114200AF0B6F803211520F7
:1064A0000AF0B2F894F8F03043F0010384F8F030C9
:1064B00085F3118870BD00BF001002402DE9F04740
:1064C00000F5805588B095F8F830012B04468846D1
:1064D000164600F28A80864F57F8232042B947F8C3
:1064E000230000F0A9FC95F8F83000EB8300C463AA
:1064F000D7F800A0C4F8348084F83860BAF1000FEF
:1065000065D095F8F830012B71D001212046FFF7B6
:106510009FFF302383F31188E26B136823F002039B
:106520001360E26B136843F001031360E36B002711
:106530005F6187F3118801212046FFF79BFD00284A
:1065400000F09680D5F8840001F0F4F904F5845940
:10655000BA4609F110092022002168460CF0EEFA33
:1065600002A8FFF701FCCDF818A06A4609EB070363
:106570000DF1180E9446BCE80300F445186059600C
:10658000624603F10803F5D1DCF8000018602037FB
:106590009CF804201A71602FDDD195F8F0306FF36C
:1065A0008203002785F8F0306A4641462046ADF860
:1065B0000070ADF802708DF80470FFF7FFFCE36B1C
:1065C00048BB4FF400421A6008B0BDE8F08741F2C2
:1065D0003810F7F7C7FB814610B15146FFF780FC32
:1065E000C7F80090B9F1000F8BD10020ECE73868B4
:1065F00003689B6B98470146002886D13868FFF7EF
:1066000027FF3868036832465B6841469847002890
:106610007FF47BAFE9E761221A609DF802309DF8B4
:1066200003201B06120402F4702203F0407313438C
:10663000BDF80020C2F3090213439DF8042012059F
:10664000022E02F4E0020CBF4FF000410021134380
:10665000E26B0B43D361E36B13225A61E26B136865
:1066600023F00103136039462046FFF703FD08B904
:10667000E36BA6E795F8F83093BBE16BD1F8002205
:1066800042F00102C1F80022E16BD1F8002222F4AD
:106690007C5222F00E02C1F80022E16BD1F80022F8
:1066A00042F46062C1F80022E26BC2F81432E26B7D
:1066B000C2F80432E26B41F6FF71C2F80C12E26BD1
:1066C000C2F84032E26BC2F84432E36B0122C3F8F5
:1066D0001C22E26BD2F8003223F00103C2F8003230
:1066E00095F8F03043F0020385F8F0306CE700BF16
:1066F000FC3B002008B500F023FF50EA01030246EE
:1067000002D0421E61F10001044B186810B10B4623
:10671000FFF7EEFCBDE8084008F032BCFC3B00206F
:1067200008B50020FFF7C8FDBDE8084008F028BC08
:1067300008B50120FFF7C0FDBDE8084008F020BC07
:10674000036800211B681847036800211B6818476D
:106750007047000008B504300AF096FC012008BD1F
:1067600004300AF087BC000008B504300AF0E6FDEA
:10677000B0FA80F0400908BD08B5302383F31188D2
:10678000C368002B02DC04300AF00AFE0AF0AEFDFA
:10679000002383F3118808BD10B50446F7F7EAFA21
:1067A000204610BD2DE9F84306460D4621B90430B8
:1067B0000AF03EFC012424E003685B689847002847
:1067C000F8D100F0BDFE104B8846D3F800904FF48E
:1067D0007A7107464D43D9F828000368C8219B68A1
:1067E0009847336830465B68984704460028E1D1F3
:1067F00000F0A6FEC01B61EB0801A84271F1000386
:10680000E9D32046BDE8F88330100020F8B5051D17
:106810000C4671B14EF66027BC42264628BF3E4664
:10682000B1B228460AF0B2FD50B1A41BF4D1204603
:1068300005E028460AF0AAFDB0FA80F04009F8BD4C
:106840000120FCE708B5302383F31188C368002BCF
:1068500002DC04300AF0A4FD002383F3118808BD94
:1068600010B5044B044640F8043B0AF09FFB204659
:1068700010BD00BF04CE0208034BC068DB68C31A1A
:1068800058425841704700BF7079002010B5044B42
:10689000044640F8043B0AF035FD204610BD00BF19
:1068A000E0CD02080CB430B585B008AC0A46074903
:1068B00054F8043B0D6800940146E86A0394F7F726
:1068C00017FD05B0BDE8304002B070473010002021
:1068D00013B5054C0093246813460A460146E06A46
:1068E000F7F706FD02B010BD301000202DE9F3418E
:1068F000134601920E460A46002107460846FFF756
:10690000E7FF041E019B05DC4FF0FF34204602B078
:10691000BDE8F08104F101080121404601930BF02C
:10692000D7F905460028EFD0019B32464146FFF7D4
:10693000CFFF3D60EAE700000EB403B503AA52F8AA
:10694000041B0192FFF7D2FF02B05DF804EB03B025
:10695000704700000A460146014808F05FBB00BFCF
:10696000887000200FB407B5054B04A91B6851F8C7
:10697000040B0191984703B05DF804EB04B0704735
:10698000140E00207047000013B5046800922469BB
:106990000B46A04702B010BD7047000000207047B2
:1069A0000020704713B56C4684E8060000F114031C
:1069B00094E8030083E8050002B010BD0020704792
:1069C00013B56C4684E8060000F10C0394E803005C
:1069D00083E8050002B010BD0023C0E9033370470F
:1069E00082B002AB03E9060002B0704770470000B6
:1069F000002070477047000013B5046800922469B6
:106A00000B46A04702B010BD002070470020704721
:106A100070470000002070470020704782B002A934
:106A200001E90C0002B07047704700000020704779
:106A30007047000070470000012070470120704738
:106A4000012070472830704782B002A9002001E978
:106A50000C0002B070470000704700007047000053
:106A60007047000008460AF0FFBF000008460BF020
:106A7000C5B8000073B51E460C461546011D102210
:106A800001A8F7F703FB3246294620460BF036F8FB
:106A9000044601A8F7F71CFB204602B070BD0000B9
:106AA00013B50D220C46011D01A8F7F7EFFA204699
:106AB0000AF0ECFF044601A8F7F70AFB204602B0F3
:106AC00010BD00000AF0CEBF08460AF0C7BF0000A4
:106AD00008460AF0BBBF000010B5064B044640F85C
:106AE000843B00F0E9FE04F1700000F0E5FE204672
:106AF00010BD00BFD0D7020808B53020F7F732F933
:106B000070B10023C0E90333C0E905330371037A90
:106B1000022262F302030372024B0360024B8362A0
:106B200008BD00BFACCE0208B8D1020810B4BDF851
:106B3000044001945DF8044B00F0E4BB10B4BDF8D0
:106B4000044001945DF8044B00F08ABB00F0A0BB48
:106B500000F0CEBB38B5084B036090F80431044612
:106B600043B9D0F800512DB1284600F0A5FE2846C3
:106B7000F7F700F9204638BDE8D4020810B5044BF9
:106B800003600446406A08B1F7F7F8F8204610BDE4
:106B900030CE020810B50446FFF7F0FF2046F7F7A5
:106BA000E9F8204610BD000010B51C4B0360002121
:106BB00090B004460171102200F54A700BF0BEFF40
:106BC00004F54E70FFF74CFE12200AF047FF144BFD
:106BD0000A94CDE90B34134BCDE90D34124B0F93CE
:106BE00010A9024611E9030005AB83E80300DDE9C3
:106BF0000C0103AB83E80300DDE90A0101AB83E884
:106C000003000A4B009304F10801234604F5597070
:106C100001F020F9204610B010BD00BFECCF0208F3
:106C20003D6B01084D6B0108516B01082D6B01088C
:106C30001B4A1C491C4B10B502611C4A42611C4A8C
:106C4000826102641B4A42641B4A82641B4AC1611E
:106C5000C2641B491B4A016202651B491B4A41620F
:106C600042651B491B4A0360816282651A4B1B49BE
:106C70001B4A4360C162C2651A4B1B491B4A8360B1
:106C8000016300231A4902661A4AC360044641633D
:106C90004266C36300F022FC174B2360204610BD00
:106CA000DC460020043C002088CE02085842002028
:106CB000083F00207040002080400020E841002074
:106CC000103C0020F8410020F83C00200842002041
:106CD000FC45002018420020F4450020603E0020C2
:106CE00028420020F8450020180E002038420020DD
:106CF0006C3C0020484200204CCF020808B53023ED
:106D000083F31188074B1B689A68996B8A4201D0FC
:106D1000824200D2986098630AF0E8FA002383F375
:106D2000118808BD683C00207FB51422002101A80D
:106D30001C46334E334D0BF001FF69464FF461435F
:106D40003148009309F0FEFE304BF2681A60B4201F
:106D50002C600AF039FC06F0F5FA0BF00DF92C4B1B
:106D60001C684FF4E131206CF7F742FA20690368A0
:106D70001B689847A06A03681B6898470A20FFF7BA
:106D8000BDFF0BF00DFA40B1224813210BF018FAA9
:106D900020494C2288180BF0A9FE1F4B28680122BD
:106DA0009A7303681B6898471C4B1B6813B11B6AD6
:106DB000DB0701D50BF0BEF9E06A03685B68984712
:106DC00038B1FAF7CBF94FF497724FF40061FAF744
:106DD000B1F9114804F074FCA06A0F4C03681B6BF6
:106DE0009847F3680E4ADA61B4200AF0EDFB286890
:106DF00003685B689847204604F062FCF7E700BF31
:106E000070790020883C002088700020683C0020B9
:106E100030100020643E0020FC450020E4460020A5
:106E20001CCE0208014B1868704700BF683C002068
:106E3000004870478C3C0020004870478C3C002084
:106E400038B500214B484C4C05F010F84B4A4C49E2
:106E500048480BF063FD4B4800F0E6FF02214A482A
:106E600005F004F84649454A47480BF057FD4748A6
:106E700000F0DAFF464800F0D7FF464800F0D4FFA4
:106E8000454800F0D1FF454800F0CEFF444800F0EF
:106E9000CBFF444800F0C8FF434801F061FB434B7F
:106EA000434A1A60434800F091FF4348FFF77CFED5
:106EB000324A424940480BF031FD414806F0C8FDD6
:106EC0002046404B40F8043B242200210BF036FEC4
:106ED00004F13400FFF7C4FC4FF0FF33274A3A496E
:106EE000E3642046394C0BF019FD302323714FF435
:106EF0007A73E38020464FF4FA632381344B40F8E1
:106F0000143BFFF7ADFC4FF4C8720023C4E93623ED
:106F10000023C4F80031012384F804311420F6F76B
:106F200021FF054610B16C2100F0B4FCC4F80051FB
:106F300000252849114A84F804512448264C0BF0B6
:106F4000EDFC264804F060FB254B264A83F89C5054
:106F500020461A60244B40F8043BFFF781FC204692
:106F6000064A22490BF0DAFCBDE838402048FFF71A
:106F70005FBE00BF083F0020103C0020E04600201C
:106F8000D96A01087040002080400020E8410020BC
:106F9000F84100200842002018420020284200202A
:106FA0003842002048420020F4450020F8450020E7
:106FB00010CF0208DC46002058420020596A010820
:106FC000043C0020ACD302085D6A0108F83C0020B4
:106FD000E8D40208556B01086C3C0020FC450020F9
:106FE000603E0020F4D9020828CF0208616A010837
:106FF0008C3C002070470000037933B108304FF417
:1070000048730860136001207047184670470000FD
:1070100000F5597001F036B910B50446007948B151
:1070200000F08CFAD4F86033C01AB0F5FA6F2CBFB8
:107030000020012010BD000008B5FAF78FF8A22249
:107040004FF40031FAF776F8002008BDF8B506468F
:10705000EAB1CC0801390A44C2F3CC050127A542A4
:1070600015D3632C0ED8630906EB830304F01F02CB
:1070700007FA02F1D3F828230A43C3F8282301347E
:10708000A4B2ECE7FFF7D8FF0028ECD1F7E7F8BD92
:10709000122110B513220446A0F858130548FFF733
:1070A00061FC04F5597001F035F910B9024800F09F
:1070B00017FA10BD50CF020876CF020810B501793B
:1070C000044671B9102200F54A700BF037FD2046D6
:1070D000FFF7DEFF022121710248BDE81040FFF7F3
:1070E00041BC10BD94CF0208B3F5487FF8B5074600
:1070F0000E4614461D460DD8C3F548739A4209D86A
:107100000834FFF7DBFF2A4639193046BDE8F8405E
:107110000BF0ECBCF8BD0000B3F5487F2DE9F3415E
:1071200005460E4690461C4622D8C3F54873994240
:107130001ED801F1080707442246394640460BF0A5
:10714000C5FCA8B12846FFF7B9FFF12205F54E713D
:1071500001A8F6F79BFF2246414638460BF0C6FCD5
:107160002846A2B23146FFF771FF01A8F6F7B0FF3B
:1071700002B0BDE8F081000037B505460C4601A815
:107180000121F6F769FFE10089B2082205F559707F
:1071900000F0BAFF044601A8F6F76AFF204603B0E4
:1071A00030BD00002DE9F74F0379044603B300F525
:1071B0004A7300F54E7853F8042B32B94345FAD19F
:1071C00000F0BCF9C4F8600312E000250123C5F308
:1071D0004A1604EB860605F01F07D6F8282303FAA3
:1071E00007F717421FFA85FA05D10135642DEED154
:1071F00003B0BDE8F08FED0008354FF488724146CA
:1072000001A8F6F743FF04EB050B6359C4F85033AC
:10721000DBF80430C4F8543301A8F6F759FF23799A
:10722000022B04F55479E3D151462046FFF7A4FF21
:107230000028DDD04FF49C72414601A8F6F726FFE6
:107240000822594648460BF041FC28B9D6F82833A5
:1072500023EA0703C6F8283301A8F6F739FFC7E782
:1072600038B51C46094BB0F858031B685B6B1546D4
:107270001A680144126818469047BDF81020411959
:1072800020460BF033FC012038BD00BF3010002039
:107290002DE9F743DFF8549006460F4605244FF4D6
:1072A0007A7101A8F6F7D8FED9F80080B6F858131D
:1072B000D8F8340003683944DB689847054630B194
:1072C00001A8F6F7D5FE284603B0BDE8F083D8F84C
:1072D0002800036801215B689847013C01A8F6F784
:1072E000C7FE14F0FF04DAD1EDE700BF3010002034
:1072F000034B1B68DB6A93F89C0080F00100704729
:10730000301000202DE9F04F2DED028B08EE103AE1
:107310002A4BD3F800900446D9F834000F4603688E
:10732000B4F858131B6885B039449046BDF840B096
:107330009847052500EB080A012103A8F6F78CFE03
:10734000D9F83400036818EE102A1E6951465B46CE
:10735000B047064640B103A8F6F78AFE304605B0AE
:10736000BDEC028BBDE8F08FD9F82800036801213D
:107370005B689847013D03A8F6F77AFE15F0FF0514
:10738000DAD12046FFF7B4FF0028E7D000F0D6F8A6
:10739000D4F85C3341F28832C31A9342DED9C4F880
:1073A0005C0304F5597000F0A3FF5B460090424671
:1073B00039460348FFF7D6FAD0E700BF3010002067
:1073C000B4CF020870B51D46164B1B6813B11B6A7B
:1073D000DB0725D5144B1E68F46A94F84630C3B910
:1073E000124BA4F84400DB6884F84610E26163B1F4
:1073F0009A6884F84720D96939B194F9483023B99B
:10740000042204F1480000F09DF8094B5B68C4E9D0
:107410000835F06A1321BDE8704004300AF0CABE96
:1074200070BD00BFE44600203010002070790020BD
:1074300000ED00E000B59BB0EFF3098168226846DB
:107440000BF054FBEFF30581074BC9B29A6BD86A76
:10745000986A986A986A986A986A9B6A059B7B20E2
:10746000FFF7B0FFFEE700BF00ED00E000B59BB006
:10747000EFF30981682268460BF038FBEFF30581D2
:10748000064BC9B29A6B986A986A986A986A986A21
:107490009B6A059BBF20FFF795FFFEE700ED00E02C
:1074A00000B59BB0EFF30981682268460BF01EFB24
:1074B000EFF30581064BC9B25A6B986A986A986ACD
:1074C000986A9B6A059BE320FFF77CFFFEE700BFFD
:1074D00000ED00E0FEE70000FEE70000704700005E
:1074E0000FB483B504AC0F4F54F8048B0E4EF9F76C
:1074F00035FE4FF4A5722021F9F71CFE42F21075FB
:10750000214640460194FFF725FA3846FFF72AFA4C
:107510003368986A036829465B6898474FF4FA75A0
:10752000EEE700BF49720208301000200AF04CBCA0
:10753000014B586A80B27047004001400AF080BC9D
:107540000AF026BCF8B50D460746114628461646F1
:107550000BF0E0FF864204468CBF421C02462946DF
:1075600038460BF0C3FA2046F8BD000070B5467BE4
:1075700005460EBB4468836804EB8404A40804F544
:107580000074E21A914288BFCC180C4B29681B6822
:10759000D86A0368621C1B6D984718B901232B73C6
:1075A000304670BDAB68C5E90004E21A00211844FA
:1075B0000BF0C4FA0126F3E70026F1E730100020B3
:1075C0000EB470B5017B85B0044619BBD0E9012328
:1075D0009A421BD0134B1E680AADD4E901212068E2
:1075E0000095521A099B03950144F06AF6F780FE54
:1075F00000280FDBD4E90123D21A82420FD8411CA4
:107600002046FFF7B3FF0028E7D103E0FFF7AEFF06
